:020000040800F2
:10000000F0FF0120499B0608BDF60008A5D50408AD
:10001000C19B0608C19B0608C19B060800000000A2
:10002000000000000000000000000000B9F6000819
:10003000B5F6000800000000B1F6000831A1040880
:10004000C19B0608C19B0608C19B0608C19B060808
:10005000C19B0608C19B06085DE9040889EA0408FB
:100060004DEA040811EA0408D5E90408357A0608BF
:10007000257A0608157A0608057A0608F179060831
:10008000DD790608C9790608C19B06080000000052
:1000900000000000000000000000000099E90408D2
:1000A0002962040875620408196204089962040848
:1000B00069620408596204084962040859880608FC
:1000C000618806084D88060855880608C19B060801
:1000D000C19B06084DA3040891A20408000000007B
:1000E00021E90408C19B0608790F010800000000FF
:1000F000000000000000000000000000B5790608C4
:1001000000000000D554060839620408C19B0608A7
:1001100000000000000000000000000000000000DF
:10012000A17906088D7906087979060865790608A7
:1001300051790608000000000000000000000000E7
:100140000000000000000000000000004DF000086A
:100150003D7906082979060815790608D5A104080D
:1001600041880608498806080000000000000000D9
:10017000000000000000000000000000000000007F
:1001800000000000C19B0608000000000000000005
:08019000C19B0608C19B060893
:08019800E896060001000000DA
:1001A0000E02010002000000286A00209C6A002064
:1001B0000000000060EE07081402010005000000C6
:1001C000183C0020A06A00200000000062EE070832
:1001D000130201000400000014260020A86A002079
:1001E0000000000068EE0708122001001100000066
:1001F000886A0020AC6A0020000000006CEE07084E
:100200000D1001004C00000024650020C06A002091
:10021000000000006DDC030809020100010000007D
:100220008C6400200C6B0020000000007EEE0708AC
:10023000FD0101002400000044640020106B002038
:100240000000000063490408FB01010001000000F8
:10025000845F0020346B00200000000079640508F2
:10026000FC01010009000000505E0020386B0020F6
:100270000000000081640508F7010100060000008D
:10028000445E0020446B00200000000080EE070860
:10029000F901010004000000405E00204C6B0020CA
:1002A0000000000051D80408160215003F000000AD
:1002B000B82F0020506B002000000000A16405084A
:1002C0003400010010000000705D0020906B0020E1
:1002D000000000000199020811020100080000005E
:1002E000485D0020A06B00200000000086EE07089B
:1002F0001212010004000000405D0020A86B0020E5
:10030000000000008EEE07081830010034000000E5
:100310000C5D0020AC6B0020000000008574050817
:10032000000201000B00000090590020E06B00204B
:1003300000000000C5640508FF1101000600000070
:100340003C590020EC6B00200000000059640508B7
:10035000081203000F00000048590020F46B002031
:1003600000000000CD640508FA0101000300000050
:100370002C530020046C0020000000009964050844
:100380000A9001002C000000EC4A0020086C0020BC
:10039000000000004D0A0208204201000600000093
:1003A00048490020346C0020000000002599020814
:1003B0000610010024000000D42E00203C6C002018
:1003C00000000000496505080C020100040000005F
:1003D000E0420020606C0020000000006964050815
:1003E000FE01010014000000903D0020646C00201C
:1003F000000000001D640508261001000E0000002A
:10040000B0D80020A0D80020000000004921010839
:100410000B3001001A00000060D10020F0D800204D
:100420000000000094EE07081F50010024000000A7
:1004300084D000200CD9002000000000B0EE070896
:10044000050201000400000058D3002030D900202C
:1004500000000000D4EE0708030101000A000000BC
:10046000B0D0002034D9002000000000F11B0108AA
:10047000010201000B00000010DF002020F000202E
:1004800000000000B564050802020100030000003E
:1004900008DF00202CF00020000000000000000019
:1004A0001B02010010000000F4DE002030F00020EC
:1004B00000000000356505081B1001000C0000005D
:1004C00040DC002040F0002000000000E58501082D
:1004D00021020100F000000074DA00204CF000203E
:1004E00000000000299B01083710010030000000C7
:1004F000CCDF00203CF1002000000000D8EE07080F
:100500001610010006000000B8DE00206CF100208B
:100510000000000008EF07082F1001002200000073
:10052000FCEF002074F10020000000000EEF07082F
:100530002322010010000000D0DD002098F10020EF
:100540000000000030EF07081E0001000900000055
:10055000C4DD0020A8F100200000000040EF0708E3
:10056000052001000C00000088DE0020B4F100200E
:10057000000000004CEF0708FD0701007C000000B0
:1005800040D90020C0F1002000000000697F010870
:10059000F59101006C00000000DA00203CF2002020
:1005A00000000000BD92010823200100100000009F
:1005B0002EDF0020A8F2002000000000A50A02089B
:1005C000F62101000C00000044FF00202000012063
:1005D0000000000058EF07081C0202001C00000089
:1005E000D4FE00207000012000000000CD6F05083F
:1005F0002830010016000000F0FE00208C000120D1
:1006000000000000D91702081400010005000000D6
:10061000CCFE0020A40001200000000064EF0708C9
:10062000012001000C000000C8F70020AC000120F0
:10063000000000006AEF07080C400600E40000001C
:10064000F8F50020B80001200000000099D7030849
:100650000E200300BC01000014F400209C010120C6
:100660000000000039990208130001000400000096
:10067000D0FB0020580301200000000078EF07089D
:10068000010101000400000058F300205C03012078
:100690000000000000000000000101000400000054
:1006A00050F3002060030120000000007CEF0708E9
:1006B00002010100030000004CF30020640301204C
:1006C00000000000D9D70308220201001C0100002D
:1006D000B8F9002068030120000000003D740508FF
:1006E0001A0001000E0000005C110120B011012071
:1006F0000000000080EF07081500100070000000E7
:10070000D80F0120C01101200000000000000000EF
:100710000300010001000000D00F01203012012071
:1007200000000000000000002A0008006000000037
:10073000E00A01203412012000000000D9980208CC
:100740002C00040010000000A412012094120120CB
:1007500000000000A19602082B00120024000000F7
:10076000D8120120B4120120000000007596020882
:100770002920140078000000580D0120FC120120EF
:10078000000000000000000019020100100000003D
:10079000FC0C01207413012000000000A564050872
:1007A000F82101000600000050170120F81F012069
:1007B000000000008EEF070810100100020000008A
:1007C000F4150120002001200000000094EF07082C
:1007D00019000100050000008413012004200120FD
:1007E0000000000096EF0708020001000C00000066
:1007F000DC2101209C2301200000000000000000FB
:1008000025201E002C010000E8210120A823012042
:10081000000000000000000029020100400000006C
:1008200024210120D4240120000000009CEF0708AF
:100830000A020100140000001C20012034250120C0
:100840000000000065D7030828020400040000002F
:10085000402F01204C3001200000000031650508C8
:1008600027020400040000003C2F0120503001202A
:1008700000000000256505081F02080010000000A8
:10088000902C012054300120000000003564050840
:100890001A0201003C0000006C2601206430012097
:1008A00000000000E1740508031201003D00000093
:1008B0002C2C0120A030012000000000DCEF0708F4
:1008C000381001000100000064250120E030012003
:1008D000000000001AF00708040008008000000073
:1008E000AC3101202C33012000000000000000008A
:1008F0000B2201003D0000007C3B0120384201201A
:10090000000000001CF007082A0201000B00000094
:10091000B433012078420120000000005AF007089B
:100920001D0202000600000008420120844201204E
:10093000000000000000000006120300120000008A
:10094000184201200C530120000000009970050896
:100950002700010004000000D03B012020530120AB
:100960000000000066F0070810020100010000000E
:10097000188D0120148D0120000000006AF0070886
:100980000403090412010002EF02014083045632FD
:1009900000020102030100001201000202020040F5
:1009A000830440570002010203010000FFFFFFFF24
:1009B00000600240106002400000000000000000E3
:1009C000000B00000000000000000000000000001C
:1009D00000600240286002400100000000000000AA
:1009E000060C0000000000000000000000000000F5
:1009F0000060024040600240020000000000000071
:100A0000100D0000000000000000000000000000C9
:100A10000060024058600240030000000000000037
:100A2000160E0000000000000000000000000000A2
:100A300000600240706002400400000000000000FE
:100A4000200F000000000000000000000000000077
:100A500000600240886002400500000000000000C5
:100A60002610000000000000000000000000000050
:100A700000600240A060024006000000000000008C
:100A80003011000000000000000000000000000025
:100A900000600240B8600240070000000000000053
:100AA000362F0000000000000000000000000000E1
:100AB00000640240106402400000000000000000DA
:100AC00000380000000000000000000000000000EE
:100AD00000640240286402400100000000000000A1
:100AE00006390000000000000000000000000000C7
:100AF0000064024040640240020000000000000068
:100B0000103A00000000000000000000000000009B
:100B1000006402405864024003000000000000002E
:100B2000163B000000000000000000000000000074
:100B300000640240706402400400000000000000F5
:100B4000203C000000000000000000000000000049
:100B500000640240886402400500000000000000BC
:100B6000264400000000000000000000000000001B
:100B700000640240A0640240060000000000000083
:100B800030450000000000000000000000000000F0
:100B900000640240B864024007000000000000004A
:100BA00036460000000000000000000000000000C9
:100BB000000004010000000000000002100000001E
:100BC000070000007D000000F45C0708FC5C0708DB
:100BD0000000000061D80308A086010004000000A6
:100BE0000000000000000000000000000000000005
:100BF00000000000000000000000000000000000F5
:100C0000000000000000000000000000F45C070885
:100C1000045D070800000000A5580408E803000070
:100C200004000000000000000000000000000000C0
:100C300000000000000000000000000000000000B4
:100C400000000000000000000000000000000000A4
:100C50000C5D070800000000000000008D3B030849
:100C60007D000000FF000000000000000000000008
:100C70000000000000000000000000000000000074
:100C80000000000000000000000000000000000064
:100C900000000000C0E9070800000000000000009C
:100CA000D56C03087D000000FF000000000000007C
:100CB0000000000000000000000000000000000034
:100CC0000000000000000000000000000000000024
:100CD0000000000000000000707107080000000024
:100CE00000000000418E03087D000000FF000000AE
:100CF00000000000000000000000000000000000F4
:100D000000000000000000000000000000000000E3
:100D1000000000000000000000000000145D070853
:100D2000000000000000000069530408E803000010
:100D300003000000000000000000000000000000B0
:100D400000000000000000000000000000000000A3
:100D50000000000000000000000000000000000093
:100D6000185D07080000000000000000C9420308E9
:100D70001027000003000000000000000000000039
:100D80000000000000000000000000000000000063
:100D90000000000000000000000000000000000053
:100DA0000000000098E507080000000069920208B2
:100DB000657204085F760000050000000000000076
:100DC0000000000000000000000000000000000023
:100DD0000000000000000000000000000000000013
:100DE000000000000000000064E9070800000000A7
:100DF0000000000009D604081027000001000000D0
:100E000000000000000000000000000000000000E2
:100E100000000000000000000000000000000000D2
:100E2000000000000000000000000000245D070832
:100E30000000000000000000F9470408E80300007B
:100E4000050000000000000000000000000000009D
:100E50000000000000000000000000000000000092
:100E60000000000000000000000000000000000082
:100E7000305D07080000000000000000D9DA030818
:100E8000204E0000030000000000000000000000F1
:100E90000000000000000000000000000000000052
:100EA0000000000000000000000000000000000042
:100EB00000000000405D0708000000000000000086
:100EC000D5D80308204E00000300000000000000F9
:100ED0000000000000000000000000000000000012
:100EE0000000000000000000000000000000000002
:100EF0000000000000000000505D07080000000036
:100F0000000000000D4A0408400D0300030000002B
:100F100000000000000000000000000000000000D1
:100F200000000000000000000000000000000000C1
:100F3000000000000000000000000000605D0708E5
:100F40000000000000000000D90E04081027000077
:100F50000100000000000000000000000000000090
:100F60000000000000000000000000000000000081
:100F70000000000000000000000000000000000071
:100F8000685D0708000000000000000055E401084B
:100F90001027000003000000000000000000000017
:100FA0000000000000000000000000000000000041
:100FB0000000000000000000000000000000000031
:100FC000000000006C5D0708000000000000000049
:100FD0005D5B0208A0860100010000000000000027
:100FE0000000000000000000000000000000000001
:100FF00000000000000000000000000000000000F1
:101000000000000000000000745D07080000000000
:1010100000000000D551040850C30000010000008A
:1010200000000000000000000000000000000000C0
:1010300000000000000000000000000000000000B0
:101040000000000000000000000000007C5D0708B8
:101050000000000000000000C14D0408A86100006D
:10106000010000000000000000000000000000007F
:101070000000000000000000000000000000000070
:101080000000000000000000000000000000000060
:10109000885D07080000000000000000A1A7040808
:1010A000A00F000001000000000000000000000090
:1010B0000000000000000000000000000000000030
:1010C0000000000000000000000000000000000020
:1010D00000000000945D0708000000000000000010
:1010E0007DD0010810270000010000000000000072
:1010F00000000000000000000000000000000000F0
:1011000000000000000000000000000000000000DF
:101110000000000000000000A05D070800000000C3
:101120000000000065C801081A410000010000002D
:1011300000000000000000000000000000000000AF
:10114000000000000000000000000000000000009F
:10115000000000000000000000000000A45D07087F
:101160000000000000000000291C010810270000FA
:10117000010000000000000000000000000000006E
:10118000000000000000000000000000000000005F
:10119000000000000000000000000000000000004F
:1011A000B05D070800000000000000007D33020869
:1011B00050C300000100000000000000000000001B
:1011C000000000000000000000000000000000001F
:1011D000000000000000000000000000000000000F
:1011E00000000000B45D07080000000000000000DF
:1011F000A9280108400D03000000000000000000C5
:1012000000000000000000000000000000000000DE
:1012100000000000000000000000000000000000CE
:101220000000000000000000BC5D07080000000096
:10123000000000009DD80308400D030000000000DE
:10124000000000000000000000000000000000009E
:10125000000000000000000000000000000000008E
:10126000000000000000000000000000C45D07084E
:1012700000000000000000003DF4010850C3000021
:10128000030000000000000000000000000000005B
:10129000000000000000000000000000000000004E
:1012A000000000000000000000000000000000003E
:1012B000D05D0708000000000000000049E90308B5
:1012C00040420F000000000000000000000000008D
:1012D000000000000000000000000000000000000E
:1012E00000000000000000000000000000000000FE
:1012F00000000000DC5D07080000000000000000A6
:101300007DE0030850C30000000000000000000062
:1013100000000000000000000000000000000000CD
:1013200000000000000000000000000000000000BD
:101330000000000000000000E85D07080000000059
:1013400000000000916C0108102700000000000060
:10135000000000000000000000000000000000008D
:10136000000000000000000000000000000000007D
:101370000000000000000000000000009D83000845
:1013800099830008958300088983000885830008F5
:10139000918300088D830008000000008D8D0008F7
:1013A000E1AD0008FD8C000821AF0008658E000843
:1013B0000D840008F9830008DD8300087DA500087E
:1013C0008D90000849920008B992000835930008F2
:1013D0008D94000859140108E5830008D58300089E
:1013E000010000000000803F01410108054601089E
:1013F0007D410108F5140108D916010805150108F9
:1014000021150108CD140108BD14010800000000D9
:101410000000000009022000010104C0320904009C
:10142000000208065005070581024000000705017B
:101430000240000009026400030100C032090400F8
:1014400000010300000009211101000122360007FC
:1014500005830309000A080B0102020201000904C6
:101460000100010202010005240010010524010011
:101470000204240202052406010207058203080073
:10148000FF09040200020A000000070501024000F3
:10149000000705810240000009024300020100C06C
:1014A00032090400000102020100052400100105B8
:1014B000240100010424020205240600010705821C
:1014C000030800FF09040100020A000000070501EB
:1014D000024000000705810240000000FF000000FC
:1014E000140000FF0000000000000000AA550701E2
:1014F000000001AA55050100002D202D2D202D2DC5
:101500002D2D202D2D2D2D000000000000000000AD
:10151000000000000000000008000000D0CF060816
:10152000FF1FFF1F05010905A101A10005010930E9
:10153000093109320933093509340936093715816A
:10154000257F7508950881020509190129081500EC
:101550002501950875018102C0C000000902220022
:10156000010100E032090400000103010200092129
:10157000110100012236000705830309000A00005B
:101580000000000001020304010203040607080929
:10159000AA550B010000AA5505010000AA55090231
:1015A000000000AA5503009F01000000C0120000C7
:1015B000E8D8002000000000C0D800200000000093
:1015C000010000000100000000000100E0017EFFBA
:1015D000FFFFFFFFFF000000FFFFFFFF0801FF010B
:1015E0000100000091FF0108000000000000000061
:1015F00090D7060800000000000000000000000076
:1016000068F0060800000000000000000000000074
:1016100020F10608000000000000000000000000AB
:10162000CCF006080000000000000000110B0208CA
:10163000C6F8002001010000951F0208000000000C
:1016400000000000F4F10608F52202080000000086
:1016500000000000ACF106082D202D2D202D2D2D91
:101660002D202D2D2D0000000000000000000000A6
:101670000000000000000000FFFFFFFF3D10020817
:101680000000000000000000F8EF06080100000064
:10169000FA0000000100000001000000010100004C
:1016A00000010101000000003CF700200000F401EF
:1016B000010000003AF700200000F40101000000E2
:1016C00038F700200000F4010100000036F7002088
:1016D0000000F4010100000034F700200000F401D4
:1016E0000100000032F700200000F40101000000BA
:1016F00030F700200000F401010000009D080208FE
:101700006108020800000000CCD9060820F700207C
:10171000053201002EF700206400F40101000000F2
:101720002CF700206400C409010000001EF700200F
:10173000E803D007010000001CF70020E803D007F1
:10174000010000001AF70020E803D00701000000A4
:1017500018F700201E00B80B0100000026F700203B
:1017600005000F000100000028F7002003000A0018
:101770000100000016F700201E00F4010100000027
:101780002AF700200200000058DA060814F70020AB
:10179000140064000100000022F700203200E8037A
:1017A0000100000012F700200000C8000100000046
:1017B000F5F5002000C80100F4F5002000500100FC
:1017C000F3F50020005A0100F1F5002002000000AE
:1017D00064DA06083C68070844680708C4F8002073
:1017E0000100C40900000000C2F800200100C40983
:1017F00000000000C0F800200100C4090000000043
:10180000BEF800200100C40900000000BAF8002062
:101810000100C40900000000BCF800200100C40958
:1018200000000000B8F800200100C409000000001A
:10183000B6F800200100C4090000000077F3002082
:1018400000C8010076F3002000C8010074F30020F6
:101850000000FFFF0A00000072F300200100C80032
:101860000100000070F300203200307532000000EB
:101870006EF300207EFF1400050000006CF30020D2
:1018800005002C01050000006BF30020055A05003F
:1018900068F3002000FF01006AF30020020000004E
:1018A000EC0F002066F3002003000000CCD10608F6
:1018B00067F3002000FF010069F300200200000030
:1018C000EC0F002065F3002003000000CCD10608D7
:1018D000C4F20020FF7F0100C0F2002000000000E1
:1018E000FFFFFFFF01000000BCF20020000000002D
:1018F000FFFFFFFF01000000B8F200200000000021
:10190000FFFFFFFF01000000F10702088107020846
:101910000000000070DA0608D8F70020EE02CA08BE
:1019200001000000D6F7002000C80100640000009C
:10193000D5F7002000C8010064000000D4F70020A3
:10194000020000007CDB06085EF300200000803E01
:10195000050000005CF3002080C1803E050000000F
:1019600056F300200083007D0500000054F30020A2
:1019700080C1803E050000004FF3002000FF010001
:1019800048F300206400F4010100000046F3002049
:101990006400F4010100000044F300206400F4013D
:1019A0000100000042F300200400000088DB06086C
:1019B00041F30020020000009CDB060803F4002035
:1019C0000D000000A8DB060800F400200064010000
:1019D000FEF30020320010270A000000FCF3002074
:1019E0000D000000A8DB0608FBF300200D0000003E
:1019F000A8DB0608FAF3002002000000E0DB06087E
:101A0000000000000000000000000000ECDB060801
:101A1000DDF700204200000024DC0608DBF7002090
:101A20000300000030DD0608DCF7002004000000A1
:101A300040DD060805F400200300000054DD060820
:101A400004F400200300000054DD0608E2F5002045
:101A5000000A0100E0F500200000E803010000009A
:101A6000DEF500200000E80301000000DCF50020A6
:101A7000000A0100DAF500200000E8030100000080
:101A8000D8F500200000E80301000000D0F5002098
:101A90000000E80301000000D6F500200000E80384
:101AA00001000000D4F500200100E803010000005F
:101AB000D2F5002001050100F0F500200200000031
:101AC00064DD0608EEF500200000F40101000000CE
:101AD000ECF500200000F40101000000EAF5002010
:101AE0000000F40101000000E8F500200000F4010E
:101AF00001000000E6F500200000E80301000000FE
:101B0000E4F500200000E8030100000002F70020D7
:101B1000006401000A00000001F7002000640100D9
:101B20000A000000EFF6002019640100EEF6002024
:101B30000200000070DD0608ECF60020E803D00784
:101B40000A000000EAF60020006401000A0000001C
:101B5000DFF6002000640100DEF6002000640100D2
:101B6000E6F60020006401000A000000E5F600200F
:101B7000006401000A000000E4F600200064010097
:101B80000A000000E9F6002000FF01000A00000042
:101B9000E8F6002000FF01000A000000E7F6002040
:101BA00000FF01000A000000E3F6002001FF010031
:101BB0000A000000E2F6002001FF01000A00000018
:101BC000E1F6002001FF01000A0000000EF40020F1
:101BD0000000F401010000000CF400200000E80304
:101BE000010000000AF400200000E80301000000EA
:101BF00008F400200000E8030100000006F40020C3
:101C00000000E8030100000017F900200096010021
:101C100010F9002000C801000FF900200064010045
:101C20000EF90020006401000DF90020006401009D
:101C30000CF90020006401000BF90020FF080100EE
:101C40000AF9002001640100F9050208BD05020837
:101C5000000000007CDD060813F9002001320100BD
:101C600012F9002001000000ECDD060811F9002047
:101C700004000000F4DD060809F9002000960100C8
:101C800008F900200064010006F900201400E803B0
:101C90000100000004F90020000030750A00000077
:101CA00002F9002000C8010001F9002000C801006D
:101CB00000F9002000C80100FFF8002000320100F8
:101CC00016F900200014010015F90020004B010056
:101CD00014F900200400000008DE0608FEF80020C9
:101CE000006401000A0000000DF7002032C8050062
:101CF0000A0000000CF700200100000018DE0608B2
:101D00000FF7002032C805000A0000000EF700207F
:101D10000100000018DE06080BF7002032C805009D
:101D20000A0000000AF7002032C805000A0000007F
:101D300009F7002032C805000A00000008F700205B
:101D400032C805000A00000007F7002032C805006D
:101D50000A00000006F7002032C805000A00000053
:101D600005F7002032C805000A00000004F7002033
:101D70000200000020DE060826F900200000D0073F
:101D80000100000020F9002000C801001FF9002018
:101D900000C801001EF9002000C8010024F900203D
:101DA0000000D007010000001DF9002000C801005C
:101DB0001CF9002000C801001BF9002000C8010028
:101DC00022F900200000D007010000001AF90020CD
:101DD00000C8010019F9002000C8010018F900200E
:101DE00000C80100A10302088903020819100208B3
:101DF0002CDE0608F7F30020005A0100F6F300205D
:101E000000C80100F4F30020E803D007010000003F
:101E10000000000000000000510B0208C8DE0608A8
:101E200064F30020030000001CDF060863F30020B9
:101E30000003010062F3002000030100C502020854
:101E400079020208000000002CDF060839020208AF
:101E5000F101020800000000C8DF060811030208B3
:101E6000FD0F02080000000048E0060860F30020B3
:101E7000010301005DFF01083DFF010800000000B3
:101E8000BCE30608790902084D09020800000000B9
:101E90003CE4060861010208090102080000000094
:101EA000ACE40608B1030208792A02080000000029
:101EB00064E50608ED140208A50902080000000008
:101EC0000CE6060801040208000000000000000003
:101ED000A8E60608E50402088504020800000000E0
:101EE0000CE706088105020845050208000000000D
:101EF000C4E706084973020835060208000000001E
:101F000050E8060811F70020010601004904020804
:101F1000150402080000000068E90608657202085E
:101F2000C111020800000000D8E90608DD06020819
:101F3000650602080000000054EB06088D730208D5
:101F4000A11202080000000050EC060810F7002063
:101F500001030100590302082903020800000000E0
:101F600024ED06089D0F020800000000000000009C
:101F700088ED0608B9010208E50F0208000000001C
:101F800024EE060800000000000000000000000031
:101F9000C0EE060859070208991302080000000065
:101FA00040EF0608000000000000000000000000F4
:101FB00068F1060820D100209CFF2C0100000000E1
:101FC00068FB0020E0150C17000000006AFB0020F1
:101FD00002000000A0F106083CF3002088136F17F0
:101FE000010000003EF3002088136F17000000007E
:101FF000A66900200000000000000000A469002085
:102000000000000000000000A269002000000000A5
:1020100000000000A0690020000000000000000097
:102020009E69002000000000000000009C69002064
:102030000000000000000000C40D002000000000AF
:1020400000000000C5F200200300000090F2060826
:1020500034F3002088136F17010000004ED30020D6
:1020600088136F17000000004900020800000000FC
:1020700000000000A0F2060881F800200100000026
:10208000F4F2060850D300200100000000F3060817
:1020900046D300200200000008F3060800000000FC
:1020A000000000000000000014F3060831000208E0
:1020B0000000000000000000B0F30608000000006F
:1020C000000000000000000004F40608000000000A
:1020D000000000000000000074F4060840F3002037
:1020E00002000000ACF406084AD30020E0150C17EB
:1020F00000000000040601205806012001F11F3FE6
:10210000D60101FF01000000789C0020FFFFFFFFC7
:102110000000803F00000000000000000000000000
:1021200000000000000000000000000000000000AF
:1021300000000000000000000000803F00000000E0
:102140000000000000000000010000000000803FCF
:102150000000000000000000000000000000803FC0
:102160000000000000000000000000000000FA4332
:102170000000FA43E910040800000000000000001D
:10218000000000000000803F000000002425012026
:1021900008000000000000001425012008000000D5
:1021A0002000000059400108E9150108F13F01082D
:1021B00000000000B9140108D9480108413F010896
:1021C0008D3B0108000000000000000079140108A8
:1021D000AD830008A1830008898C0008A58C000845
:1021E0006D8C0008518C0008358C000811400108E6
:1021F000C5150108453F01080000000091140108C1
:10220000913B0108153F0108ED3A0108000000006C
:102210000000000085140108FFFFFFFF685E0C004E
:1022200002FF0100A00F0000B80B000002FFFF0139
:10223000FFFF00008CE5070800000802050303000B
:102240000000000094E507080100080205040300EF
:10225000000000007C8807080200FE010110030056
:1022600000000000B06B0708030014020003000028
:10227000000000009CE5070804001F02020008009F
:1022800000000000A4E5070805001F020201080085
:1022900000000000FFFFFFFF1A0300000000000025
:1022A000000000000000000000000000000000002E
:1022B00000000000040309041201000200000040B5
:1022C0008304205700020102030100000002906015
:1022D00006000000881300000204089001049070BA
:1022E00006000000102700000204088B0205908001
:1022F00006000000204E000000040A8803069090AB
:1023000006000000409C000000040A8500001850F0
:1023100006000000D007000001040C9701011860BE
:1023200007000000A00F000002040E9402031870C2
:10233000070000000A1A000003040C90030518901F
:1023400006000000204E000000040C8B517B0508A5
:10235000257B0508C97A050815660508E57A05088C
:10236000897A050811660508781C0020417C05085B
:10237000617C0508317C0508F5650508ED7B0508DD
:10238000A57B0508E5650508541C00205D7505085A
:10239000FD650508F9650508F1650508AD750508D1
:1023A000ED650508E9650508544E070875480108FC
:1023B000A5150108554701080000000000000000B5
:1023C000ED3E0108FD3D0108000000000000000096
:1023D000000000006D1401089D660508916605085F
:1023E000B17C0508CD7C050849660508957C050883
:1023F000797C0508FFFFFFFF1F0000001C000000A4
:102400001F0000001E0000001F0000001E00000052
:102410001F0000001F0000001E0000001F00000041
:102420001E0000001F0000000068214C0100000099
:10243000F45707080100000050C3000000800202AA
:102440001F00000053544D202020202050726F6444
:10245000757420202020202020202020302E303194
:10246000008002021F00000053544D202020202035
:1024700050726F647574202020202020202020209E
:10248000302E3031010101FF01000000F401000095
:10249000FFFF0000B01C0020000000000000000052
:1024A000000000000000000000000000000000002C
:1024B000000000000000000000000000000000001C
:1024C000000000000000000000000000000000000C
:1024D00000000000000000000000000000000000FC
:1024E00000000000000000000000000000000000EC
:0824F0000000000000000000E4
:08280000082800080040000850
:10800000134B0268196821EA02011960596821EAD4
:108010000201596019680A431A609968026821EAE6
:1080200002019960D96821EA0201D96041791029D9
:1080300007D001F1804303F59E3319680A431A60A3
:108040007047996811439960D9680A43DA607047AC
:10805000003C0140F0B401292A4C2B4D23684FF01D
:10806000000694BF00270127EE626662A66267637E
:10807000676B47EA42076763EE63EC6B002A38D10F
:1080800044F49574EC631C6824F001041C601C68C3
:10809000E407FCD4490289085960D8601968EAB934
:1080A00021F04001196019498B421DD018494FF445
:1080B0007410C860196841F01E011960596941F0D7
:1080C00080015961196841F00101196022B90E4A15
:1080D000D36A43F00803D362F0BC704741F040011B
:1080E00019600A498B42E1D14FF0746041F8500C9D
:1080F000E0E744F01A04EC63EC6A44F00804EC6234
:10810000C1E700BF101D0020002C01405864024050
:10811000006402400A4BB3F89C204AB1D3F898108F
:10812000C889904204D0D3F894000280CA8100BF6D
:10813000D3F8A03013B11A689B885383704700BFEF
:10814000101D00201248002302461178032902F175
:10815000060218D00133062BF7D10E4AD2F8D430DC
:10816000052B0FD0591C03EB4303C2F8D41000EBCE
:108170004303032040F2EB3140F2FF321870598084
:108180009A807047704703EB430300EB4303F0E72B
:10819000C01D0020101D002070B4C3080D4CE25C0F
:1081A00000F00706B24004EBD004D2B20020C6F1C2
:1081B00008038B4228BF0B46C3F108052A419840AB
:1081C000C91A40EA02004FF0000614F8012FEED160
:1081D00070BC7047881D0020084AD2E936319942A8
:1081E0000AD0D118013391F8E0100170C3F30A03EB
:1081F000C2F8D8300120704700207047101D0020C1
:10820000064AD2F8E038D2F8E428934294BF4FF4FB
:1082100000600020013B9B1A18447047101D00208D
:10822000012380F85130704707B501A8FFF7D4FF4C
:108230000028FAD09DF8040003B05DF804FB044B5D
:10824000D3E93603984288BF03F50063181A7047D4
:10825000101D002001207047024BC3F8E828C3F826
:10826000EC187047101D0020024BC3F8F028C3F82B
:10827000F4187047101D00207047704730B4134D3C
:10828000D5E936239A4286BF03F50064A21A9A1AEA
:108290000A44B2F5006F13D8A9B101444A1E01384F
:1082A00010F8014FE918824203F1010381F8E04020
:1082B000C3F30A03F4D1C5F8DC30002030BC7047AA
:1082C000022030BC70470846F8E700BF101D0020B0
:1082D000212838B50C4605D022282ED0202813D0CE
:1082E000002038BD0029FBD0072AF9D11A4BD3F85A
:1082F000F80893F8FC1893F8FD2893F8FE382060EE
:1083000021716271A371EBE70029E9D0072AE7D157
:10831000114DD5F8EC381BB10968D5F8E808984735
:10832000206821796279A379C5F8F80885F8FC18E6
:1083300085F8FD2885F8FE38D2E70029D0D0022A3A
:10834000CED1054AD2F8F438002BC9D00988D2F82A
:10835000F0089847C4E700BF101D0020024B002022
:10836000C3F80009704700BF101D0020044B002017
:108370000522C3F80029C3F8F408C3F8EC087047D5
:10838000101D0020704700BF704700BF704700BF3E
:10839000704700BF704700BF704700BF704700BF05
:1083A000042301480B8070479801002010B4074A4D
:1083B000074B92F80409122403F114020C800128DF
:1083C0000CBF184610465DF8044B7047101D002086
:1083D0009C01002000487047701D00200048704735
:1083E000701D0020034B93F85C00032894BF00200D
:1083F00001207047101D0020034B93F85C000328F8
:1084000094BF002001207047101D0020034B93F8FB
:108410005C00003818BF0120704700BF101D00200D
:10842000A0B182680D4B12B107229A70704719787B
:10843000DA6003294FF004000CBF80214FF48071F3
:10844000C3E901111A611A7598707047034B41F224
:10845000E47101225A545A70704700BFE0B0002006
:108460000378022B10D0006908B9012070470C4B2B
:108470001B78032B0EBF0B4B80B24FF6F77398425D
:1084800094BF0020012070470549436841F650021F
:108490008A58B3EB422F2CBF01200020704700BF49
:1084A000E0B00020F7FFFF0F0378022B14D030B4A8
:1084B000104A4368006941F6480402F5C251155953
:1084C000096841F63C042B4012595B0A023801FB53
:1084D0000030104430BC7047064B426841F634010E
:1084E00041F630005958185800EB410000EB52207B
:1084F000704700BFE0B0002008B5084BD3F89420C7
:1085000013899907FCD513891B06F9D40A203EF07C
:10851000B7FDBDE80840024846F0D4BC101D00205D
:10852000A01D00200E4B70B5D3F8944041F034FDEF
:10853000A389054642F20F7623899B0705D520467D
:10854000FF21BDE870405FF07DBA41F025FD401B82
:10855000B042F1DD204646F0F9FCC0B270BD00BF6C
:10856000101D0020F8B5194F0023BB65FFF7DAFF97
:10857000D7F8944041F010FDA389054642F20F76EA
:1085800023899B0710D52046FD215FF05BFAFFF79A
:10859000C9FFFF2811D1FFF7C5FFFF280DD1042324
:1085A000022087F85C30F8BD41F0F6FC401BB04279
:1085B000E6DD204646F0CAFCE9E7D7F80839FB6457
:1085C0000923002087F85C30F8BD00BF101D002093
:1085D000F8B51A4C94F80C39002BFBD159B301446F
:1085E0004E1E451ED4F8E428D4F8E01815F8017F93
:1085F000531CC3F30A038B422CBF4FF400600020CE
:10860000C91A22440144012982F81079C4F8E438D7
:108610000FD1012041F0ECFCD4F8E038D4F8E41894
:108620008B4294BF4FF4006200225B1A1344012B6B
:10863000EFD0B542D6D10020F8BD00BF101D0020FC
:1086400010B5094CD4F80039084611465BB1D4F88E
:108650000039052B07D1002AD4F8083903DDFFF7CC
:10866000B7FFD4F8083910BD101D002010B590F8E0
:108670005010002380F8503081B10B4CD4F8002901
:1086800072B1D4F80029052A0CD13C30D4F808394D
:10869000FFF79EFFD4F80839012010BD0120FCE748
:1086A0001046FAE71846F8E7101D0020002280F86F
:1086B0005120DBE790F85020531C0244DBB280F8D5
:1086C000503082F83C1090F851200AB1132B00D999
:1086D000CCE770472DE9F84F454B98420ED003F593
:1086E00068530833984247D0424B0020C3E91D002D
:1086F000A3F87000A3F87C00BDE8F88F3D4C3E4F16
:10870000DFF800810223A36104F11C060025FB6A47
:10871000AB42294605F1010503D0D4F88C0052F094
:10872000FBFE94F89030D4F88C2086F82430326226
:108730003046414653F022F9A3699D4206F12806CE
:10874000E5DB002384F87E30D4E90903A169228C9B
:10875000A58DC4F8943012FB01F203FB01F3A4F8D9
:108760007020618C254AA4F87C50C4E91D03A4F84C
:108770007210E2660120BFE71E4C1F4F0223A36167
:1087800004F11C054FF0000B4FF4806A4FF04009D4
:108790004FF40068FA6A01265A455946B34403D09B
:1087A000D4F88C0052F0B8FED4F88C1094F89020D5
:1087B000296285F824204FF400314FF00062C5E9AA
:1087C0000212A5F804A0A5F81090A5F80680AE74D2
:1087D000FFF7B8FC28466E7653F022F8A269084BE2
:1087E00045F8283B9345D5DB84F87E60ACE700BFB5
:1087F0001971EF00082E00209801002084CC060893
:1088000058CC06081940EF002DE9F04FD04ED14D5D
:1088100086468C4617460FCE05F198042DED068B43
:108820000FC40FCE0FC496E8070089B095F8CE307C
:10883000039784E80700CDE904EC042B00F24281A1
:10884000DFE813F0A80140013B010500B8019FEDEE
:10885000C28ADFEDC28AC249C5F8B410C149C24B11
:10886000C24AC5F8B0100399002918BF134638EE64
:10887000887AF5EE006AC6EE879ABD4EC5F8BC3020
:10888000A6F1120B06F1C0080027DFEDC17A9FEDBB
:10889000B99A28EE278AB0EE67AA059BBB4200F082
:1088A00006811BF8019B05EB090309F1010993F807
:1088B000D3405FFA89F9002C00F07F81002203E0A9
:1088C0000132152A00F0798102EB4201530018F8B9
:1088D0000100A042F4D12944029391F8B11100297A
:1088E00000F0738120463DF021FF824600683DF094
:1088F000C1FE9AF805103DF039FF90F800C0BCF1B8
:10890000000F40F05A81029BE9182309013B032222
:10891000042B81F8F19181F8F02104F00F0000F2AE
:10892000FC80954C04EB4301B1F884C04CFA00F193
:1089300011F0010100F00981012101FA00F0013874
:1089400000EA0C00029360F051FF029BDFF83CC28A
:108950002344032293F8903018440CEBC003736156
:108960009A7183F807905CF830009AF8082000F1BB
:108970003F4C0CF57E0C04EB9C24012194F89840AC
:1089800004F01F0C6409032C01FA0CF100F0D680EE
:10899000042C00F0CC80022C00F0C2809B8806934F
:1089A000B3FA83F3C3F11F03C3F3CC0100EB8101DE
:1089B00003F007030C6A9B004FF00F0C0CFA03FC4A
:1089C00024EA0C040C620C6A02FA03F323430B62E0
:1089D000022306A907930CF08FFA039B002B76D095
:1089E000B5F8CC30D5F89C1407EE903AF8EEE77A5B
:1089F000FCEEE77A17EE900AB1FBF0F202F57F4247
:108A0000FF32120CB1FBF2F295F8CE10B2FBF0F08F
:108A1000042983B272D007EE902AF8EE676A66EEF8
:108A2000887A29EE677A95F8CF0004990091A8EE2C
:108A3000A67A019051463046C6ED027A86ED037A59
:108A400035F030FB002F64DD7368D5F8F4209342D5
:108A500061D0012F5DD0D5F80C2193425BD0022F5D
:108A600057D0D5F82421934255D0032F51D0D5F8B3
:108A70003C2193424FD0042F4BD0D5F85421934240
:108A800049D0052F45D0D5F86C21934243D0062F0D
:108A90003FD0D5F88421D31A18BF01230137012212
:108AA000082F3374727406F118067FF4F6AE33485B
:108AB00009B0BDEC068BBDE8F08F9FED318AF0EE7A
:108AC000488AC8E69FED2F8AF0EE488AC3E6B0EEEA
:108AD000690A61F0F3FEFCEEC07A4FF6FF7317EE01
:108AE000902AD5F89C14B1FBF2F21A44120CB1FB97
:108AF000F2F295F8CE10042918468CD107EE900AB0
:108B000007EE102AF8EE677AF8EE476A67EE8A7A7F
:108B100087E70123C2E70023C0E7C6F814C05CE77B
:108B2000194CD4F844C041EA0C01616436E7164C94
:108B3000D4F830C041EA0C0121632FE7124CD4F87D
:108B400040C041EA0C01216428E7716145E700BF9C
:108B5000B0CC0608082E0020ACC5A737ACC5A73698
:108B6000F9390308F94904087D370308ED49040879
:108B7000F82E002000007A4458CC0608A02E0020D1
:108B8000282930386F120339003802402430002081
:108B90006F12833A1FED028A0D4A0E4BC5F8B420BE
:108BA000C5F8B03000220123CDE90332F0EE488A47
:108BB000094B5CE69FED098AEEE7094A064BC5F8CA
:108BC000B420C5F8BC30002072E70B68FFDE00BFA0
:108BD000F9390308F9490408ED49040800000000C8
:108BE000CD380308F8B5104ED6F89C440546006809
:108BF0000F4664080CF084F8B4FBF7F1B1F5803F40
:108C000003D3012CFAD96408F6E72246284689B234
:108C10003DF02AFC054BC6F8043D28460449BDE852
:108C2000F84000223DF040BB082E00204D240208F1
:108C30000C3B002010B5044C04480A4621460AF0BB
:108C4000D9FE204610BD00BF143B0020705C070811
:108C500010B5044C04480A4621460AF0CBFE2046D3
:108C600010BD00BF143B0020805C070810B5044C09
:108C700004480A4621460AF0BDFE204610BD00BF4A
:108C8000143B00208C5C070810B5044C04480A46CD
:108C900021460AF0AFFE204610BD00BF143B002065
:108CA000985C070810B5044C04480A4621460AF0AF
:108CB000A1FE204610BD00BF143B0020A45C0708A5
:108CC00010B50C4C94F8AD200023A36512B10A4AEC
:108CD000C2F80C3E5CF05EFC20B10423022084F854
:108CE0005C3010BDD4F80839E364092384F85C30A3
:108CF00010BD00BF101D0020082E002070B50D4DC6
:108D000095F85C30042B04460E460AD0082B06D199
:108D10006B6D83420CD0FFF7D3FF022801D00120F6
:108D200070BD0823C5E9154685F85C30022070BD8A
:108D3000022070BD101D002010B50AF02FFE114C4E
:108D400058B194F85C30032B12D894F850300133AA
:108D5000DBB2072B84F8503003D9002384F85C3051
:108D600010BDD4F80839E364012384F85C3010BDE9
:108D7000054846F0BDF80021024604F190005EF07F
:108D800095FEE2E7101D0020801A060070B54379B9
:108D9000234C002B14BF0123002384F8883003D117
:108DA000002384F85C3070BD1E4D002195F9132E10
:108DB000032045F05DFF0028F2D0466830465DF0A4
:108DC00063FA84F8AC000028EAD095F8113E003B25
:108DD00018BF0123304684F8AD305DF035FB0AF052
:108DE000DDFD38B994F8503084F85C00013384F824
:108DF000503070BD5CF0B8FC40B194F850300022A7
:108E0000013384F8503084F85C2070BDD4F8082910
:108E100084F850000123E26484F85C3070BD00BF28
:108E2000101D0020082E002010B55CF09DFC58B1EC
:108E30000B4C94F850300133DBB2072B84F85030E0
:108E400003D9002384F85C3010BD0AF0A7FD002888
:108E5000F7D0D4F80839E364012384F85C3010BDFE
:108E6000101D00202DE9F041854C94F88850002D0C
:108E700000F0F48094F85C20824F0226531E082BE9
:108E800040D8DFE803F036389C3F674F153F0500B8
:108E90005CF080FB002840F0E880E36CD4F80829FF
:108EA000FA3393422BD2FFF7BFFF94F85C20E5E73B
:108EB0005CF070FB0028F0D0A36D0022012B84F839
:108EC000502040F2D680616D94F8AD00013B013135
:108ED000C4E9151310B16B4BC3F80C2E082284F8AB
:108EE0005C20A2F10805B5FA85F56D092846BDE8B4
:108EF000F08184F85C605CF04DFB002841D194F86F
:108F00005C20531EDBB2022B09D8D4F80839E16C7F
:108F10005B1AC82BE5D9FFF787FF94F85C20042A79
:108F2000DFD1E3E7236B002BDBD1666CD4F8083983
:108F3000E364072284F85C20002ED2D0D4E90E210D
:108F4000A36C0120B047DAE7E36CD4F80819643366
:108F50008B42C6D2D4F82C80B8F1000FF4D15CF06B
:108F600019FB0028A1D0666C84F85080042384F893
:108F70005C30002E77D0D4E90E21A36C4046B04778
:108F8000BDE75BF0ADFF0028B9D197F8153E002B87
:108F9000A3F10203B3FA83F314BF022201225B0997
:108FA00084F8512084F852305BF09AFF00287FF457
:108FB0007AAF354A0323926C226684F85C305BF00A
:108FC0008FFF00289BD12F4BA06593F8446EB3F818
:108FD000460ED3F848EED3F848CED3F8487ED3F8FF
:108FE000482E84F8666093F84C1EA4F8640093F849
:108FF0004D6E84F86A2093F84D0ED3F8502EE26639
:10900000B3F8568EB3F8562E84F86B10B3F8561E8C
:10901000C2F30B1343EA182303F00F0301F00F020E
:109020004FEA1E6E4FEA1C4C3F0A360900F00F0053
:1090300003F5FA63042184F8710084F867E084F88A
:1090400068C084F8697084F87060A4F8723084F89D
:10905000742084F85C102846BDE8F08184F85C50E8
:109060002846BDE8F081054640E7042384F85C30DB
:109070003CE7FAD1FFF724FE94F85C20531E41E749
:10908000101D0020082E0020203C00202DE9F0417A
:109090004379414C002B14BF0122002284F8882020
:1090A00003D184F85C30BDE8F08190F8018008F1CC
:1090B000FF3676B2054630460F4646F087F8022363
:1090C000C4F8940084F890302B78002B40D1ED78D0
:1090D00095BB3248C4F8A05045F00AFF0021024673
:1090E0002F485EF0E3FC4FF47A7040F081FFD4F833
:1090F000A00045F0F3FB002211460A23284845F062
:1091000021FFD4F89410274B0A8992070AD50A89BF
:1091100012F0800206D1D4F8081984F850200123F7
:10912000E164BEE7013BEFD194F8502084F85C3055
:10913000531C84F85030B6E7284644F087FF0546B4
:1091400008B11E23C3800921284645F017FAC0E75D
:1091500006EB86063E44414696F90320002045F082
:1091600087FD064630B140685DF08EF8B36884F83C
:10917000AE3018B9002384F8A430A8E70A4A431E89
:1091800002EB431317210022C4F8A8305DF08EF8DB
:10919000012384F8A4309AE7101D0020801A0600ED
:1091A000A01D0020A1860100C801002070B5054661
:1091B0000E460924FFF7B6F9FF2803D1013CF9D187
:1091C000012070BDFE2801D0022070BD33462A4622
:1091D0000021044845F0B6FEFFF7A4F9FFF7A2F915
:1091E000002070BDA01D002070B582B040F0400688
:1091F0000C0E05460A0A080C95238DF801408DF8DF
:1092000004108DF800608DF802008DF803208DF8B1
:1092100005300824FFF786F9FF2802D0013CF9D178
:1092200065B9084806230022694645F08BFE0924EB
:10923000FFF778F9FF2802D1013CF9D1FF2002B0F5
:1092400070BD00BFA01D00202DE9F843194C94F813
:109250005C60042E0546894690461F4608D0082EBD
:1092600002D00020BDE8F883FFF77CF90228F8D18E
:10927000FEF750FF94F8523093B969021120FFF7BE
:10928000B3FF98B9D4F80839C4F838900522C4E976
:109290001187E56384F85C20E3640120BDE8F8836E
:1092A00029461120FFF7A0FF0028EBD0FFF724F993
:1092B000D7E700BF101D002070B51D4D95F85C303C
:1092C000042B06460C4608D0082B20D16B6D834238
:1092D0002BD0FFF747F9022819D1FEF71BFF002119
:1092E0003720FFF781FF21461720FFF77DFFB0B938
:1092F00095F852306BB971021920FFF775FF70B9FC
:109300000823C5E9156485F85C30022070BD012092
:1093100070BD31461920FFF767FF0028F0D0FFF736
:10932000EBF8FFF709FD032070BD022070BD00BF00
:10933000101D00202DE9F04F93B0524C01920646CB
:109340000F46994694F85C30042B0DD0082B07D1BA
:10935000636DB34200F09280FFF704F90228F1D068
:10936000012013B0BDE8F08FFEF7D4FE94F8523020
:10937000002B7BD171021820FFF736FF002877D130
:1093800094F85C50FFF7CEF8082D0CBFFC21FE21AD
:10939000D4F89480009140F0FFFDB8F80C200099BB
:1093A000824642F20F7BB8F80820930748D5404622
:1093B0005EF048FB94F8A420002A50D003A80BF0DC
:1093C000C7FA94F8AE20D4F89430D4F8A8100597D2
:1093D00052060C3348680392049340220023CDE9DF
:1093E0000A3306920D934FF4806208930C934FF466
:1093F0000073099207930BF0E9FAD4F8A83003A997
:1094000058680BF0B7FAD4F8A830D4F8942059680B
:109410000B6843F001030B6093889BB243F0020397
:1094200093800199A763012206230020C4E9111942
:10943000E66384F8402084F85C3013B0BDE8F08F18
:10944000009140F0A9FDA0EB0A055D450099AADD59
:10945000404645F07BFD94F8A420002AAED14FF49D
:1094600080733946084845F06DFDDAE7314682E7FA
:10947000FFF742F8FFF760FC032072E7FFF752F8AE
:10948000FC2185E7101D0020A01D00202DE9F047DC
:10949000D44C94F8886086B0002E00F0AD8194F82A
:1094A0005C10D14F42F20F754B1E082B69D8DFE8D4
:1094B00013F07C00A2002901680057000900E000B9
:1094C0006800CB0094F8A420002A40F0CF81A36B61
:1094D00094F84010C54803EB01214FF4807345F028
:1094E00031FD94F840300133DBB2022B84F8403078
:1094F00044D1D4F8949040F04FFDB9F80C30804638
:10950000B9F808309A0740F15781484600215EF0CB
:1095100099FAD4F8949040F03FFDB9F80C308046A9
:10952000B9F808309B0740F15281484600215EF0AF
:1095300089FAFEF7F7FF00F01F00052800F03582DA
:10954000FFF7FAFBD4F84480B8F1000F00F08881EF
:10955000E16BA36C00220120C04794F85C10A3E7E4
:10956000A06B4FF40071FFF721FE012800F060812D
:10957000022800F06481002800F0B28194F85C10A9
:109580004B1EDBB2022B00F24181D4F80839E26CA9
:109590009B1AC82B00F23681A1F10806B6FA86F6AE
:1095A0007609304606B0BDE8F087FEF7B3FD00212E
:1095B0000846FFF719FE8046FEF79EFFB8F1010F3F
:1095C000DCD14FF0000984F85190FEF7A3FD40F282
:1095D000AB110820FFF708FE052800F044810128A0
:1095E00000F01881FEF788FF94F8511000295AD036
:1095F000022384F85C30FEF78DFD94F85130022B85
:109600000CBF4FF080484FF0000800213720FFF7D3
:10961000EBFD41462920FFF7E7FD8046FEF76CFF92
:10962000B8F1000FAAD194F85130022B00F06D81EF
:1096300084F85280FEF76EFD00210920FFF7D4FD6B
:10964000A0B3FEF759FF99E74FF00808FEF76AFF4D
:10965000FF2800F0A481B8F10108F7D1E36CD4F839
:109660000829FA33934289D2FFF766FB94F85C101D
:109670001AE7FEF757FFFF284FF0080806D0B8F1A9
:109680000108EBD0FEF74EFFFF28F8D1A36D0022B2
:10969000012B84F8502040F29B81626D013B013226
:1096A000C4E91523082184F85C1075E7504810219F
:1096B000FFF77CFD80460028C3D101217F20FEF703
:1096C0006BFD01288146BCD140460221FEF764FDB6
:1096D000002800F046810128B3D116213A20FEF778
:1096E0005BFD013080022066FEF706FFFEF712FDEB
:1096F00000210A20FFF778FD002840F01F81032396
:1097000084F85C30102102A8FFF750FD00287FF498
:1097100035AF9DF815309DF816109DF810209DF876
:1097200009C09DF80A001B01DBB243EA111303F5DF
:10973000FA63A4F87230DDF8113001F00F0184F8FB
:1097400074101BBA110902F00F0240EA0C2084F8D1
:10975000701084F871209DF808109DF80B20E366C6
:10976000039BA366A4F8640084F8661084F867205D
:10977000FEF7C2FE94F852306BB9FEF7CBFC4FF403
:1097800000711020FFF730FD8046FEF7B5FEB8F1FE
:10979000000F7FF469AF174845F0AAFB002102468D
:1097A00012485EF083F9002204233046A26584F853
:1097B0005C3006B0BDE8F08740F0EEFBA0EB08009F
:1097C000A8427FF79DAE484645F0C0FBA1E640F0B9
:1097D000E3FBA0EB0800A8427FF7A2AE484645F0A5
:1097E000B5FBA6E6101D00200F640240A01D00205E
:1097F000881D002040787D01304684F85C6006B00A
:10980000BDE8F087FFF798FA94F85C1004297FF41C
:10981000C3AEC6E604237648494602AA45F092FB49
:109820009DF80B30AB2B04BF022384F85130D9E6EE
:10983000E36CD4F8082964339342BFF49FAEFEF77B
:109840005BFEFFF779FAD4F84480B8F1000F07D037
:109850000022E16BA36C1046C04794F85C1023E62D
:1098600094F85C1020E684F85180BBE6D4F8A82078
:109870006048D2F804C0604BD269BC4598BF03462B
:10988000900062D55868DFF874E1104010EA0E0FBE
:109890003FF482AE02EA0E02DA60DCF80030D4F85F
:1098A000949023F00103CCF80030B9F80830DA07BF
:1098B00005D5B9F80C30B9F80830DB07F9D4B9F898
:1098C00008309807FBD5B9F808301906F7D4B9F86D
:1098D000043023F002031B041B0CA9F804300AE631
:1098E0000190FEF709FE656C019884F8500004238E
:1098F00084F85C30002D3FF454AED4E90E21A36C03
:10990000A84794F85C104B1E3BE6FEF703FC41466B
:109910003A20FFF769FC414681460423344802AAF5
:1099200045F010FBB9F1000F08D1FEF7E5FD029BF1
:109930001BBAC3F3807384F852307BE6FEF7DCFD7C
:10994000FFF7FAF994F85C10AEE51868DFF8ACE0C0
:10995000104010EA0E0F3FF41FAE02EA0E029A60AA
:109960009BE704212C20FEF717FC032180464E20A4
:10997000FEF712FC0C2182463620FEF70DFC0AF1A0
:10998000020A431C03FA0AF309FA08F0A3FB0001D8
:10999000430A43EAC1532366FEF7AEFDA6E6FEF78F
:1099A000ABFD042384F85C30FBE5656CD4F8083922
:1099B000E364072184F85C10002D3FF4EDADD4E999
:1099C0000E21A36C0120A84794F85C104B1ED8E52B
:1099D00008D0042384F85C30FEF78EFD94F85C1008
:1099E0004B1ECEE5FEF7BEFD02287FF4C7AD28E68C
:1099F000A01D002000600240006402407D0F7D0F2A
:109A00002DE9F04FC14C94F8701E83B00546C1F3A8
:109A10004001D4F8780E44F067FF94F8701ED4F833
:109A2000740EC94301F001016F1E44F05DFFFBB2EB
:109A30000193002D00F0D080B54EDFF8DC82B54DEB
:109A40004FF01009D4F8780E44F038FFD4F8740EB3
:109A500044F034FFB4F8803E002B40F04E8194F87F
:109A6000821ED4F8840E44F03FFF4FF0FA0A4FF400
:109A70007A710120D8F80430C3F30803002B40F0BA
:109A80000F81EFF31183002B40F00A81D6F80829EB
:109A9000D5F808C0D6F808399A42F7D1D4F8A83ECC
:109AA0009C45F3D8D4F8A47E01FB07F3A3EB0C0389
:109AB000B3FBF7F301FB0232D8F80430C3F3080319
:109AC000002B40F0AB80EFF31183002B40F0A68019
:109AD000D6F80839D5F808B0D6F80879BB42F7D1DE
:109AE000D4F8A87EBB45F3D8D4F8A47E01FB07FCCC
:109AF000ACEB0B0CBCFBF7FC01FB03C39B1AB3F5EF
:109B00007A7FD9D3BAF1010AB4D1D4F8780E44F0EF
:109B1000D5FED4F8740E44F0D1FEB4F8803E002B8C
:109B200040F0DF8094F8821ED4F8840E81F00101A9
:109B300044F0DAFEFA204FF47A714FF0010CD8F8B5
:109B40000430C3F30803002B40F08980EFF3118346
:109B5000002B40F08480D6F80829D5F808E0D6F824
:109B600008399A42F7D1D4F8A83E9E45F3D8D4F8E4
:109B7000A4AE01FB0AF3A3EB0E03B3FBFAF301FB64
:109B80000232D8F80430C3F3080343BBEFF3118368
:109B90002BBBD6F80839D5F808B0D6F80879BB42FF
:109BA000F7D1D4F8A87EBB45F3D8D4F8A4AE01FB16
:109BB0000AFEAEEB0B0EBEFBFAFE01FB03E39B1AA3
:109BC000B3F57A7FDDD30138B9D1019B5F1EFBB2BB
:109BD000FF2B01937FF436AF03B0BDE8F08FEFF3B6
:109BE000118A89F31288AF682B68DB0344BFC4F87D
:109BF000A0CEAF68D6F80839D4F8A0EE5FFA8AFA9A
:109C00008AF31188D4F8A4AE734401FB0AFEAEEBCC
:109C1000070EBEFBFAFE01FB03E3D0E7EFF3118E64
:109C200089F31288D5F808B02B68DF0344BFC4F865
:109C3000A00ED5F808B0D6F80839D4F8A0CE5FFA4F
:109C40008EFE8EF31188D4F8A47E634401FB07FCDA
:109C5000ACEB0B0CBCFBF7FC01FB03C34EE7EFF3D3
:109C6000118E89F31288D5F808A02B68DA0344BF57
:109C7000C4F8A0CED5F808A0D6F80839D4F8A02E9C
:109C80005FFA8EFE8EF31188D4F8A4EE1A4401FB1D
:109C90000EF3A3EB0A03B3FBFEF301FB023270E702
:109CA000EFF3118C89F31288D5F808E02B68DB03F9
:109CB00044BFC4F8A00ED5F808E0D6F80839D4F8A7
:109CC000A02E5FFA8CFC8CF31188D4F8A47E1A4481
:109CD00001FB07F3A3EB0E03B3FBF7F301FB023227
:109CE000EAE6D4F89C3E002B3FF424AFD4F8883E3B
:109CF000C3F800A084F899AE1CE7D4F89C3E002B72
:109D00003FF4B3AE40F034FAAFE600BF082E0020B7
:109D1000101D002010E000E000ED00E02DE9F04F04
:109D2000BD4CBE4E94F8701ED4F8780EDFF8F48265
:109D3000BB4D83B0C1F3400144F0D6FD94F8701ED2
:109D4000D4F8740EC94301F0010144F0CDFD0523A0
:109D500001934FF01009D4F8780E44F0AFFDD4F819
:109D6000740E44F0ABFDB4F8803E002B40F04C8103
:109D700094F8821ED4F8840E44F0B6FD32274FF4D6
:109D80007A710120D8F80430C3F30803002B40F0A7
:109D90000F81EFF31183002B40F00A81D6F80829D8
:109DA000D5F808C0D6F808399A42F7D1D4F8A83EB9
:109DB0009C45F3D8D4F8A4EE01FB0EF3A3EB0C03FF
:109DC000B3FBFEF301FB0232D8F80430C3F30803FF
:109DD000002B40F0AB80EFF31183002B40F0A68006
:109DE000D6F80839D5F808B0D6F808C96345F7D1D0
:109DF000D4F8A8CEE345F3D8D4F8A4EE01FB0EFCCA
:109E0000ACEB0B0CBCFBFEFC01FB03C39B1AB3F5D4
:109E10007A7FD9D3013FB5D1D4F8780E44F04EFD06
:109E2000D4F8740E44F04AFDB4F8803E002B40F0A4
:109E3000E08094F8821ED4F8840E81F0010144F091
:109E400053FD32204FF47A710127D8F80430C3F360
:109E50000803002B40F08B80EFF31183002B40F0C0
:109E60008680D6F80829D5F808E0D6F808399A424D
:109E7000F7D1D4F8A83E9E45F3D8D4F8A4AE01FBA0
:109E80000AF3A3EB0E03B3FBFAF301FB0232D8F89B
:109E90000430C3F3080343BBEFF311832BBBD6F8A5
:109EA0000839D5F808B0D6F808E97345F7D1D4F8E1
:109EB000A8EEF345F3D8D4F8A4AE01FB0AFEAEEB4E
:109EC0000B0EBEFBFAFE01FB03E39B1AB3F57A7F90
:109ED000DDD30138B9D1019B5F1E17F0FF03019359
:109EE0007FF439AF03B0BDE8F08FEFF3118A89F347
:109EF0001288D5F808B02B68DB0344BFC4F8A07EF5
:109F0000D5F808B0D6F80839D4F8A0EE5FFA8AFA86
:109F10008AF31188D4F8A4AE734401FB0AFEAEEBB9
:109F20000B0EBEFBFAFE01FB03E3CEE7EFF3118E4F
:109F300089F31288D5F808B02B68DB0344BFC4F856
:109F4000A00ED5F808B0D6F80839D4F8A0CE5FFA3C
:109F50008EFE8EF31188D4F8A4EE634401FB0EFC50
:109F6000ACEB0B0CBCFBFEFC01FB03C34EE7EFF3B9
:109F7000118E89F31288D5F808A02B68DA0344BF44
:109F8000C4F8A07ED5F808A0D6F80839D4F8A02ED9
:109F90005FFA8EFE8EF31188D4F8A4EE1A4401FB0A
:109FA0000EF3A3EB0A03B3FBFEF301FB02326EE7F1
:109FB000EFF3118C89F31288D5F808E02B68DA03E7
:109FC00044BFC4F8A00ED5F808E0D6F80839D4F894
:109FD000A02E5FFA8CFC8CF31188D4F8A4CE1A441E
:109FE00001FB0CF3A3EB0E03B3FBFCF301FB02320A
:109FF000EAE6D4F89C3E002B3FF423AFD4F8883E29
:10A000001F6084F8997E1CE7D4F89C3E002B3FF437
:10A01000B5AE40F0ADF8B1E6082E0020101D0020CE
:10A0200010E000E000ED00E00E4B30B4DB68427859
:10A0300001780D4CDB43C3F30223C3F10403DBB20D
:10A0400002FA03F360181B0101F01F050122490900
:10A0500003F0F003AA4080F8003344F8212030BC1C
:10A06000704700BF00ED00E000E100E000F01F02DB
:10A0700040090123032803FA02F304D004280CD07A
:10A08000022805D07047074A116C0B4313647047D0
:10A09000044A516C0B4353647047024A116B0B43E3
:10A0A000136370470038024000285FD00368374AC6
:10A0B0002DE9F04103F13F4404F57E0402EB9422C4
:10A0C000012492F8982002F01F055209032A04FA8D
:10A0D00005F456D0042A4FD0022A48D08588B5FA14
:10A0E00085F0C0F11F00C0F3CC0603EB860600F03C
:10A0F000070082000F24306A944020EA0400306296
:10A10000306A01FA02F20243002132624FF0010E7E
:10A110000A464FF0030C02270EFA02F838EA05004F
:10A1200002F101021CD118680CFA01F420EA0400C3
:10A130001860186807FA01F606431E609E6826EA52
:10A1400004069E6098689860586820EA0800586085
:10A1500058685860D86820EA0400D860D868D86089
:10A16000102A01F10201D7D1BDE8F0817047084AF9
:10A17000556C2C435464B1E7054A156B2C431463AA
:10A18000ACE7034A156C2C431464A7E758CC0608C7
:10A1900000380240002861D00368384A03F13F418B
:10A1A00001F57E0102EB91222DE9F04192F8982011
:10A1B00002F01F0452090121032A01FA04F158D0C8
:10A1C000042A51D0022A4AD08588B5FA85F2C2F114
:10A1D0001F02C2F3CC0403EB840402F00702216ADD
:10A1E00092000F20904021EA00012162206A0C2198
:10A1F00001FA02F202430021226208464FF0010EEA
:10A200004FF0030C02270EFA00F838EA050200F1BD
:10A2100001001DD11C680CFA01F224EA02041C6042
:10A220001E6807FA01F434431C609E6826EA0206A1
:10A230009E609E6816439E605C6824EA08045C6029
:10A240005C685C60DC6824EA0202DA60DA68DA6082
:10A25000102801F10201D6D1BDE8F0817047084A0B
:10A26000546C21435164AFE7054A146B21431163D9
:10A27000AAE7034A146C21431164A5E758CC0608E9
:10A28000003802402DE9E047304D95F8AC3E012BF7
:10A2900085B00F46164640D0022B2ED1B5F8B83EF9
:10A2A00040F08001002B44D1D5F8BC3E13B11A68B0
:10A2B0009B885383D5F8B0AE03913FF06DFEBAF89A
:10A2C0000C300399804642F20F79BAF808309B07A8
:10A2D00017D550465DF0B6FB3346D5F8B00E3A467A
:10A2E00000215DF089FCD5F8BC3E6BB31A689B88F1
:10A2F0001383012005B0BDE8E087002005B0BDE86C
:10A30000E08703913FF048FEA0EB08034B4503991B
:10A31000DBDD504644F01AFEDEE70091134695F867
:10A32000B11E024695F9B00E5EF0FEF805B0BDE82C
:10A33000E087D5F8B42ED0899842B5D0D5F8B00EC4
:10A340000380D38100BFAFE70120D7E7082E0020AC
:10A3500058B183884FF00042B3FA83F332FA03F323
:10A3600003D002490A6813430B607047003C014068
:10A370002DE9F04385B00D461646044644F0C6FA72
:10A3800000284EDB334FDFF8D48007EB800308EB67
:10A39000000C07F6347229462046C3F8F42E9CF8C8
:10A3A000A09044F0EBF8002C51D0256805F13F4512
:10A3B00005F57E05AD0A204644F0A8FA00F0FC033E
:10A3C00003F1804303F59C3300F003009A6880009A
:10A3D0000F21814022EA01029A609A68EDB205FAE3
:10A3E00000F0104398602CB1A0884FF00044B0FA00
:10A3F00080F0C440184B08EB86064F445C61D6F8E9
:10A40000B0108DF80D100123002202A88DF80E3037
:10A4100002948DF80C20FDF7F3FD97F8383FF02BF0
:10A4200002D805B0BDE8F083C844F02198F8BC30EC
:10A430008DF8043003224FF4807301A887F8381F89
:10A440008DF80520ADF80630FFF7EEFDE9E74FF097
:10A45000FF35B0E7082E0020003C014058CC06082C
:10A46000002864D0F0B58388B3FA83F3202B0A4622
:10A4700085B00446C3F11F0143D02D4D2D4E05EB91
:10A4800081037718C3F8F42E002197F8A07044F0E8
:10A4900075F8B4F804C02268274CBCFA8CFCCCF1E7
:10A4A0001F0303F0FC0101F1804101F59C3103F031
:10A4B000030398004FF00F0E02F13F438A680EFA33
:10A4C00000FE22EA0E0203F57E038A60C3F38723AF
:10A4D000834088684FF0004222FA0CF203433D4467
:10A4E0008B6002A8626101234FF400618DF80E3089
:10A4F0000292ADF80C10FDF783FD95F8383FF02B74
:10A5000001D805B0F0BD3E44F02196F8BC308DF87E
:10A51000043003224FF4807301A885F8381F8DF8AA
:10A520000520ADF80630FFF77FFD05B0F0BD7047A0
:10A53000082E002058CC0608003C014010B4B8B1E9
:10A540000D4CD4F8403F102B05D15DF8044B05218C
:10A5500000203CF04DBC03EB4302224482F8451F2F
:10A5600001210B4482F8440F82F8461FC4F8403F93
:10A570005DF8044B704700BF082E0020C0782021F2
:10A58000DCE700BF2DE9F04FDFF884A32DED028B4F
:10A590009AF8881F002297B0CAF8782FCAF87C2F43
:10A5A000CAF8802FCAF8842FCAF8742F19B19AF804
:10A5B000892F8AF8742F9AF88A2F1AB19AF88B2F5C
:10A5C0008AF8832F9AF88E2F1AB19AF88F2F8AF86B
:10A5D0007E2F9AF88C2F1AB19AF88D2F8AF8792F3E
:10A5E0009AF8903F05935A1ED3B257B204937B1C3E
:10A5F00000F0AA80BC4ABD4E52F83780029602EBAA
:10A60000C70200231279019308EE102A1D46344632
:10A61000994626783946304645F04EF9834630460D
:10A62000BBF1000F1ED043F011FDEA1D1321D2B281
:10A6300020B14FF0000E827180F807E043F09EFFDA
:10A64000207845F063F94FF0070309F10102237107
:10A650004FF0010384F802906070CDF804B05FFA07
:10A6600082F9E3700135042D04F10504D1D118EE0F
:10A67000100A029ECDF80C90FFF7F8FC9C499D4A09
:10A680004868024042F440324A600FB9019B5BB90E
:10A69000994C4820FFF7EAFC204602215EF0F2F8D0
:10A6A000A26842F00102A2609148934A4168BAF858
:10A6B000924F41F400014160516821F48051516092
:10A6C000916B21F4401141F480119163D16841F400
:10A6D0006001D160956B85F44011C1F3015101EB2C
:10A6E00081011F2000FA01FC25EA0C0C112505FA56
:10A6F00001F141EA0C019163D16841F0E061D16060
:10A70000956BC5F30151C1F10401C9B201EB81019F
:10A7100088404FF0120C25EA00000CFA01F10843C2
:10A720009063E4B1BAF8941FCAF89C4FA1B1BAF88B
:10A73000962FCAF8A01F62B1019B7048521A90FB75
:10A74000F2F2CAF8A42F6BB917B0BDEC028BBDE8CA
:10A75000F08F6B4A1288EFE76A4A1188E7E76A4A86
:10A760001488DFE7404603995EF08CF85F4B0120C8
:10A7700003F114090723F278441CE4B252B375784C
:10A780003279A5F10A0101EB410105EB450C092DD8
:10A7900003FA01FE03FA0CFB02FA01F140F28E808B
:10A7A000D8F80C2022EA0E0E41EA0E01C8F80C106F
:10A7B000421E02EB82021F21062801FA02FC05FA62
:10A7C00002F261D8D8F8341021EA0C010A4320467D
:10A7D000C8F834200536B145CDD1D8F80820049901
:10A7E00042F40072C8F80820D8F8082042F48072B9
:10A7F000C8F80820D8F80820574442F00102C8F8E9
:10A80000082097F9982F022044F032FA04460028D5
:10A810009AD040685BF038FD059A06215BF046FD52
:10A8200060680AF0D3F807A80AF092F8039EA368BC
:10A83000364A0793012E8CBF4FF48060002000231E
:10A840000D9008F14C054FF40060089509920A93A9
:10A850004FF480720C930E904FF4003360680B96A7
:10A8600007A94FF40055CDE90F5211930AF082F871
:10A870006268136843F001031360D8F8083043F0AE
:10A880008043C8F808305FE7C11FA0F10D0201EB5B
:10A8900081014FF01F0E02EB82020C280EFA01FC20
:10A8A0000EFA02F005FA01F113D8D8F8302022EAA6
:10A8B0000C0211432046C8F830108BE7D8F810106E
:10A8C00002FA0CF221EA0B0B42EA0B02C8F8102044
:10A8D0006EE7D8F82C1005FA02F221EA00010A43CB
:10A8E0002046C8F82C2075E71CCD06087C3D0020CA
:10A8F00000230140E030FCFF0020014080380100CF
:10A900002E7AFF1F2C7AFF1F2A7AFF1FB03D0020EE
:10A91000082E00202DE9F0472E4C054600EB800064
:10A9200004EBC004D4F8B47F2FB10E4694F8C91FCD
:10A9300001F0FF0821B14FF000084046BDE8F08764
:10A94000994692463FF028FB71000123C9B284F872
:10A95000CA1F84F8CBAF84F8CD3F84F8CE8F84F83B
:10A96000CC3F84F8C93F84F8C88FBA88C4F8D09F18
:10A9700091050646C4F8D49F1CD43B88DA050FD451
:10A9800042F20F7404E03FF007FB831BA34215DC87
:10A990003B889B05F7D43B889BB243F480733B8094
:10A9A000BB889BB243F440734FF00108BB80404624
:10A9B000BDE8F08798464046BDE8F087064A32F881
:10A9C000D03C01339BB2284622F8D03C5DF02CFBF2
:10A9D000B3E700BF082E0020003F0020F8B5764DF9
:10A9E00005EB001757F8CC3C002B00F09280044692
:10A9F000060117F8C40CFFF739FB17F8C43C03F045
:10AA00001F015B090122032B02FA01F200F097807B
:10AA1000042B00F08480022B7CD0AB19013413F896
:10AA2000C80C43F013FBE4B2074610B11223C47103
:10AA30008371AB1913F8C70C43F008FB10B1132353
:10AA4000C4718371AB1913F8C60C43F0FFFA10B14F
:10AA50001423C4718371AC190A2114F8C52C38462B
:10AA600043F0BAFB14F8C70C43F0F0FA14F8C52C05
:10AA70000A2143F0B1FB14F8C60C43F0E7FA14F8CE
:10AA8000C52C0A2143F0A8FB54F8CC3C4B4A934216
:10AA90005AD04B4A934247D04A4A93425FD04A4ADF
:10AAA000934267D0494A93426FD0494A934277D044
:10AAB000AB19484A53F8CC1CB2F832520888B2F8A5
:10AAC0003032B2F8344200F441502B430343B2F821
:10AAD0003A02B2F83C5223430343B2F83E42B2F882
:10AAE00040022B4323439BB243F00303022501247E
:10AAF000A2F83652A2F838420B808B8B23F4006305
:10AB00001B041B0C8B8308820B889BB243F0400311
:10AB10000B80F8BD304B596A0A435A627DE72E4BD1
:10AB200019690A431A6178E702F500324FF4804050
:10AB3000136A43F4804313620AF0DAF8B8E7264B4D
:10AB4000196A0A431A6268E702F584324FF48050AA
:10AB5000536A43F4805353620AF0C2F8A8E702F53F
:10AB6000FE324FF40040136A43F4004313620AF0CC
:10AB7000BFF89DE702F582324FF40050536A43F468
:10AB8000005353620AF0ACF892E702F568424FF4C2
:10AB90008010536A43F4801353620AF0A1F887E7E8
:10ABA00002F564424FF40010536A43F400135362F9
:10ABB0000AF096F87CE700BF003F0020003001401B
:10ABC00000380040003C004000340140005001408B
:10ABD00000540140980100200038024070B5464EF4
:10ABE00016F89C4C04EB440306EBC303650013F812
:10ABF000983C032B6ED8DFE803F059291E02254448
:10AC000006EBC50555F8940C002870D116F8383CB1
:10AC10009C425FD0013404F00302934206F89C2C5E
:10AC200058D002EB420406EBC404022344F8940C0F
:10AC300004F8983C70BD2B1906EBC30353F8942C11
:10AC400072B1013A43F8942C002070BD2B1906EB29
:10AC5000C30353F8942C002AF3D1022203F8982C52
:10AC6000254406EBC50515F88C3C013BDBB205F825
:10AC70008C3C8BBB214B16F8386CD3F8441255F83A
:10AC8000900C621C02F003024B1E0324B2420344E8
:10AC900005F8984CB3FBF1F045F8940C1AD09942A2
:10ACA00018D8013845F8940C012070BD44F006FD19
:10ACB00080B1124B2C44D3F8442206EBC40401218A
:10ACC00002F51C5304F8981C0F33B3FBF2F344F85D
:10ACD000943C70BD012070BD084BD3F84422012084
:10ACE00002F2E733B3FBF2F345F8943C70BD013850
:10ACF00045F8940C002070BD003F00209801002012
:10AD00002DE9F84F3249DFF8D4B091F8151E01242F
:10AD10000229074619461046CBF82C404FF0000296
:10AD20002C4C1D4618BF7F02FDF794F92A4B636235
:10AD30006B02A362E36A40F2FF5943F093034FF4BE
:10AD400000704FF48A62E3620121C4F83890A06079
:10AD50001020E2605AF010FA012D40F251434E46A5
:10AD6000C4F83890CA4640F252488EBF4FF01209DC
:10AD700098464FF011090A25C4F838A00121A760B0
:10AD80004846C4F80C805AF0F7F903464FF0000C1F
:10AD900040F2774201213720A6632BB900231846E1
:10ADA000CBF82830BDE8F88FA663C4F808C0E2608D
:10ADB0005AF0E2F9013DA6630028EFD015F0FF0537
:10ADC000DAD10346CBF82C50CBF82830BDE8F88F09
:10ADD000082E0020002C014000E1F505101D002088
:10ADE0002DE9F843184C94F85C60042E054689461A
:10ADF00090461F4608D0082E02D00020BDE8F883F8
:10AE0000FDF75EFF0228F8D101234A4628460021BB
:10AE1000FFF776FF50B1FEF707F8656C002DECD018
:10AE20000022A36CE16B1046A847E6E7D4F8083986
:10AE3000C4F838900522C4E91187E56384F85C20E2
:10AE4000E3640120BDE8F883101D00202DE9F84FD0
:10AE50002F49DFF8C49091F8151E1E4602292D4B8C
:10AE600007464FF0010418BF4702012E40F259482F
:10AE70001C6398BF4FF48B683B469346474640F2AD
:10AE8000FF55B0468CBF4FF0190A4FF0180A0A243C
:10AE90001E4640F2FF53C9F838300121C9F8086056
:10AEA0005046C9F80C705AF067F903464FF0000C91
:10AEB00040F2774201213720C9F83850A3B95846EB
:10AEC00041460122FDF7C6F84646134A134B53622A
:10AED00076029662D36A43F09103D3620D4B002150
:10AEE00008469962BDE8F88FC9F83850C9F808C01B
:10AEF000C9F80C205AF040F9013CC9F83850002834
:10AF0000DDD014F0FF04C4D1024B1C63BDE8F88F00
:10AF1000082E0020101D0020002C014000E1F50546
:10AF20002DE9F047364C82B005460E461746984646
:10AF300094F85C0004280CD0082806D1636DAB425D
:10AF400007D0FDF7BDFE0228F2D0012002B0BDE817
:10AF5000F087DFF8B4A0A663DAF80C9EE563C9F3C6
:10AF60004F210F294FEA592222D8A36D0193FBB13B
:10AF700094F8AD00E0B1B9F5005F13D02148314637
:10AF80004FF40072484461F0B5FD09F50072C2F358
:10AF90004F211029CAF80C2E4FEA522202D0019BF1
:10AFA000012B21D192B2013A164EAD1A0B4600E0A8
:10AFB0000123324628460626012500216764C4F88D
:10AFC000488084F8405084F85C60FFF73FFF002819
:10AFD000BCD0FDF729FF666C86B12846A36CE16BF7
:10AFE0000022B0470320B1E7626D013B013204212A
:10AFF000C4E9152384F85C100220A7E70320A5E725
:10B00000101D0020786C0020082E0020144A154BDB
:10B01000D2F89C24B3EB920F15D2B3EBD20F14D21B
:10B02000B3EB121F13D2B3EB521F12D2B3EB921F2A
:10B0300011D2B3EBD21F10D2B3EB122F34BF4FF4A7
:10B0400080708020704702207047042070470820DD
:10B05000704710207047202070474020704700BF85
:10B06000082E0020809698002DE9F0472E4C94F889
:10B07000AC3E022B82B005460F46164611D0012B7E
:10B080000BD10091134694F8B11E024694F9B00E0C
:10B090005DF04AFA02B0BDE8F087002002B0BDE8DA
:10B0A000F087B4F8B83E8BBBD4F8BC3E13B11A6835
:10B0B0009B885383D4F8B0AE3EF06EFFBAF80C30E4
:10B0C000804642F20F79BAF808309B0714D529461A
:10B0D00050465CF0B7FC3346D4F8B00E3A46002137
:10B0E0005CF08AFDD4F8BC3EDBB11A689B88138300
:10B0F000012002B0BDE8F0873EF04EFFA0EB080350
:10B100004B45E0DD504643F021FFE4E7D4F8B42E90
:10B11000D1899942C8D0D4F8B01E0B80D38100BF2A
:10B12000C2E70120B6E700BF082E002070B5027804
:10B13000022A04460D4613D0012A01D0002070BD1A
:10B140000C4B90F9040003F8372C421CF6D003286E
:10B15000F4DC0A46373B6179BDE87040FFF7DABBA3
:10B1600059F0B2FE294620460122BDE8704043F066
:10B17000C3BF00BF003F002010B50B4CD4F8BC0E7D
:10B1800043F0ACFBD4F8BC0E08B12123C3800121ED
:10B1900043F0F4F9FFF73AFFBDE8104002460321FF
:10B1A00002485CF083BC00BF082E0020B43C0020A5
:10B1B00073B50D4E05460C46FF230A460146304640
:10B1C0008DF8073043F098FF01230DF1070245F099
:10B1D0008001304643F05EFF9DF80700031B584294
:10B1E000584102B070BD00BFB43C002030B583B000
:10B1F0000D46012301460DF107020446074844F0BD
:10B2000065F89DF8072035EA020304D003482A4375
:10B21000214644F027F903B030BD00BFB43C002004
:10B2200037B5394C00238DF8073014F8283C03F06B
:10B23000FD02012A05D114F8202C12B90C2204F8C1
:10B24000202C022B314D1DD0032B2FD001220B219E
:10B25000284657F0DDFF04203EF0CAFE01230DF121
:10B2600007020021284657F0F4FFB8B39DF80730D5
:10B27000482B33D1264B44F8343C264B44F8303C21
:10B2800003B030BD54F8180C43F028FB54F8180CE8
:10B2900008B13523C380012143F070F9FFF7B6FEF2
:10B2A0000321024628465CF001FCCFE71A4B54F814
:10B2B000240C46F2A812C3F854263721122257F064
:10B2C0007BFF54F8240C0D22242157F075FF54F80D
:10B2D000240C30226A2157F06FFFB7E714F8283C9E
:10B2E000022B03D0032B07D00020C9E754F8180C19
:10B2F00043F0ACFD0020C3E754F8240C10223721A2
:10B3000057F05AFFF0E700BF003F0020D83E002072
:10B31000AB3206082D330608980100202DE9F047CE
:10B32000334F344BD7F89C24B3EB920F0646884634
:10B3300080F0DA82B3EBD20F80F0D882B3EB121F29
:10B3400080F0DF82B3EB521F80F0DD82B3EB921FFF
:10B3500080F0DF82B3EBD21F80F0DF82B3EB122FDD
:10B3600034BF4FF480718021234C00234FF4F072DE
:10B37000A18304F120002021A377E37761F01BFC77
:10B3800004F500704FF4F072202161F014FC94F881
:10B39000E10340B394F8E2332BB30509013D042DDA
:10B3A00000F00F0000F22382DFF8549009EB450310
:10B3B000B3F8842042FA00F3DB0740F1188201233E
:10B3C00003FA00F0013810404D445EF00FFA95F892
:10B3D00090200A4B104403EBC000C4F8F4038379B7
:10B3E00083B1412B0ED06FF00100BDE8F08700BFA4
:10B3F000082E002080969800003F00202430002076
:10B4000058CC06082323C380092143F0B7F8D4F8A9
:10B41000F41311B10B688A881A8394F8E233013B64
:10B420005BB25D1C00F0E781022B00F3E481D7F8EA
:10B430009C24CE4804EB03134FF0020C53F8CC5C71
:10B44000C4F8E853B0EB920F22FA0CF384F8E4C38B
:10B4500080F06782C54AB2EB530F80F05082B2EBA6
:10B46000930F80F05282B2EBD30F80F05082B2EB98
:10B47000131F80F05082B2EB531F80F05082B2EB6A
:10B48000931F34BF4FF4807380235B002A88B84831
:10B4900022F040021204120C2A802A8822F038027C
:10B4A000120485424FEA124200F09F81B148854262
:10B4B00000F09B81B3F5807FA8BF4FF48073002B11
:10B4C00093FAA3F3B3FA83F308BF4FF0FF33013BC2
:10B4D00042EAC3039BB22B802B88B4F8F0239BB2C3
:10B4E00043F040032B80002A40F0538111B10B68D8
:10B4F0008A885A833EF050FDAB89814642F20F7A2A
:10B500002B89980740F13A8128468C215CF09AFA01
:10B51000D4F8E8A33EF040FDBAF80C30054642F2FC
:10B520000F79BAF80830990740F100815046FF21A1
:10B530005CF088FAD4F8F433002B00F006811D6823
:10B54000998829831B2840F0F0812322DA80B4F8FF
:10B55000F0230120A077002A40F035816983D4F8D8
:10B56000E8A33EF019FDBAF80C30054642F20F7917
:10B57000BAF808309A0740F1CF8050460A215CF0B3
:10B5800061FAD4F8E8A33EF007FDBAF80C3005469E
:10B5900042F20F79BAF808309B0740F1B380504669
:10B5A00040215CF04FFAD4F8E8A33EF0F5FCBAF87D
:10B5B0000C30054642F20F79BAF80830980740F18E
:10B5C000978050468A215CF03DFAD4F8E8A33EF01B
:10B5D000E3FCBAF80C30054642F20F79BAF80830AD
:10B5E00099077AD55046FF215CF02CFAD4F8F43351
:10B5F000C0F3801184F8F81300F0400013B11A680A
:10B600009B88138394F8E023012A00F02E81022AFC
:10B6100000F00E81002A00F04A81A28B94F8F933E1
:10B62000182B05D1A4F8FC83A4F8FE13A4F8002479
:10B63000514803215CF03AFAB4F8F033002B40F0A3
:10B64000B680D4F8F43313B11A689B885383D4F8C6
:10B65000E8533EF0A1FCAB89074642F20F782B89F4
:10B660009A0731D5284600215CF0ECF9D4F8E8536C
:10B670003EF092FCAB89074642F20F782B899B077C
:10B6800019D5284602215CF0DDF9D4F8F43313B162
:10B690001A689B8813837278B378317884F804141D
:10B6A000C2F12002C3F1100384F8052484F80634A3
:10B6B0000020BDE8F0873EF06FFCC31B4345DDDD95
:10B6C000284643F043FCE0E73EF066FCC31B4345DD
:10B6D000C5DD284643F03AFCC8E73EF05DFC431B5D
:10B6E0004B457FF77BAF504643F030FCC0B27DE75F
:10B6F0003EF052FC431B4B457FF75EAF504643F094
:10B7000025FC62E73EF048FC431B4B457FF742AF08
:10B71000504643F01BFC46E73EF03EFC431B4B45C6
:10B720007FF726AF504643F011FC2AE73EF034FC89
:10B73000431B4B457FF7F5AE504643F007FCD4F86A
:10B74000F433C0B2002B7FF4FAAE1B2840F0ED803A
:10B75000B4F8F0230123A377002A3FF400AFD4F814
:10B76000EC13CB89934233D1F9E600BF8096980061
:10B7700000380040003C0040E44200203EF00CFC59
:10B78000A0EB090353457FF7BBAE284643F0DEFB31
:10B79000BEE6D4F8EC33D88990423FF4A7AE2A80B5
:10B7A000DA8100BFD4F8E853D4F8F4139EE6D4F855
:10B7B000EC23D18999423FF444AFD4F8E8130B80CD
:10B7C000D38100BF3DE7D4F8EC13C889904209D07B
:10B7D000D4F8E8331A80CA8100BFD4F8F433002BC0
:10B7E0003FF4BDAE1D689988B8E65B0862E60020AC
:10B7F000C4F8F40308E6D7F89C2457484FF0020C2D
:10B800000025B0EB920F22FA0CF384F8E4C3C4F8DD
:10B81000E853FFF41FAE2B8823F040031B041B0CDE
:10B820002B802A8822F038021204120C04233DE6F1
:10B83000D7F89C04484BB3EB900F14D2B3EBD00F66
:10B8400059D2B3EB101F58D2B3EB501F6BD2B3EBEE
:10B85000901F71D2B3EBD01F70D2B3EB102F34BF57
:10B860004FF480728022A283D8E6D7F89C243A4B0A
:10B87000B8F1000F01D000283AD0B3EB920F69D293
:10B88000B3EBD20F37D2B3EB121F36D2B3EB521F4A
:10B8900049D2B3EB921F4FD2B3EBD21F4ED2B3EBD0
:10B8A000122F34BF4FF480728022A283B6E6D7F8FD
:10B8B0009C24294BB3EB920F1DD2B3EBD20F3FD296
:10B8C000B3EB121F3ED2B3EB521F3DD2B3EB921F2C
:10B8D0003CD2B3EBD21F3BD2B3EB122F34BF4FF4A9
:10B8E000807280225200BEE702213DE504213BE543
:10B8F000B3EB920FE1D30422B5E70822B3E70423A8
:10B90000C3E5082130E510212EE50823BDE510230D
:10B91000BBE5202128E52023B7E5402124E540238D
:10B92000B3E50423B2E510229DE71846202142F03A
:10B9300025FE4FF0FF30BCE6202294E7402292E73C
:10B940000422CFE70822CDE71022CBE72022C9E767
:10B950004022C7E7022286E780969800094B93F8B9
:10B96000CE30042B08D9053B032B08D801231A46F7
:10B9700000B103701046704700230122F8E700234E
:10B980001A46F5E7082E0020F0B40D6800240CE0FC
:10B99000BCF1050F18D8A0F137030A2B14D104EB22
:10B9A000840415F8010B03EB4404A0F13003DEB26C
:10B9B000092EA0F16107A0F1410CF0D9052FE7D8BD
:10B9C000A0F157030A2BEAD00D601460F0BC704759
:10B9D0009FED717A07EE901A20EE070AF8EE677A6B
:10B9E00027EE800AFDEEC07A17EE903A2033402B06
:10B9F00000F2C280DFED697AB4EEE70AF1EE10FAE8
:10BA0000F0EE407A0CDD9FED666ADFED666AB0EE1F
:10BA1000677AB4EEE67AF1EE10FA77EEC67AF6DCE3
:10BA20009FED617AF4EEC77AF1EE10FA0CD59FED36
:10BA30005C6ADFED5E6AB0EE677AB4EEE67AF1EE4C
:10BA400010FA77EE867AF6D49FED597AF4EEC77A3B
:10BA5000F1EE10FA00F388809FED567AF4EEC77A83
:10BA6000F1EE10FA44BF9FED507A77EE677A27EE39
:10BA7000A76ADFED515A9FED517ADFED516AA6EECC
:10BA8000257A67EE865AE6EE076AB6EE007AE5EEAC
:10BA9000A67A27EE877ADFED466A70EE267ABDEE4B
:10BAA000E76A16EE103A2033402B62D8B4EEE60A6D
:10BAB000F1EE10FA0CDDDFED3A5A9FED3A6AF0EE46
:10BAC000676AF4EEC66AF1EE10FA77EEE57AF6DC14
:10BAD000DFED356AF4EEE67AF1EE10FA0CD5DFED23
:10BAE000305A9FED326AF0EE676AF4EEC66AF1EE04
:10BAF00010FA77EEA57AF6D4DFED2D6AF4EEE67A49
:10BB0000F1EE10FA3BDDDFED256A76EEE77A67EEBF
:10BB1000A75A9FED295A9FED296ADFED296AA5EE04
:10BB2000856A27EEA55AE5EE866AB8EE006AE5EE6C
:10BB3000267A67EE867AC7EE206AB7EE006A76EE5E
:10BB4000865A76EE666A86EE257A67EE277A66EE84
:10BB5000876AC0ED017AC0ED037A80ED007A80ED4E
:10BB6000027AC0ED046A70479FED0C7A77EE677A2F
:10BB70007DE7DFED147ADEE79FED127A8BE7DFEDEC
:10BB80000D6AF4EEE67AF1EE10FA44BFDFED066AD4
:10BB900076EEE77ABBE700BF27D4D236DB0F494009
:10BBA000DB0FC940E4CB1641DB0F49C0E4CB16C123
:10BBB000DB0FC93FDB0FC9BF92E741B99730083CA3
:10BBC00015A82ABE000000002DE9F047DFF8E48345
:10BBD000D8F80C3498F8485A07EE903AF8EE670A0D
:10BBE00008F644232DED028BC3ED000A002D78D119
:10BBF000DFF8C4E3C8F8505A98F854CA9EF80050C9
:10BC0000BCF1000F40D0B8F84C3A9FEDD36A9FEDDD
:10BC1000D37A07EE903AF8EE677A20EE877AC6EE8E
:10BC2000276ACF4B0022BCF1010F1A6076EE876ABB
:10BC3000C7EE267AC3ED017A26D0BCF1020F9A60D6
:10BC4000C3ED037A20D0BCF1030F1A61C3ED057A6E
:10BC50001AD0BCF1040F9A61C3ED077A14D0BCF17D
:10BC6000050F1A62C3ED097A0ED0BCF1060F9A6275
:10BC7000C3ED0B7A08D0BCF1070F1A63C3ED0D7A40
:10BC800002D09A63C3ED0F7AB64B9FEDB76A93F873
:10BC9000EE309FEDB67A9FEDB60AB64A07EE903ABF
:10BCA000F8EEE77A9EF8343AC6EE276A1D4415FB93
:10BCB0000CFC5FFA8CFC07EE90CA60EE870AF8EE87
:10BCC000E77AC2ED006AA7EEA00A5EF0BBFEBDEC0B
:10BCD000028BFCEEC07A17EE903A88F8A43BBDE8E0
:10BCE000F087B8F84A3A98F8497A9FEDA37ADFF8D6
:10BCF000C8E2DFEDA26A98F854CAC8F850EA07EE25
:10BD0000903A06EE107AF8EEE77ABCEEE02A27EEDB
:10BD1000877AB8EEC66AB8EE422A012322EE262AB6
:10BD20008EED037A8EF80050CEED040A8EED016A96
:10BD300088F84E3ABCF1000F00F0E8809FED907A51
:10BD40009FED904ADFED905AC7EE271A0CEB4C0698
:10BD500006EBC6066FF06B0A0EEB86060AFB0CFAC2
:10BD60004FF00009B1EE611A9FED886A0AEB0604F4
:10BD700000229FED873ADFED873ADFED876A1046B4
:10BD8000234607EE902AB8EEE77A27EE027AFDEE18
:10BD9000C77A17EE901A2031402900F2CB80B4EE1A
:10BDA000C47AF1EE10FAF0EE477A0CDDDFED7B4A53
:10BDB0009FED7B5AF0EE672AF4EEC52AF1EE10FAF9
:10BDC00077EEE47AF6DCF4EEE57AF1EE10FA0CD5D3
:10BDD000DFED724A9FED735AF0EE672AF4EEC52A42
:10BDE000F1EE10FA77EEA47AF6D4F4EEC67AF1EE1C
:10BDF00010FA40F3A68074EE677A27EEA75AB0EEE9
:10BE0000630AA5EE030ADFED684AE5EE004A65EE37
:10BE1000272AB7EE005AE2EEA47AB0EE458AF0EE99
:10BE2000454AA1EEA78AE1EE274AC5EE088A84EECC
:10BE3000880A77EE067ABDEEE75A15EE101A203121
:10BE4000402974D8B4EEC67AF1EE10FA0CDD9FEDFD
:10BE5000535A9FED537AF0EE674AF4EEC74AF1EE7B
:10BE600010FA77EEC57AF6DCF4EEE57AF1EE10FA28
:10BE70000CD59FED4A5A9FED4B7AF0EE674AF4EEEF
:10BE8000C74AF1EE10FA77EE857AF6D4F4EEC67A68
:10BE9000F1EE10FA41DD74EE677A27EEA75AF0EE64
:10BEA000632AE5EE032A9FED407AA5EE227A65EE3D
:10BEB000274AB8EE005AE4EE877A67EE857A87EE75
:10BEC000887A013085423A4403F1240343ED048A21
:10BED00003ED037A03ED017A43ED028A83ED000A54
:10BEE000C3ED026AC3ED016AC3ED046AC3ED036AE0
:10BEF0003FF747AF6C34A6427FF43AAF09F5587963
:10BF0000B9F5226F06F558767FF42EAF9FED277AAC
:10BF1000C7EE207ACEED027A72E69FED257AF4EE36
:10BF2000C77AF1EE10FA48BF75EEE77AB5E7F0EEA2
:10BF3000667AC4E7B7EE000AF0EE408AB0EE408AB7
:10BF400077E79FED1B5AF4EEC57AF1EE10FA48BF81
:10BF500075EEE77A51E700BF83F9223EBD3786359B
:10BF6000A84A0020082E0020555555406E12833AED
:10BF700048E1FA3EA04A00200AD7233C27D4D23613
:10BF800000004842DB0F4940DB0F49C0DB0FC93FCF
:10BF900092E741B99730083C00000000DB0FC94030
:10BFA000E4CB1641E4CB16C115A82ABE0060EA48CE
:10BFB000DB0FC9BF003F0020789C00202DE9F04F27
:10BFC000DFF808B49FEDED0ABBF8104CBBF80A1C73
:10BFD000BBF80E2CABF8E82B2DED048B07EE900A86
:10BFE00062008A42F8EE677AB8BF0A4683B097B219
:10BFF00080EE270A0094ABF8184CABF81A2C019786
:10C000005EF0A2FC7D00B0FBF5F5012DB8BF012567
:10C01000EDB2B0FBF5F293B208EE903ADFEDD87ACC
:10C020008BF81C5CF8EE688AB6EE009A68EEA78A78
:10C0300007EE904AB8EEE78A0BF5426288EE280ACE
:10C0400006460BF5985909F110090BF63844C2ED74
:10C05000008A30EE090A5EF077FC07EE907AF8EE7F
:10C06000E77A022887EEA80AB8BF0220C7B28BF889
:10C07000247C30EE090A5EF067FC07EE906AF8EE69
:10C08000E77AF2EE086A86EEA77A2328BD4BA8BFAE
:10C0900023205FFA80F8A8EB070693F810228BF8AC
:10C0A000258C0BF62841013696FBF5F60136F6B2E3
:10C0B000DFEDB57AD1ED018A77EE277AC7EE276AF0
:10C0C000C1ED006A002A40F0E480AE4BDFEDAF0A1C
:10C0D000DFEDAF5ADFEDAF1ADFEDAF4ADFEDAF2A8C
:10C0E0009FEDAF3ADFEDAF3A9FEDAF4A9FEDAF1A4C
:10C0F00003F5057107EE902AB8EEE76A66EE207A3E
:10C1000037EEA57AFDEEC76A16EE903A2033402B43
:10C1100000F2D281F3EE026AB4EEE66AF1EE10FAB2
:10C120000CDD9FEDA35ADFEDA36AB0EE472AB4EE13
:10C13000E62AF1EE10FA37EE457AF6DCB4EEE47A50
:10C14000F1EE10FA0CD59FED9A5ADFED9B6AB0EE36
:10C15000472AB4EEE62AF1EE10FA37EE057AF6D465
:10C16000B4EEE57AF1EE10FA40F3A981DFED936ABF
:10C1700036EEC77A67EE076AB0EE432AA6EEA22A29
:10C18000B0EE630AA2EE260A27EE265AA5EE007A42
:10C1900027EE047AFDEEE76A16EE903A2033402B44
:10C1A00000F28781DFED866AB4EEE66AF1EE10FAFE
:10C1B00040F395819FED7E0A9FED7E2AF0EE676A3F
:10C1C000B0EE665AB4EEC25AF1EE10FA76EEC06ADC
:10C1D000F6DC9FED7A2AB4EEC25AF1EE10FA13D5CE
:10C1E0009FED732A9FED745AB0EE660AB4EEC50A4D
:10C1F000F1EE10FA76EE826AF6D4DFED716AB4EEF3
:10C20000E66AF1EE10FA0CDD9FED696ADFED696A0E
:10C21000B0EE675AB4EEE65AF1EE10FA77EEC67A4F
:10C22000F6DCF4EEE47AF1EE10FA0CD59FED606ADC
:10C23000DFED616AB0EE675AB4EEE65AF1EE10FA3D
:10C2400077EE867AF6D4F4EEE57AF1EE10FA40F362
:10C250003E81DFED5A6A76EEE77A67EEA76AB0EEC6
:10C26000435AA6EEA25AB0EE632AA6EE852A26EE1F
:10C27000A76AE6EE027A67EE847A0132242A81ED1B
:10C28000007AC1ED017A01F108017FF433AFDFEDEF
:10C290004D8A4FF0000A4FF490720021204604F8B6
:10C2A00008AC04F8077C04F8068C04F8045C04F875
:10C2B000056C60F080FC4FF49072A018002104F52A
:10C2C000127460F078FC4C45E5D107EE905AB8EE58
:10C2D000E77AF7EE007AC7EE876A9BF8D0293A4BE7
:10C2E00028488BF8D559012180F8101207EE102A42
:10C2F000B8EE476AC3ED958A87EE867AC3ED006A89
:10C30000002A00F0D180DDE90001091A07EE901A39
:10C31000F6EE006A67EE266AF8EEE77AB0EE486A53
:10C32000A7EEA66A012AF0EE466A83ED086A40F29B
:10C33000E280B7EE086A27EE066AF0EE485AE7EEAA
:10C34000865A022AC3ED095A4CD0B0EE046A27EE91
:10C35000066AF0EE485AE7EE865A032AC3ED0A5AF7
:10C3600040D0B0EE0C6A27EE066AF0EE485AE7EECF
:10C37000865A042AC3ED0B5A34D029E000247449AC
:10C38000398E633CF84F002083F9223DC3B8B23D9B
:10C39000DB0FC93F00000000DB0F49C092E741B945
:10C3A0009730083C15A82ABE72F97F3FDB0FC9BF42
:10C3B000DB0FC940E4CB1641E4CB16C1DB0F49408B
:10C3C00000001042BC297E3FD8480020003F0020DA
:10C3D000B1EE026A27EE066AF0EE485AE7EE865A98
:10C3E000C3ED0C5AB7EE086A27EE066AF0EE485A1B
:10C3F000E6EE275A424B1946E1EC016A022AC1EDEA
:10C40000005A21D0B0EE046A27EE066AF0EE485AD0
:10C41000E6EE275A032AC3ED025A15D0B0EE0C6A95
:10C4200027EE066AF0EE485AE7EE865A042AC3ED74
:10C43000035A09D0B1EE026A27EE066AF0EE485AB6
:10C44000E7EE865AC3ED045AB7EE086A27EE066A8D
:10C45000F0EE485AE7EE865A2A4B1946E1EC016A9B
:10C46000022AC1ED005A1FD0F0EE046A67EE266A78
:10C47000B0EE486AA7EEA66A032A83ED026A13D0DB
:10C48000F0EE0C6A67EE266AB0EE486AA6EEA76A7E
:10C49000042A83ED036A07D0F1EE026A27EE267ABA
:10C4A000A7EE878A83ED048A03B0BDEC048BBDE858
:10C4B000F08FF0EE617AE0E6B0EE617A6AE6B4EE13
:10C4C000C17AF1EE10FA48BF34EEC77A52E6F4EEC4
:10C4D000C17AF1EE10FA48BF74EEE77ABDE6DFEDFF
:10C4E0000A6AB4EEE66AF1EE10FA48BFF0EE676A47
:10C4F0003FF576AE95E683ED0D6A83ED126AD3E7DC
:10C500000C49002020490020000010C208480023E8
:10C5100002461178022902F1060204D00133062BEB
:10C52000F7D10020704703EB430300EB4300704753
:10C53000C01D002010B582B00A88ADF80620002387
:10C540000C468DF805308DF804004FF0B3FD042142
:10C550000DEB010031F0CCF8BDF80630238002B0BD
:10C5600010BD00BF10B582B00A788DF807201823DF
:10C57000040A8DF804308DF806008DF805404FF060
:10C5800099FD04210DEB010031F0B2F802B010BDAD
:10C5900010B582B019220023040A8DF803308DF8FB
:10C5A00001408DF800200C468DF802004FF082FD0E
:10C5B0000521684631F09CF89DF80430237002B0E4
:10C5C00010BD00BF30B5044683B000BF006942F023
:10C5D0007FF94CF2050301AA6946ADF800306068A6
:10C5E000032300258DF802505BF006FB206942F022
:10C5F00075F900BF9DF8060003B030BD2DE9F0438A
:10C60000804CDFF8208285B004F1B00024220021A4
:10C6100060F0D1FA98F835530023C4F8D430002DD7
:10C620003CD1794F2E46FB6E63B39B6A53B3774878
:10C630009847836833B30388754F013B9BB2BC4670
:10C640003D4600212878032805F106051ED001315A
:10C650000629F7D100223978022907F1060700F0F0
:10C66000A7800132062AF6D1D4F8D410052909D0C2
:10C67000481C02FB01C2C4F8D400022000219380B0
:10C6800010705180304605B0BDE8F083062303FBEF
:10C690000141B1F8B230013B9BB2DBE798F83403BB
:10C6A00008F54F73C8F8383310B9574F0026BAE76A
:10C6B00041F0CCFC0646C8F84C0300287ED08379B4
:10C6C0000BB1412BF1D1013D022368B288F83C3314
:10C6D00042F07CFD0028E8D02023C8F84003F38016
:10C6E0000921304641F04AFFD8F83833494D1869DE
:10C6F000454F42F0F3F84848D8F8386342F0F8FB69
:10C700000321024630465BF0D1F9D5F8CC00D5F8CC
:10C71000D010D8F838330090012632208DF804105C
:10C72000C7F88C3087F890603DF062FC4FF0000C49
:10C7300005236946D8F838038DF80AC002AA8DF897
:10C7400009C042F0A3FB9DF80A909DF809309DF8BE
:10C750000B104FEA092949EA034949EA0109494608
:10C7600007F16C004FF00AF930BB4846FBF7B2FF07
:10C77000034608BB9DF80B009DF80A209DF80C109D
:10C78000000240EA0240254A0843904223D0C7E90C
:10C790001D33A7F87030A7F87C30FBF79BFF0646E7
:10C7A00050B998F8340341F051FC42F04FFB3AE79E
:10C7B000062101FB02C260E7012634E7013D0223A6
:10C7C00068B288F83C3342F001FD00283FF46DAFB9
:10C7D000C8F8400384E7124A3A674FF400334FF039
:10C7E00000627B674023BA67A7F87C3087F87E60D9
:10C7F000FBF7A8FC07F16C0087F885604FF010F894
:10C80000FD6610E7101D0020082E0020742E002069
:10C81000C01D002058CC0608404B4C0021AAEF0058
:10C8200000040008F84F00202DE9F041C54BC64E2A
:10C83000C64DC74C0822C3F88820336B82B043F042
:10C840000103336307464FF4C052284640F20233D7
:10C8500088466946CDE9002308F04EFB6B6AC4F8B0
:10C86000348923F470436B626B6AC4F83C7943F4F7
:10C8700020436B626B6AB749C4F8381923F47023FC
:10C880006B626B6AB448C4F8500343F420236B62B4
:10C89000736CB249C4F8541343F480437364736BEC
:10C8A000AF48B049C4F8600343F0800302257363C6
:10C8B000AD4F84F85853AD4EAD4DC4F8A4134FF0AE
:10C8C000A043C4F85C33AB4AC4F86C7303F534631B
:10C8D000A1F5D071C4F8A853C4F87063C4F8AC33A0
:10C8E000C4F874130123DFF8BCC2C4F868C307F5A9
:10C8F0001077A5F5E465A6F5A066A1F58C61C4F8EE
:10C90000B073C4F86453C4F81C6484F85B3305F551
:10C91000A075536106F5B076C4F8E01384F862346C
:10C920001946954B954AC4F8E853A7F5BC67A0355E
:10C93000C4F8F463924EC4F8F073C4F8F83307F502
:10C94000D45703F56953C4F8FC534FF05025002029
:10C95000DFF854E2C4F82024ACF5687C02F5A0426C
:10C96000C4F82474C4F8286407F5A04706F5A04667
:10C97000C4F82C34C4F83054A3F5485304F5547566
:10C98000C4F83424C4F83C64C4F85C34C4F8E4E368
:10C99000C4F8ECC30246C4F838742B4684F8640427
:10C9A000402683F81C21A3F822210132042AC3E97E
:10C9B000496083F81D1183F81F01C3F8300103F1AA
:10C9C0002803EED1002211462B46402083F8742321
:10C9D000A3F87A230132042AC3E9DF0183F875132F
:10C9E00083F87713C3F8881303F12803EED14FF0CF
:10C9F000A04364489A6822F001029A60DA6842F023
:10CA00004002DA6007F036FB94F859330022212106
:10CA100061F317420BB142F4801294F85313D4F827
:10CA20005C3301299A6300F0E480DA68D4F85C642E
:10CA3000D4F86003C2F3076121F0600141F04001C6
:10CA400061F31F620021DA603160026861F3CC2279
:10CA5000026094F85B23012A00F0B88010214A4854
:10CA600007F05AFE484807F03DFED4F8600394F8FA
:10CA7000513300224FF0FF31026142618161C26196
:10CA800053B305F11407414E114607EB83074FEAF4
:10CA9000830C4FF0FF0E56F8042F1368002BACBF29
:10CAA00000234FF09043B74213601161C2F808E0D1
:10CAB000F1D105F15003364963440027FF2651F8B0
:10CAC000042F1568002DACBF00254FF0904599420A
:10CAD000156017619660F2D1036994F8531343F41B
:10CAE00080730129036161D0D4F85C2329480023B5
:10CAF000936100294FF0FF336FF080415161536023
:10CB0000516114BF00231023906143F470139069A6
:10CB1000D4F8381943F4605343F008030343936196
:10CB20009368096843F00103936088471A4B1B4AD6
:10CB3000DA6068461A4B0093FDF776FA02B0BDE85A
:10CB4000F08100BF00E100E0003802400000024038
:10CB5000F84F0020940B0020080401004000400121
:10CB600000080050000B0050200900504009005000
:10CB7000200B0050003C0140C00500500010005048
:10CB80000030005054530020485300205C530020D4
:10CB9000985300200008008000ED00E00005FA0531
:10CBA000430200010009005020050050D4F85C2326
:10CBB000144B03636FF08041134D00234FF0FF309F
:10CBC000936151615060516195619EE701680F4A20
:10CBD0000F4E41F003010160802159629E62C3F84B
:10CBE0000421E022C3F80821C0F24002C3F80C215E
:10CBF00034E79A6822F03E0141F02A0161F307020E
:10CC00009A6012E70301810000080080A000400044
:10CC10008000200010B51A4C94F84609C0B9194B91
:10CC200083F88900C3F88C0094F84939012B05D0AA
:10CC3000022B21D0D4F84C391BB910BD124BC4F8CB
:10CC40004C3912495B68BDE81040A1F10C0018474F
:10CC500041F0FCF994F848290A49003A18BF01222A
:10CC600081F88920C1F88C000028DDD01F22C28005
:10CC7000202141F083FCD7E7054BC4F84C39E0E7AD
:10CC8000F84F0020101D0020D40B00204859002030
:10CC9000B00B002099B10A6B824216D9154BD3F81C
:10CCA0008C29914221D34C3991421ED30B6B98426F
:10CCB000F9D38B6B9842F6D80B46184670470D4B4C
:10CCC000D3F88C190A6B904212D30B680BB9F4E7B6
:10CCD0000A6B90420B4602D38A6B9042EDD951F811
:10CCE0004C3F002BF4D1184670470023184670477C
:10CCF0000A46D8E7F84F00202DE9F047CC0143D190
:10CD00000346224A43F8082B4FF0FF3242600224C8
:10CD100018467E26DFF87880D8F890992644013EA0
:10CD2000051D49466FF070474FF0010A08E0A34225
:10CD30001CD0631C45F8043C321B1C460435CAB1A8
:10CD40000B6BA34202D88B6BA34204D22046FFF7A1
:10CD5000A1FF014690B10A794B6B002AE7D1A342AB
:10CD600004D0E6D245F8042C631CE5E745F8047CC2
:10CD7000631CE1E7C8F89019BDE8F08745F804ACFA
:10CD8000321B631C4946D8E78026C3E7F8FFFF0F34
:10CD9000F84F0020036870B55E6A26B1334605225D
:10CDA000BDE87040184704460D464E1D00E023685C
:10CDB0009B68204698470028F9D0236815F8011B86
:10CDC0001B6820469847B542F1D170BD0A44914294
:10CDD00017D010B40139541E11F8013F08225840F1
:10CDE000430010F0800F08BF400083F0D50314BF4C
:10CDF000D8B2C0B2013AF3D1A142EDD15DF8044BF3
:10CE0000704770472DE9F047164D0746002095F909
:10CE10009D9905F6A41684B007EB010805F6444574
:10CE200004464FF0B60A3368ABB193F83830142B90
:10CE300011D019F1020F01D04B450CD100226946E7
:10CE40003046CDE90244CDE90078ADF808A08DF870
:10CE50000E4031F0C9FEE036B542E4D104B0BDE881
:10CE6000F08700BFF84F002030B583B04D1C009311
:10CE700003688572C2729C690023A04703B030BD6D
:10CE80002DE9F0410C4F0124A0231825E6B2FF2B19
:10CE90000BDCC5F11B0103F10108D7F8440CDBB230
:10CEA0003246C9B2FFF7E0FF4346013DEFD10134FE
:10CEB000052CEAD1BDE8F081F84F002070B4447928
:10CEC00041BB03684FF400524FF400762025022145
:10CED0003CBB1A8C22F001021204120C1A841A8B29
:10CEE000188C22F0F30280B2120420F00A00120C17
:10CEF000014342F0010241F001011A8319841A8BA7
:10CF000022F00C021204120C1A831A8B92B270BC1B
:10CF10001A83704700220368164615461146002CF6
:10CF2000D7D0042C21D0082C38D0198C21F4805172
:10CF30000904090C19849C8B1D8C45F6FF7040F682
:10CF4000FF4128402140024342F4805241F4807165
:10CF500099831A849A8B22F440621204120C9A83E9
:10CF60009A8B92B270BC9A8370471A8C22F010028E
:10CF70001204120C1A84188B198C89B240F6FF42E5
:10CF800021F0A00102400D4342F4807245F01005EB
:10CF90001A831D841A8B22F44062B3E71A8C22F4A0
:10CFA00080721204120C1A84998B1A8C21F0F301EE
:10CFB00092B2090422F42062090C324342F48072D6
:10CFC00041F0010199831A849A8B22F00C02C4E784
:10CFD00038B50E4D0446006807F092FED5F89C2443
:10CFE000204652084FF6FF7139F03EFA20460021E4
:10CFF000FFF764FF064BC5F8083D05F608512046CB
:10D000000022BDE8384039F04FB900BF082E00209B
:10D010001D0C02082DE9F0479AB0DDE9226ADDF81F
:10D02000909004460D461746984602E020683DF071
:10D03000A7FB20683DF0ACFB0028F7D10146642235
:10D0400001A85FF0B8FD264B8DF80450CDF85CA028
:10D050000293002D40D0AB1E012B3FD9042D14BFED
:10D06000002203221F4B0396D3F808398DF80520C0
:10D070001E440123CDE9059404968DF85B3037B149
:10D080004246394607A85FF035FD8DF85A80164EA6
:10D0900096F88A9C00231893B9F1000F19D196F8DD
:10D0A000890C642202FB006001A900F68C405FF04D
:10D0B00021FD012386F8899C86F88A3C236843B1C8
:10D0C00043463A46294620461AB0BDE8F04712F0DA
:10D0D00091B91AB0BDE8F0870522C3E70222C1E783
:10D0E000405C0020101D0020F84F00200C480D4B24
:10D0F000D0F80C1D10B40C4CC0F8FC3C8A1E223138
:10D10000B0F8263D1B01A4FB03C3DB08A3F5B06305
:10D1100022F8023F9142F3D15DF8044B704700BF03
:10D12000F84F0020A97F0208CDCCCCCC70B5084CBC
:10D13000251D2E4614F8010B31F026FF28B1037887
:10D1400005F8013BB442F5D170BDFF23F8E700BFFD
:10D15000405D00202DE9F0471D4F012607F108052D
:10D16000B2464FF03C094FF0000817F8010B40F0B1
:10D170006DFF044690B180F80690C671FB7803F00D
:10D180007F02012A18D013F0800F20460DD185F8B8
:10D19000048041F09DFB85F805802C600136052E4A
:10D1A00005F10805E1D1BDE8F08785F804A041F05C
:10D1B00095FB85F805A0F0E71B0605D40121204664
:10D1C00041F0DCF9FB78DEE741F088FBF6E700BFD1
:10D1D000485D00202DE9F04FDFF8E491DFF8E4A18D
:10D1E00083B009F10C05012419F8018BB8F1000F87
:10D1F00000F0C0804FEA1817013F042F08F00F021B
:10D2000000F2BB800AEB4703B3F8840040FA02F651
:10D2100016F0010600F0C38001239340013B184043
:10D2200057445CF0E3FA97F890305F4E184406EBF1
:10D23000C00604236E61F471B371002303E001336F
:10D24000152B00F09780594903EB43025F00895C7E
:10D250004145F4D1564B1A4492F8B111002900F01F
:10D26000A080404639F062FA8046006839F002FA40
:10D2700098F8051039F07AFA0378002B7AD14C4BE4
:10D280003B44042283F8F14183F8F021002E58D06A
:10D29000336898F8080003F13F4202F57E020AEB7A
:10D2A0009222012792F8982002F01F015209032AC6
:10D2B00007FA01F169D0042A62D0022A6AD0B6F8CE
:10D2C00004C0BCFA8CF2C2F11F02C2F3CC0103EB22
:10D2D000810102F007020E6A92000F27974026EAAA
:10D2E00007060E620E6A90403043002208624FF03B
:10D2F000010B11460BFA01FE3EEA0C001CD1186826
:10D300000326964020EA060018601F68022090401D
:10D31000384318609F6827EA06079F6098689860FE
:10D32000586820EA0E00586058685860D86820EAAB
:10D330000600D860D868D8600131102902F10202D5
:10D34000D8D11C4B1C4AB3F8781DB3F87A3D009134
:10D35000002001340190B2FBF3F328469BB2414612
:10D36000E4B230F09FFE0123092C6B7405F118051F
:10D370007FF43AAF03B0BDE8F08F00266E615CE742
:10D380000E4F3A6B0A433A6399E70C4A176C3943DC
:10D39000116494E7094A576C394351648FE76E6111
:10D3A0004BE70B68FFDE00BF24300020B82F0020C1
:10D3B000082E0020F84F002040420F0000380240A5
:10D3C000745D002058CC06082DE9F041214E224F13
:10D3D00096F84B3E87F8703E06F6486607F6746589
:10D3E00000244FF0050816F8010B20BB286001341B
:10D3F000032C05F10405F6D197F8701ED7F8740ECA
:10D40000C94301F0010141F06FFA97F8701ED7F897
:10D41000780E81F00201C1F3400141F065FA97F8FE
:10D42000701ED7F87C0E81F00401BDE8F041C1F315
:10D43000800141F059BA40F009FE01340121286011
:10D44000E3B210B180F80680C371286841F096F805
:10D45000CEE700BFF84F0020082E00202DE9F04154
:10D460002A4C2B4DB4F8506EA5F8806E82B0EEB900
:10D4700094F84C0E40F0EAFD94F84D2EC5F8840E59
:10D48000003A18BF012285F8822E48B194F84E1E4A
:10D490002B22002914BF11210121C28041F06EF816
:10D4A000002002B0BDE8F0413CF074BE94F84C8E10
:10D4B000002240462B2139F0A9F90746404640F0AA
:10D4C000C5FDF8B1F7B12B22C5F89C0EC280397AA0
:10D4D000FCF7EAFD4FF000080E4AB2FBF6F3C3F387
:10D4E0004F0000909BB23946CDF8048005F6886065
:10D4F000A4F8526E30F0D6FDD5F8883EC3F800800F
:10D5000085F8998E02B0BDE8F08100BFF84F002089
:10D51000082E002040420F002DE9F84F254C94F8CA
:10D52000603E84F8543E04F65767002604F674649F
:10D530005FFA86FB0BF101085FFA88F8012117F802
:10D54000010F42460E448A4639F060F94FF0000957
:10D55000054640B3387804F80E9C04F80D9C04F896
:10D560000FBC04F810AC44F8045C40F06FFD18B137
:10D5700080F806A080F80780297AFCF795FD0E4A0E
:10D580000021284638F070FF0C4B23600C4B221D05
:10D5900021462846C4E9013938F086FE69792868B1
:10D5A0004A4630F05DF8082E04F11C04C0D1BDE8F5
:10D5B000F88F00BFF84F002040420F0099D60308B3
:10D5C0004935030870B52C4C2C4B94F88C0FC4F8DB
:10D5D000843F00220221C4F8442FC4F8482FC4F825
:10D5E0004C2FC4F8802FA4F8882F39F00FF90028A9
:10D5F00041D0234B0268054603F1C000597C11B1AC
:10D6000059688A422BD018338342F7D1002394F80B
:10D610008C0FC4F8705E84F8643E40F017FD08B1CA
:10D620000223C380297AFCF73FFD2846154A0021D2
:10D6300038F01AFF144A1549C4F8741E0026111F49
:10D640002846134BC4F8783EC4F87C6E38F02CFEA4
:10D65000697928683246BDE8704030F001B8138D12
:10D660000C490D4A9BB2D2F89C240133B2FBF3F370
:10D6700081F8603ACAE770BDF84F002000FFFF0054
:10D68000F82E002040420F00705E00207135030824
:10D690001137030898010020082E00202DE9F04FD3
:10D6A000C64EC74D87B089460446C02206F1F00039
:10D6B0000021CDF80C905FF07EFA95F8F83F002B32
:10D6C00000F0DD8095F8F93F002B00F0F78096F828
:10D6D000DC30012B69D0022B00F0FC80B94BBA4F33
:10D6E00004931C460FCF0FC40FCF0FC497E8070059
:10D6F00096F8D2C096F8CE30DFF8F882B34FC5F86E
:10D70000DC7F84E80700BCF1000218BF0122072B70
:10D7100008F8F72C00F23081042B00F26D81DFF85D
:10D72000B8B20027ABF11209039BBB424FF00301D3
:10D7300039DD19F801AB06EB0A030AF1010893F889
:10D74000D3405FFA88F82046424639F05FF8034636
:10D7500020461C46002B00F0298140F077FCCBF8D6
:10D76000140020B14FF00303837180F8078096F80E
:10D77000CF2096F8CE30F9B2002A00F01581E27978
:10D7800082F00102009220465246013758F02EFFE7
:10D79000002800F00B814FF00103082F8BF81130A7
:10D7A0000BF1180BC0D1049B67E0894F894C96F8A8
:10D7B000D2C0DFF840820FCF0FC40FCF0FC497E85D
:10D7C000070084E807000021039B834F48F8F43CDE
:10D7D000BCEB010C96F8CE3008F8B43C18BF4FF003
:10D7E000010CA8F1B0004FF44072059708F8F7CC8F
:10D7F00008F8F61C89465FF0DEF9A7F1120308F578
:10D80000147B049358F8F43C4B4540F3AD80049AE4
:10D8100012F8013B0492334493F8D340204639F088
:10D8200029F80746204640F011FC96F8CF30044610
:10D83000002B00F09B80FB7983F0010A0AF00107BE
:10D8400018F8F70C013708F8F87C08B18AF0010ADB
:10D85000002C00F09880A17900295AD0412958D095
:10D860005E4B5F495F4AC5F8AC3F012308F8F63CC0
:10D87000C5F8A81FC5F8B42F0023C5F8FC3FD5F89C
:10D88000FC3F63B10022039883F82C00012183F848
:10D890002D101A6383F82E2007B0BDE8F08F524E8A
:10D8A000524C0FCE0FC40FCE0FC496E80700A4F160
:10D8B000200384E80700C5F8FC3FEDE796F8D02088
:10D8C0000399003A204618BF0122FAF79DFFC5F8D8
:10D8D000FC0FD4E796F8D230002B3FF4FFAE96F859
:10D8E000CE30082B7FF461AF374FDFF808810FCFC0
:10D8F00005F6C47404940FC40FCF0FC497E8070053
:10D90000324BC5F8DC3F012784E8070008F8F77CB4
:10D9100035E0204640F0FAFF790109F1010941F0B4
:10D9200009014FF00303CBF81410CBF80400CBF837
:10D930000C408BF810A084F80790A371204640F0AB
:10D940001DFE1AF0010F204613D040F0C1FF059ACA
:10D95000DBF80C305361B9F1080F02F118030BF139
:10D96000200B05937FF44EAF1A4B86E797F807A07C
:10D9700064E740F0B3FFEAE7082B7FF4D0AE1C4B1E
:10D9800048F8F03CCBE6204640F0C0FF7F0147F06E
:10D99000090109F10109CBF81410CBF80400CBF808
:10D9A0000C408BF810A0C9E7E279EBE60D4B0B4A6F
:10D9B000C5F8E83FC5F8E02F00235EE7082E0020F9
:10D9C000F84F0020BC5F002058CD0608D53D060862
:10D9D00084CD0608885F0020F82E0020F549040851
:10D9E000F9490408ED4904082CCD06080860002018
:10D9F000C9D80408F060002096F8D130064A48F8EB
:10DA0000F02C012B05D0022B06BFBCFA8CF35B096E
:10DA1000002308F8EC3C82E6F9D804082DE9F0412F
:10DA20006E4F97F8200D97F8215D40F00FFB60B125
:10DA30002D23C3802021044640F0A0FD0A2039F0A8
:10DA40001FFB204640F058FF28B9DFF89881D8F82E
:10DA50005033DA0001D5BDE8F081013D092DFAD837
:10DA600097F81F4DD4B9402033F042F80028F2D087
:10DA700090F9043097F8F51C092BC8BF143B4344B8
:10DA80000A2993F8544300F09B8093F8603397F889
:10DA90001E2D002A08BF1C46002CDCD0204640F07A
:10DAA000D5FA0546002800F083802D23C38001218C
:10DAB00040F064FD0121084638F05CF92B68AA8823
:10DAC0001A833C203CF094FA0021012038F052F9EE
:10DAD00097F8213D002B4CD0414C00261FE02B68CD
:10DAE000AA885A8339F0CCFA94F8701ED4F8740ED0
:10DAF00001F0010140F0F8FE94F8701ED4F87C0E9D
:10DB0000C1F3800140F0F0FE2B68AA881A837820C8
:10DB100039F0B6FA97F8213D01369E4229DA94F899
:10DB2000701ED4F8740EC94301F0010140F0DCFE10
:10DB300094F8701ED4F87C0E81F00401C1F38001CA
:10DB400040F0D2FE7820002DC9D1782039F098FA23
:10DB500094F8701ED4F8740E01F0010140F0C4FE78
:10DB600094F8701ED4F87C0EC1F3800140F0BCFE26
:10DB7000CDE797F81F3D9BB9D7F8203D03F0FF1381
:10DB8000B3F5803F7FF467AFD8F8503313F080537C
:10DB90007FF461AF87F8213DBDE8F0414CF05CBDFA
:10DBA00032203CF025FA2846002140F0E7FCE3E76C
:10DBB000012140F0E3FC0121084638F0DBF880E762
:10DBC000D8F878335B057FF546AF09F037FD0028BC
:10DBD0007FF441AF002C7FF461AF3CE7F84F0020A9
:10DBE000082E0020F0600020084BD3E9DF029042AD
:10DBF000D3F8843302DC114602460846984204DD1D
:10DC00009A42B8BF1A46104670477047F06000202D
:10DC10000B6810B414681B1B036054684B681B1B13
:10DC200043608B6892685DF8044B9B1A8360704771
:10DC30002DE9F047041E0D4612DB092C26DC824A32
:10DC40000B468248A0FB0410C00800EB8000A4EB48
:10DC500040000021125C1A7059702846BDE8F08718
:10DC600064422D23092C01F8013B24D8764A774BD6
:10DC7000A3FB0403DB0803EB8303A4EB43030020B3
:10DC8000D35C48700B702846BDE8F0876F4B632C5F
:10DC9000A3FB04264FEAD60621DC6B4A0B466B49F0
:10DCA000A1FB0601C90801EB8101A6EB4101515C12
:10DCB00003F8011BC5E7654A632CA2FB04364FEA53
:10DCC000D60637D8604A614BA3FB0603DB0803EB9B
:10DCD0008303A6EB4303D35C01F8013BC7E7A3FB37
:10DCE0000627B4F57A7F4FEAD7070DD2564A0B467E
:10DCF0005649A1FB0701C90801EB8101A7EB4101CE
:10DD0000515C03F8011BCAE7A3FB072842F20F721C
:10DD100094424FEAD80836D84B4A0B464B49A1FBF0
:10DD20000801C90801EB8101A8EB4101515C03F82E
:10DD3000011BDDE7A2FB0637B4F57A7F4FEAD70770
:10DD40000CD2414A414BA3FB0703DB0803EB8303DF
:10DD5000A7EB4303D35C01F8013BB4E7A2FB073810
:10DD600042F20F739C424FEAD80821D8364A374B0B
:10DD7000A3FB0803DB0803EB8303A8EB4303D35C9B
:10DD800001F8013BDEE7324AA3FB080994424FEA5F
:10DD9000D90921D82C4A0B462C49A1FB0901C908F5
:10DDA00001EB8101A9EB4101515C03F8011BB5E7CF
:10DDB000274BA2FB08099C424FEAD90921D8224AE5
:10DDC000224BA3FB0903DB0803EB8303A9EB43030B
:10DDD000D35C01F8013BCAE71E4AA3FB0903944246
:10DDE0004FEAD30A21D80B461849174AA1FB0A016A
:10DDF000C90801EB8101AAEB4101515C03F8011B49
:10DE0000CAE7144BA2FB09029C424FEAD20A13D87C
:10DE10000E4B0D4AA3FB0A03DB0803EB8303AAEBBB
:10DE20004303D35C01F8013BCAE70A22BAFBF2F0D4
:10DE30004CF0DEF90346D7E70A22BAFBF2F04CF0C9
:10DE4000D7F90146E4E700BFBC5C0708CDCCCCCCD9
:10DE50009F8601003F420F0070B4344890F8883329
:10DE6000A3F13001092957D800F56274224600F267
:10DE7000973012F8015FA5F13001092904D88242D8
:10DE8000F7D1002070BC7047141B022C4ADD2848D3
:10DE9000002101E010F8013B01EB810103EB41039C
:10DEA000161A303B022E044603F0FF01F2DC214B30
:10DEB00003FB01F1A2424FF000030DD903EB8303F2
:10DEC00014F8016B5B00303B3344A24203F0FF03C4
:10DED000F4D1194800FB03F32E2D06D01748A0FB00
:10DEE000032301EB930070BC70470132042000242F
:10DEF000157804EB8404303D6400092D00F1FF30F7
:10DF0000A4B202D82C44A4B2013210F0FF00EFD129
:10DF1000642202FB0433E1E700211D4600F5627232
:10DF20000B46D9E7064C0021C4E700BFF060002093
:10DF3000796400208096980040420F00ABAAAAAAFC
:10DF40007864002038B504460D460A460068FF2173
:10DF50005EF031FE21682944216038BD83B50C464E
:10DF60001646054631F07EF8204631F07BF8002158
:10DF7000204B0846002E08BF1E4637F0FBFE00214E
:10DF8000012037F0F7FE28463CF002FCB0B1012139
:10DF9000002037F0EFFE28463CF0F2FB0746204613
:10DFA0003CF0F2FB0028FAD0394620463CF0F4FB66
:10DFB0003846B0470021084637F0DCFE20463CF0EA
:10DFC000E7FB0028DFD00121002037F0D3FE2046F8
:10DFD0003CF0D6FB0146284601913CF0D5FB019967
:10DFE0000028F8D028463CF0D7FB0021084637F03F
:10DFF000C1FEC8E799D80308F0B50023C1E9003392
:10E00000C1E902330B610268DFF88CC089B004AD4E
:10E01000C2F385572E4647FA03F0C007344604D5AD
:10E0200013F80C0004F8010B26460133062BF2D13D
:10E030001748C2F303240444002394F8604133706A
:10E040008DF8184000F5B47CC2F305370DF11906C0
:10E0500047FA03F0C007344604D513F80C0004F85F
:10E06000010B26460133062BF2D100233370C2F395
:10E07000834406ABCDE90134084602F00F0305499D
:10E080000095C2F303124CF0EBFE09B0F0BD00BFE7
:10E0900058CC0608E45C0708B0CD060870B5094CFA
:10E0A000D4F89823054662B10026D4F898032D21B0
:10E0B000013641F04BFAAE42F7DBBDE8704041F06B
:10E0C000F3BC70BDF06000202DE9F04F5FFA81F9DC
:10E0D000002185B007460846164637F04BFE002162
:10E0E000012037F047FE3FF01BFA022E0AD0042E23
:10E0F00044F6C01818BF4FF49648B9F1070F07D976
:10E1000000200CE0B9F1FF0F4FF41648F5D10326BB
:10E11000BE4D95F89C332BB90020C5F8A00305B07F
:10E12000BDE8F08F032EBA4C0DD0A144002299F81F
:10E13000D300032138F06AFB0028EDD0C4F8E404D2
:10E14000C3799A07E8D495F89C0384F8FF6C002201
:10E15000032138F05BFBC4F8E8080028DCD0AD4AA6
:10E16000AD4BC4F8A03402F1480003234FF48061A2
:10E17000A4F8A434C4F8B404002302F24C404FF0D5
:10E18000010A032EC4F8A884C4F8CC34C4F8AC1433
:10E19000C4F8C034C4F8BC34C4F8B804C4F8B0142B
:10E1A000C4F8C834C4F8C43484F8F03CA4F8ECAC27
:10E1B000C4F8F83CA4F8FC3C84F8FE3C91460ED030
:10E1C000D4F8E4B49BF804003FF040FFC4F8E00446
:10E1D000584614F0E1F85146484614F0F1F8322060
:10E1E0003BF006FF012E09D1D4F8E8084146FAF7C2
:10E1F000F9FCD4F8E404FEF7EBFE0AE0022E3BD172
:10E20000D4F8E40414F0B7F8D4F8E8084146FAF773
:10E21000E9FCC5F8A0934FF0060A022E11D0D5F8FC
:10E22000A0033CF0B5FA60B10121002037F0A2FD57
:10E23000D5F8A0033CF0ACFA014600287FD137F0B6
:10E2400099FD38463CF0A4FA80B10121084637F028
:10E2500091FD4FF0050B4FF0000838463CF098FA5E
:10E260000146002874D1012037F084FD042ED6D059
:10E2700005203BF0BDFED0E7032E58D14FF0000A39
:10E280005146664884F800AD40225EF094FC8DF85B
:10E290000FA04FF0010A9DF80F30072B09D95D48F8
:10E2A000012114F08DF8D4F8E8084146FAF79AFCF9
:10E2B000AFE79DF80F3003EB430304EBC30393F880
:10E2C00001316BB39DF80F3003EB430304EBC30341
:10E2D000D3F8043123B39DF80F30234493F8D300CF
:10E2E000F0B10022032138F091FA8346C0B114F056
:10E2F00042F89DF80F3094F8002D03EB430304EB34
:10E30000C30305EBC201D3F80431C1F8A4339BF871
:10E3100007300132DB0748BF81F8A8A384F8002D3D
:10E320009DF80F300133DBB28DF80F30B3E7042EC8
:10E330007FF46FAFD4F8E40414F01DF854E7D5F877
:10E34000A0033CF01DFA014638463CF025FA6FE781
:10E3500038463CF015FA95F8F23301468BB924287B
:10E3600003D14FF0010385F8F233012E04D1384672
:10E3700001913CF011FA0199D5F8A0033CF00CFA98
:10E380006BE7012B06D14D280CBF0223002385F833
:10E39000F233EAE7022B06D13C280CBF032300230B
:10E3A00085F8F233E1E7032B10D10A2802D985F86A
:10E3B000F283DAE7042385F8E50385F8E48385F83A
:10E3C000E78385F8E60385F8F233CEE7042B09D11D
:10E3D00095F8E63385F8F303434085F8E63385F88E
:10E3E000F2B3C2E7052BC0D195F8E43395F8E59375
:10E3F00095F8E6034B4513D25A1C2B44484085F848
:10E40000E60385F8E42383F8E813AEE7F060002024
:10E41000082E0020A8320020C8CD060894640020F1
:10E420008842C4D195F8F33385F8F2A3F42B9CD13C
:10E43000B9F1000F99D12421384685F8F2933CF0C8
:10E44000ABF94D2138463CF0A7F93E2138463CF067
:10E45000A3F9494638463CF09FF9F42138463CF090
:10E460009BF9F42138463CF097F9032E1BD0D4F8E1
:10E47000E404437901689D080223AB40DB439BB26F
:10E480000B828D892B408B810079202113F062FF54
:10E49000D4F8E4044A46494637F006FFD4F8E43499
:10E4A000186806F02DFC0022D4F8E808114637F071
:10E4B000FBFED4F8E838186806F022FC01202EE6AE
:10E4C00038B50F4C94F8FB1301F03F018B1C02464A
:10E4D00001F10A0584F8F93384F8F65304F57D70E8
:10E4E00084F8F72308311EF0DDFB254485F8F2039C
:10E4F00094F8F6331C44000A84F8F30338BD00BFD7
:10E50000F060002070B51D4C0968D4F820541C4EF2
:10E51000D4F81C44D6ED007ADFED1A6A491B00EEF0
:10E52000901A0168F8EEE00A091B60EEA70A00EEF7
:10E53000101A20EEA07AB8EEC00A1C46A0EE007AAF
:10E54000B1EE400AF1EEC77A67EEA67AFCEEE77A02
:10E55000C2ED007A4CF054FD9FED0B7ADFED0B7AA3
:10E56000E0EE077AFDEEE77A17EE902A002ABCBFAC
:10E5700002F50C42A032226070BD00BFF0600020A6
:10E58000FC0B00202C7D8E3FA00CB34500A00C4658
:10E5900038B50B4C002501228021204632F094FA38
:10E5A00030B194F9040032F0C3FA08B1006838BD04
:10E5B0000135062D04F10C04EDD10020F7E700BF72
:10E5C0002465002038B5041F00F1080554F8043F05
:10E5D000D81780EA430015F081FEA542F6D138BD78
:10E5E00070B5B54CDFEDB57AD4F8803494F8C854E2
:10E5F000B4F8CA6407EE103A2DED028BB8EE478AE4
:10E6000028EE278A002D59D1D4F8D43494F8E52483
:10E61000002B40F3DF8007EE902A9FEDA96ADFED23
:10E62000A96AF8EEE77AB7EE007AA7EE867AF0EEFE
:10E63000477A07EE103AF8EEC78AB7EE087A87EE07
:10E64000270AC6EEA87A20EE270A5CF07DF994F836
:10E65000C93485B2A4F8CA54002B00F00D81AE4233
:10E6600030D007EE905ADFED986A94F88454F8EEB3
:10E67000677A86EEA77A37EE087AC8EE077A95B3FE
:10E68000B4F8CC3494F8CE24B4F8D06406EE103A42
:10E69000B8EE466A8D4B86EE867AC3ED047AC3EDFA
:10E6A000087AC3ED0C7A77EE087A88EE277A83ED44
:10E6B000107A002A41D0BDEC028B70BD94F8C904D9
:10E6C00000287BD094F88454002D40F0CD8007EED4
:10E6D000906ADFED7D6AF8EE677A86EEA77A37EE0C
:10E6E000087AC8EE077AB4F8CC3494F8CE54B4F86B
:10E6F000D064002206EE903A9FED736A734BF8EEF9
:10E70000666AC3ED047A86EE267A5A609A60DA6009
:10E710005A619A61DA615A629A62DA625A639A635A
:10E72000DA63C3ED087AC3ED0C7A77EE087A88EEE7
:10E73000277A83ED107A002D56D1D4F8D43494F88A
:10E74000E524002B40F3858007EE902A9FED5C6A5C
:10E75000DFED5C6AF8EEE77AB7EE007AA7EE867A2C
:10E7600007EE903AF8EEE77AB7EE086A86EE070A07
:10E7700086EEA77A20EE070A5CF0E6F880B2A4F8ED
:10E78000D00485B3B04296D0002894D007EE900A0A
:10E79000DFED4D6A4E4BF8EE677ABDEC028B86EEEC
:10E7A000A77AD3ED006A37EE267AC6EE877AC3EDF4
:10E7B000CC7AC3EDD07AC3EDD47A70BDD4F8D4341A
:10E7C00094F8E624002B75DD07EE903A3546F8EE16
:10E7D000E78A53E094F8C904A4F8CA5400287FF4E7
:10E7E0003EAF054663E0064694F8E43484F83D38CD
:10E7F000002E3FF460AF07EE906A9FED336A344B12
:10E80000F8EE677AD3ED006A86EE277ABDEC028BCC
:10E8100000220121C3F8242384F83C18C3F82823DC
:10E82000C3F82C23C3F83423C3F83823C3F83C239C
:10E8300037EE267AC3F84423C6EE877AC3F8482316
:10E84000C3F84C23C3EDCC7AC3EDD07AC3EDD47AB0
:10E8500070BD0023A4F8D034002D7FF42CAF94F8C1
:10E86000E43484F83D3826E794F8CE34B4F8D06424
:10E87000002B7FF420AF60E794F8E6249FED106A48
:10E88000DFED106A07EE902AF8EEE77AB7EE007A2D
:10E89000A7EE867AF0EE477AB7EE087A87EE270A77
:10E8A000C6EEA87A20EE270A5CF04EF880B2A4F8F3
:10E8B000CC04D4E63546FAE7F0600020BD37863553
:10E8C000CDCCCC3D002474494E2DA63D746500206E
:10E8D000D86500201D4991F88823A2B3F0B4002622
:10E8E00005463346304637461BB991F888432D2CF0
:10E8F00023D02E2A19D0CA1800EB800092F8884342
:10E90000A4F13002092A4FEA40009CBFA0F1300276
:10E91000A0180E2B14D80133CA1892F88823002AA5
:10E92000E2D106B14042F0BC70470133002DF8D06F
:10E93000CA182A4482F88873DDE701231E46EBE7F4
:10E940000020F0BC70470020704700BFF06000203E
:10E950001FB503AC8DF80C30009400238DF80D30FA
:10E960000DF090FC04B010BDF8B50546262027F048
:10E9700025FB134C0146F8B9D4F8880890F83830D4
:10E980001E3B012B01D93BF007FF0E4F0026AE4284
:10E990000ADBB4F8AC380133A4F8AC380A4BD3F82E
:10E9A0000839C4F8BC38F8BD17F8011BD4F888083A
:10E9B0003BF0F2FE0136EAE7002384F8BA38EDE7CF
:10E9C000F06000207C690020101D002010B580211F
:10E9D000044605F035F82046002105F031F82046C0
:10E9E000BDE8104005F06CBB2DE9F041B14C94F846
:10E9F000D338C4F8C00882B088465A2B00F2B980D8
:10EA0000DFE813F0CC00B700B700DC00B700B700B8
:10EA1000B700B700B700B700B700B700B700B7003E
:10EA2000B700B700B700B7000F01B700B700B700D5
:10EA3000B700B700B700B70033017400B700B700E4
:10EA40007400B700B700B700B700B801B7006201A3
:10EA5000B700B7007C00B7000902B700B700B700E5
:10EA6000B7005B00B700B700B700B700B700B7004A
:10EA7000B700B700B700B700B700B700B700B700DE
:10EA8000B700B700B700B700B700B700B700B700CE
:10EA9000B700B700B700B700B700B700B700B700BE
:10EAA000B700B700B700B700B700B700B700B700AE
:10EAB000B700B700B700B700E40194F8D4389B075B
:10EAC00000F16982B4F8DA38D4F8D528D4F81419EA
:10EAD0005BBA9BB212BAD0188842C4F82039C4F885
:10EAE0001C2903D904F06CFF002854DB0020A4F893
:10EAF0000C090546284602B0BDE8F08194F81839A3
:10EB0000002B40F0FF8094F9D038002B31DAD4F894
:10EB1000083908469B689847002840F01E82B4F8E0
:10EB2000DA08D4F8D528D4F8143940BA80B212BA29
:10EB300015189D42C4F82009C4F81C2907D904F00F
:10EB40003FFF002827DBD4F81C29D4F82009D4F88B
:10EB50001039D4F8CC6803FB00F003FB02F2022565
:10EB6000B042C4F81C29C4F8200984F8185900F0F0
:10EB7000CF8094F8E4385A1CD2B204EBC3030520CA
:10EB80004FF40051042A84F8E42883F8E808C3F815
:10EB9000EC1800F0A0814FF0FF35ABE7D4F8CC388B
:10EBA000002BE6D1D4F8083908469B6898470546FB
:10EBB000002840F0D281A4F80C099BE73E4B0022CC
:10EBC00003F1120103F8012F8B42FBD13B4994F86A
:10EBD0000E3994F8E40870250D7098424FF00C053A
:10EBE000CD7110D004EBC300013390F8E8588D705C
:10EBF000B0F8EC08DBB2042B40BA888114BF84F86B
:10EC00000E3984F80E2994F8D73812229342A4F8CA
:10EC10000C2998BFA4F80C390025284602B0BDE89D
:10EC2000F08194F8D438DA0700F13E81D4F808393D
:10EC300094F8D708DA6901EBC10102EB81010A7986
:10EC4000531D834228BF0346A4F80C39002BE3D0A0
:10EC5000013B1A489BB201331944034411F8012DBA
:10EC600003F8012D8342F9D1D6E7154E154F3546ED
:10EC70000823073EC5F10700A4F80C39002202E082
:10EC800092F8A8211D462B46B54203F8012900EB56
:10EC9000030217FA82F2F3D1D4F808394046DB6850
:10ECA00098470028B8D0AB7863F07F03AB7000259D
:10ECB00020E700BFF0600020778C0020788C0020D7
:10ECC0007F8C002058CC0608D4F80839C74A5B6806
:10ECD0000846111D98470546002840F03E81D4F8AB
:10ECE0001439C34AD4F81019013B180E1070180CCF
:10ECF00009BAD37050701B0A082093705160A4F8B1
:10ED00000C09F7E6D4F82069D4F81C29D4F8103996
:10ED1000D4F80859B2FBF3F24FF48057BE4228BF33
:10ED20003E462D69B249A4F80C794046B6FBF3F390
:10ED30009BB2A8470028C0F2BC803346AC4AD4F846
:10ED4000C008812104F0B0FED4F81C29D4F82009B1
:10ED5000D4F82C393244851B9E1BC4F81C29C4F8F6
:10ED60002059C4F82C69002D7FF456AF032384F892
:10ED70001839BFE69E4E0027334606F10C0203F811
:10ED8000017B9A42FBD1D4F8083940465B686A4659
:10ED900001A998470546002840F0E980019BBDF88D
:10EDA0000020013B190E52BAF3713171190C1B0A84
:10EDB00071710820B371022172810C23BDF8022009
:10EDC000F07031727272A4F80C3993E6894E8A4F52
:10EDD00030460823073EC0F10705A4F80C3900228D
:10EDE00002E092F8B02118460346864203F8012952
:10EDF00005EB030217FA82F2F3D1D4F80839404642
:10EE0000DB68984700283FF407AFF37863F07F038F
:10EE1000F37000256EE694F81839002B61D194F94F
:10EE2000D038002BFFF6A5AED4F8083908469B6809
:10EE30009847002840F09180D4F808394046DB68B4
:10EE400098470546002840F0BA80B4F8DA38D4F87C
:10EE5000D528D4F814195BBA9BB212BAD0188842DC
:10EE6000C4F82039C4F81C2900F29F80D4F8101986
:10EE7000D4F8CC0803FB01F302FB01F28342C4F88F
:10EE80001C29C4F820397FF474AEB3F5805F28BF25
:10EE90004FF480530121D4F8C008554A84F818195A
:10EEA0009BB204F02BFF25E607235449A4F80C3944
:10EEB000CEE694F8E4385A1CD2B204EBC303042023
:10EEC0004FF48851824284F8E42883F8E808C3F8B4
:10EED000EC187FF460AE002384F8E4384FF0FF357F
:10EEE00008E6D4F82069D4F80809D4F81039D4F821
:10EEF0001C294569B2FBF3F2B6F5805F28BF4FF4D9
:10EF000080560846B6FBF3F339499BB2A847002860
:10EF100062DBD4F81C29D4F82059D4F82C393244B7
:10EF2000AD1B9B1BC4F81C29C4F82059C4F82C390C
:10EF30002DB9D4F8C008294604F034FFDAE5B5F558
:10EF4000805F28BF4FF48055ABB2D4F8C008284A80
:10EF5000012104F0D3FE0025CCE594F8E4385A1CD6
:10EF6000D2B204EBC30302204FF468510AE694F8CE
:10EF7000E43804EBC3020133DBB202204FF46851E2
:10EF8000042B82F8E808C2F8EC1822D084F8E438A0
:10EF90004FF0FF35AEE594F8E4385A1CD2B204EBDA
:10EFA000C30305204FF41051ECE504F009FD0028DF
:10EFB000FFF6F1ADD4F81C29D4F8203956E794F8BF
:10EFC000E4385A1CD2B204EBC30302204FF41C51A4
:10EFD000D8E584F8E478DEE594F8E4385A1CD2B237
:10EFE00004EBC30304204FF440716BE7006A002078
:10EFF000788C00207F8C002058CC0608F8CD0608BD
:10F0000010B51C203FF022F8112104463FF0B6FA5B
:10F0100020463FF05DFCC8203AF0EAFF2046BDE8FC
:10F0200010403FF05BBC00BF08B500203FF00EF879
:10F03000054BC3F8340908B12A23C380BDE8084052
:10F0400040213FF09BBA00BFF06000202DE9F04F57
:10F05000B34CD4F85C335A69D2078BB002D50BB0ED
:10F06000BDE8F08F5A699B6912EA030AF7D0CAF328
:10F0700007431AF4002F009340F00281009B5D07C4
:10F0800043D41AF0020F5FFA8AF503D0D4F85C3348
:10F0900002225A61BAF1000FC0F20D821AF4006F19
:10F0A000CAF3072740F082812E0708D59D4B9E4862
:10F0B000D3F8743A9847D4F85C3308225A61ED06C5
:10F0C00000F1E581F80600F1A581B90600F12E8175
:10F0D000009BDA0609D5934B9348D3F8843A9847B6
:10F0E000D4F85C334FF480125A61009B9B06B6D56E
:10F0F0008C4B8D48D3F8883A9847D4F85C334FF45A
:10F1000000125A610BB0BDE8F08FD4F86023936908
:10F11000D26913401FFA83FBBBF1000FB1D0DFF8B7
:10F120000882CDF80CA045464FF0000909E05FEADF
:10F130005B0B09F1010908F1040805F1280500F04D
:10F14000D6811BF0010FF2D0D4F860135FFA89F773
:10F1500008694A6B04EB8703FA40D3F86833D2019D
:10F160009B68D2B202431A40D007D3B216D54B6B7C
:10F17000D8F81820012000FA09F023EA00034B63B5
:10F18000684B6948D3F86C3A012191603946984739
:10F1900094F85363012E00F0F88101231A0703D578
:10F1A000D8F8182008239360DE0603D5D8F8182075
:10F1B00010239360580603D5D8F818204023936095
:10F1C000990703D5D8F81820022393601A06AED504
:10F1D000D5E94C60D5F82431D8F818C0311A8B42E3
:10F1E000DCF8182028BF0B46033392B2B2EB930F22
:10F1F0009DD9D4F86023323704EB8703CDE9019819
:10F2000090469946B04238D2BEB3D5F8241194F84E
:10F210005333D5F82821371AB94228BF394601F1AE
:10F22000030E4FEA9E0E83B98FB20337BF10D9F891
:10F2300058A30AD0013352F8040BCAF800009F42C9
:10F24000F8D1D5E94C60D5F82821DCF8183008440D
:10F250000A44B042C5F82821C5F834010AD195F80E
:10F260001C11D8F83420012707FA01F122EA010223
:10F27000C8F834209BB29E45C4D3DDE9019856E717
:10F28000D4F860339D69DB691D402D0C3FF4F6AE68
:10F2900004F55476DFF88CB0B046B146002708E09C
:10F2A0006D0807F1010706F1040608F128083FF48C
:10F2B000E5AEEB07F4D5F9B204EB8102D4F8603384
:10F2C000D2F8A42392685B691A40D007D3B218D54C
:10F2D00094F85303726D01239842936007D1126929
:10F2E000D8F87C33C2F312029B1AC8F88C33DBF8CF
:10F2F000683A4846984794F85333012B00F05381FD
:10F3000001239A0702D5726D022393601B07C7D5AC
:10F31000DBF8703A48469847736D08229A60BFE759
:10F32000F84F00209801002048530020D4F86033A3
:10F33000D4F868139A680868C2F34102022A08BF29
:10F3400003224FF0000514BF65F30A0062F30A00C0
:10F3500008605A6842F480725A6006A805F07EFD83
:10F36000D4E9D720D368BE49079D6FF38D23D360BE
:10F370008068C0F34100014491F8B811032900F0FE
:10F38000CD80B849B8480126294484F852638142A7
:10F390004FF04006A4F8546300F213810E2161F38C
:10F3A0008D234FF40051D360516191E6AF4B94F837
:10F3B0006224D3F87C3AAE4800218DF817108DF8FE
:10F3C00017209847D4E9D72194F85A3388684FF426
:10F3D00000615161002B3FF467AEC3077FF564AE57
:10F3E00094F86534012B7FF45FAE9DF81730032B42
:10F3F0007FF45AAED4F85C349E491A6842F0010298
:10F400001A601A6842F003021A600B6943F006039F
:10F410000B6149E6D4F86023954853684FF0000823
:10F4200023F001034146536005F076F994F85163E7
:10F43000414656B1904BFF2203EB860653F8045F1A
:10F44000D86BAA609E428260F8D1D4F860338848B5
:10F450004FF0FF329A614FF00112DA610B2262F332
:10F46000070162F30708C3F8148019611A686FF383
:10F470000A121A6004F024FED4F85C237B4B7C480B
:10F48000D3F8783A4FF48051516198471DE6D4F88B
:10F490005C339A6922F010029A611A6AC2F34340FF
:10F4A000022802F00F0144D0062823D09A6942F0C6
:10F4B00010029A6106E694F85A333BB1D4F85C2402
:10F4C000136823F0030161F307031360D4F860238A
:10F4D00066495368D1F8801A654823F001035360E8
:10F4E0008847D4F85C334FF000425A61D6E5DDF826
:10F4F0000CA0C6E501EB8101D4F8205404EBC10156
:10F500002E68D1F8DC06C4F81C69C2F30A12024462
:10F510002868C4F82009C1F8DC26C7E700214FF4A9
:10F52000007084F852130921A4F8540361F38D2369
:10F5300037E747F6F0701042B8D001EB8100C2F314
:10F540000A1204EBC00002F1030C5FEAAC0CD0F825
:10F55000D056D4F820E44FEA810818BF002006D026
:10F560000130DEF8006045F8046B8445F8D1414471
:10F5700004EBC101D1F8D056D1F8DC0615440244A1
:10F58000C1F8D056C1F8DC2690E7B9F1000F7FF43E
:10F5900004AE94F86134042B7FF4FFAD344804F0DA
:10F5A0008FFD3346FAE5002F7FF4AAAE94F861246C
:10F5B000052A7FF4A5AE4846019304F081FD019B26
:10F5C0009FE62E48A5F57401A1F51051814203D89C
:10F5D0000D2161F38D23E4E629492A48294481421B
:10F5E00003D20C2161F38D23DBE62748A5F18C7152
:10F5F000A1F54341814203D80B2161F38D23D0E66D
:10F60000224923482944814203D20A2161F38D23F0
:10F61000C7E6204920482944814203D2092161F3E9
:10F620008D23BEE61D48A5F1B771A1F55851814261
:10F6300003D2082161F38D23B3E6194919482944FF
:10F64000814203D2072161F38D23AAE616491748A8
:10F650002944814234BF0621052161F38D23A0E6B0
:10F6600058CC0608401E1BFF3F420F0098010020A7
:10F670004853002000ED00E05C530020DFC810007C
:10F680002013FBFE20D61300FF69180000D3CEFE26
:10F6900040771B00C05BB3FEC091210040AC270047
:10F6A000C01D6AFE40E13300803C36FEE09C410014
:10F6B000704700BF704700BF704700BF704700BF72
:10F6C0002DE9F0414FF0FF35324A33482C460023F4
:10F6D00004E001330B2B02F1100215D0917A0429BA
:10F6E000F7D103F5B17100EB0111C979CF07F0D45F
:10F6F000661C116801D0A942EBD21C4601330B2BCA
:10F700000D4602F11002E9D1631C02D10120BDE8CF
:10F71000F081214D04F5B17705EB07139988F1B914
:10F72000DFF880802601AB19D8F84C291B491669EF
:10F730001B4A41F2186001EB442118580023B047DE
:10F74000D0B1022808D141F2CC6205EB0717AB58C3
:10F75000013B0121AB50B9710020BDE8F081DFF819
:10F76000448005EB0413D8F84C2941F21860D268A4
:10F77000185826019047D6E741F2CC6205EB0717EF
:10F78000AB580321B97141F2D061013B0124AB5068
:10F790006C54BCE7FCC60020E0B00020F8B00020AC
:10F7A000C1F70008F84F0020044B41F2E472995C65
:10F7B00009B90121995401225A707047E0B0002024
:10F7C00038B5174D174B41F2D0640020285504E09E
:10F7D00001300B2803F1100314D053F80E4C8C4267
:10F7E000F6D11C78032CF3D16AB10F4B03EB402305
:10F7F0009A4201D0FFF7D8FF00F5B17005EB001079
:10F800000123837138BD41F2CC6100F5B1736A58B0
:10F8100005EB03130420013298716A5038BD00BF14
:10F82000E0B0002006C70020F8B0002038B5134B28
:10F8300000209C7B14B11D688D4205D001300B283F
:10F8400003F11003F5D138BD72B10D4B03EB40232A
:10F850009A4210D0FFF7A8FF0A4B00F5B17003EBF6
:10F8600000100123837138BD064B00F5B17003EB26
:10F870000010827138BD022CECD1EDE7F8C60020F3
:10F88000F8B00020E0B000202DE9F84F12F0020E91
:10F890009B4606D028B9FFF787FF02252846BDE81A
:10F8A000F88F804C41F638056559002D5BD14FF03B
:10F8B000FF367D4FB146B046B24600253B689842C0
:10F8C00000F0B68097F80EC0BCF1000F5BD0BCF121
:10F8D000010F15D105F5B17C04EB0C1C9CF807C099
:10F8E0001CF0010F0CD11CF07E0F09D15FEADC1374
:10F8F00040F0A880D7F808C0D44501D2E246A94616
:10F9000001350B2D07F11007D8D1751C04D1B8F1C2
:10F91000FF3F00F09F80464641F2C86806F5B17788
:10F9200054F80850013544F8085004EB061C41F225
:10F930001C694FEA07184CF8095044F8085041F286
:10F94000186904EB07154FF000084CF80900C5F8DA
:10F95000048004EB0715AD79042D9CD8DFE805F091
:10F960001A330F334D0004F5C25741F63C063F6889
:10F97000A65907FB0565A84299D3FFF715FF002597
:10F980002846BDE8F88F2E4601350B2D07F11007EC
:10F9900094D1BAE712F0010C70D104EB0710D51026
:10F9A00090F80780BBF1030F65F3C71880F8078054
:10F9B00062D94FF6FF7083455B4628BF03469BB272
:10F9C00004EB07108380BEF1000F16D004EB061382
:10F9D00003F5B0531833987B04280ED041F2C86564
:10F9E0004FF0040C60590130605141F2CC65586011
:10F9F00083F80EC0635901336351500705D504EBFA
:10FA00000710C37943F00103C371D30608D504EB93
:10FA10000714E379C3F34502013262F34603E3714D
:10FA2000224B012503EB46260E602846BDE8F88FE1
:10FA300005F5B17704EB07164FEA071CB67986B9CE
:10FA40002E4669E7A84601350B2D07F110077FF414
:10FA500035AF5AE7B9F1FF3F18BF4E467FF45CAFB0
:10FA60008DE741F2C8682E4654F80850013544F835
:10FA7000085044F80C506CE76346A1E70C4B0B4967
:10FA8000D3F84C390B4AD3F8088001EB4621002308
:10FA9000C04700283FF473AF04EB07140223A3719F
:10FAA000FCE600BFE0B00020F8C60020F8B000205F
:10FAB000F84F00202DF80008F0B5124D2B7841F6D4
:10FAC0003002022B0BBF070AC0F3D417C4B200F0F8
:10FAD0007F04A85883B00E4600230122384401A9B0
:10FAE000FFF7D2FE01280AD12B78022B019B16BF0B
:10FAF00053F8243033F8143023F07043336003B0EC
:10FB0000F0BD00BFE0B0002010B5144602070B4660
:10FB100010D50B4941F2C472581C8B58834204D350
:10FB200005D100232360012010BDFFF73DFE2060BA
:10FB3000012010BD21461846BDE81040BCE700BFBB
:10FB4000E0B000202DE9F0414268C2F308030B4405
:10FB5000B3F5007F82B004460D4657D390F91A30B2
:10FB6000591C0AD0304A03F5B17302EB0313FF218D
:10FB7000DA796FF30002DA71817694F91B305A1C3E
:10FB80000FD0294A03F5B17302EB0313FF20DA7992
:10FB9000C2F34501013921EAE17161F34602DA71EC
:10FBA000E0762378022B37D01F4A02F5C2531B6838
:10FBB000B5EB432F4FEA432824DC41F6480367683E
:10FBC000D6583E407342AB421CDCAB19434511D3BF
:10FBD0002169207E01AAFFF797FF012812D16768EB
:10FBE000236963614744019B2361A5EB0801BF1BA7
:10FBF00067608D192046F8F733FC20B93D446560F5
:10FC0000012000E0002002B0BDE8F081154445600D
:10FC1000012002B0BDE8F0816168012029446160E3
:10FC200002B0BDE8F08100BFE0B0002070B515461D
:10FC300004460E46FFF786FF50B994F8280028B90D
:10FC4000022384F82830C4E90B5670BD022070BD31
:10FC50001DB12046A847012070BD012070BD00BF26
:10FC600010B4D0E9011390F91A208B4238BF0B462B
:10FC7000511C83600AD0144B02F5B17203EB0212DF
:10FC8000FF21D3796FF30003D371817690F91B3094
:10FC90005A1C0FD00C4A03F5B17302EB0313FF2477
:10FCA000DA79C2F34501013921EAE17161F34602D3
:10FCB000DA71C4760022436A5DF8044B4261426007
:10FCC00011460361B2E700BFE0B0002038B544221E
:10FCD000002111485CF06FFF104B41F602011A78C9
:10FCE0004FF6FF745C52022A41F2E87118BF0322FA
:10FCF00003F5C05041F64C055A5441F60C0441F648
:10FD0000010203215D5900F8181910211D51995461
:10FD1000FFF7A6FF012038BDC8C80020E0B00020D2
:10FD20002DE9F041B1F904300F2B82B00C46164694
:10FD3000054632D02846F8F7B7FB95F91B80B8F195
:10FD4000FF3F074633D02D4B41F2186203EB0811F9
:10FD50008A58904211D1183303EB4823A18801310E
:10FD600009B203EB4113A18028463360F8F79CFBEE
:10FD70002060012002B0BDE8F081FFF715FD2846A4
:10FD8000F8F76EFB28B100230120336002B0BDE814
:10FD9000F081002002B0BDE8F0814FF40071FFF760
:10FDA000D1FE0028F5D04FF6FF73A380C2E72846A6
:10FDB000F8F756FB0028E2D10FB9FFF7F5FC3846FB
:10FDC0000023112201A9FFF75FFD0128D7D1019B74
:10FDD0000B4A9A1A48BF02F2FF12B2F5B05F4FEA1F
:10FDE000622106D24FFA81F885F81B80002BB5D12D
:10FDF000C5E7FFF7D9FC019BF6E700BFE0B00020A4
:10FE0000F8B0002030B50446C06983B010B90120B5
:10FE100003B030BD0D460023032201A9FFF734FDD6
:10FE20000128F5D1B4F92030002B03DAFFF7BCFC30
:10FE30000220EDE7019A012D4FEA431102EB431333
:10FE400003D0022D12D1E5255554A268DA6122783B
:10FE5000032A04D100221A775A779A77DA77626AEE
:10FE60005A83C2F30F429A8203B030BDE268DA616E
:10FE7000EDE700BF10B50378023B012B0446037E7B
:10FE800002D913F0060F5AD198063AD494F91A30D1
:10FE9000591C0AD02D4A03F5B17302EB0313FF215D
:10FEA000DA796FF30002DA71A17694F91B305A1CEB
:10FEB0000FD0264A03F5B17302EB0313FF20DA7962
:10FEC000C2F34501013921EAE17161F34602DA71B9
:10FED000E076237E1B070BD51C4841F2C873C35C38
:10FEE000072B01D0FFF760FC41F2C8730022C25417
:10FEF000E26A0023237084F82830FAB1BDE810408C
:10FF0000104700231249E0691A018A58904206D02E
:10FF100001330B2BBAD01A018A589042F8D10B4A00
:10FF200003F5B17302EB0313DA79C2F3450101392A
:10FF300021EAE17161F34602DA71A7E710BD012100
:10FF4000FFF760FF0128F9D1237E9DE7E0B0002094
:10FF5000F8C6002030B1027822B190F828201AB1FA
:10FF6000002070470120704710B5D0E90142A2423D
:10FF7000C16238BF22460321826080F82810FFF753
:10FF800079FF012010BD00BF2DE9F04FDFF8689127
:10FF90008A4699F80010DAF800300229174683B033
:10FFA000834641F6300240F08B8059F80250DEB2B1
:10FFB000A6EB030805EB1325B8444FF48072904478
:10FFC000BB4208F1FF38B8FBF2F875D2A844032908
:10FFD00006EB0704A4EB03040CBF80224FF48072ED
:10FFE000944228BF1446A8EB050366B994422CBF7F
:10FFF0000A220B2201A92846FFF746FC012809D056
:020000040801F1
:1000000003B0BDE8F08F0B2201A92846FFF73CFCA6
:100010000128F5D199F80020DAF80010022A01F140
:10002000010321D0A64210D2019906F18042013A83
:10003000081F00EB840001EB820242F8043F824279
:1000400003F10103F9D1DAF80010A61B7318BBF114
:10005000010FCAF800301BD09F4205F101052BD9D2
:1000600099F800100026B2E7A642EED2DDF804C0EF
:1000700006F10042013AACF1020000EB44000CEB47
:10008000420222F8023F904203F10103F9D1DCE77A
:10009000BB42E1D199F80030022B21D004F1804419
:1000A000019B013C4FF0FF3243F82420DAF8003086
:1000B0009F4205F10105D3D8012003B0BDE8F08FC0
:1000C00059F8022003F07F060329C3F3D415A6EBE9
:1000D00003081544B84414BF4FF4807280226EE7C1
:1000E00004F10044019B013C4FF6FF72584623F88F
:1000F000142003B0BDE8F08FE0B000202DE9F041FE
:1001000090F838300446032B51D8DFE803F0023270
:100110003B462D4BC0681978E76A03F5C2520329A4
:1001200011680CBF80264FF4807601FB06F141F286
:10013000C47C00EB412041F2A87841F2AC7E53F838
:100140000C20E06053F80E0053F808502261A5EB34
:100150004125A0EB4121901943F8085043F80E10B7
:1001600043F80C00C4E90C205FBB6262012384F8F1
:10017000383016480021FFF745FE012811D102232F
:1001800084F83830626B04F130010120FFF7FCFE87
:10019000012806D1032384F8383000212046FFF7D8
:1001A00031FE431EDBB2012B02D9BDE8F0810220F3
:1001B00094F82830062B04BF002384F82830BDE8CB
:1001C000F081921B2263D1E7E0B0002080C80020BC
:1001D0002DE9F04FDFF8248198F80060012887B0FE
:1001E0008CBF00230123032E02930C460B68154697
:1001F00039D0022E62D14FF480724FEA1329DFB258
:1002000001920138012823D8012203929D421AD974
:10021000384E06F1880A06F11C0B32681AB1DBF879
:10022000001099424ED0DAF8000000234844092219
:1002300005A9FFF729FB01281FD002280FD020B104
:1002400023689D42E9D82560032007B0BDE8F08F00
:1002500087B1FFF7A9FA022007B0BDE8F08F0220AE
:1002600007B0BDE8F08F80220192C3F3D41903F0E8
:100270007F07C6E7019A0392C8E7DDE902C1059A44
:10028000DDF804E098F80030022B14D0032BE6D1FF
:1002900052F8273023F07043B3FA83F35B096345C8
:1002A0000F44236823D00B4477452360EAD309F138
:1002B00001090027C5E732F81730EDE74FF48072E7
:1002C0000192D2E70C490968013A02EB4122490246
:1002D000B2FBF1F203991344B3FBF1F201FB1232CA
:1002E0000AB10B449B1A9D42236096D8ABE7AB4200
:1002F000ABD3A8E788C8002020C90020E0B00020C8
:10030000F0B5104D2B7841F63002022B0BBF070AD7
:10031000C0F3D417C4B200F07F04A85883B00E46CF
:1003200000230322384401A9FFF7AEFA012807D1C0
:100330002B78022B019B0CBF23F8146043F8246038
:1003400003B0F0BDE0B000202DE9F04390F83C3060
:10035000002983B0044614BF02210021042B7BD85E
:10036000DFE803F0030C3C476900FFF74BFD012871
:1003700070D1626B002A75D184F83C00404EDFF8E2
:100380000881404D4FF6F7771DE01FFA80F9B94517
:1003900094BF4FF000094FF0010901A9B9F1000F16
:1003A00046D1FFF789FB0128494650D1206BFFF762
:1003B000A7FF01284BD1019B2A682363013B93428D
:1003C00028BF13462B603378206B032BDDD14045CB
:1003D00094BF4FF000094FF00109DEE7426B04F1D2
:1003E00030010020FFF7D0FD012833D1032384F82A
:1003F0003C30234BE16A41F2C47003F5C2521D58F0
:100400001268195041F2A87741F2AC76D8596D1AAA
:10041000995902FB05F200EB422501EB422203F55C
:10042000BD500021DD519A51FFF7ECFC012811D19C
:10043000042384F83C3094F82830042B04BF0023B4
:1004400084F82830A36B8BB120469847012003B075
:10045000BDE8F0830228FAD194F82830042B09D0A3
:100460000220F4E7022384F83C30B8E7012003B00F
:10047000BDE8F083002384F828300220E7E700BFBE
:10048000E0B0002024C90020F7FFFF0F38B590F836
:1004900034300446052B46D8DFE803F01F033F1035
:1004A0001963006B4FF0FF31FFF72AFF01283AD1A3
:1004B000E06A002839D1032384F834300021204633
:1004C000FFF7A0FC01282ED1042384F8343094F8DF
:1004D0002830082B2DD0012038BD41F63803224D9D
:1004E000EA5800F1300102320120FFF771FE0128C5
:1004F00024D00238C0B2012815D8052384F834303E
:1005000094F82830082B04BF002384F8283041F2E7
:10051000E5730122EA54022038BDC06A216BFFF75F
:10052000EFFE0128C7D0002038BD022384F8343004
:10053000F4E7002384F82830012038BD05F5C252C5
:10054000E3681168D4E90B2003EB412341F6440131
:100550006850C4E9033002B96062012384F8343082
:10056000A0E7014DCCE700BFE0B000202DE9F04F3F
:10057000436883B0C3F308081646002A00F0E18000
:10058000714B05468946A3F1180B4FF0000AC8F5D8
:10059000007495F91A70B44228BF3446791C284675
:1005A0002ED0F7F781FF0BEB071341F218629B582F
:1005B000984205D0FFF7F8F8504603B0BDE8F08F39
:1005C000614B03EB47202246494640445CF092FAD7
:1005D000002221462846FFF729FBA2440028EBD041
:1005E0002B7E1B0706D5594B2A691B689A4201D3FB
:1005F000FFF7DAF8361BA1444FF00008C7D1DBE75C
:10060000F7F72EFF002849D12846F7F74DFF696814
:10061000C1F308032BBB21F4FF7323F0010303F59F
:100620000072AB689A422CBF062207222B7E03F091
:100630000C030C2B1CD0002301A9FFF725F901287E
:10064000BAD10198404BC31A48BF03F2FF13B3F568
:10065000B05F4FEA63224FD257B2AF760028B2D1D3
:10066000AAE72B7E03F00C030C2B4FF00702E2D11C
:100670009BF800C0364BBCF1030F1B680CBF4FF05A
:10068000800C4FF4807C03FB0CF34FEA432C0CF1FD
:10069000FF3C0CEA0101A3EB5123CDE72B7E1A07A7
:1006A0002ED59BF800102A4B95F828201B680329AB
:1006B0000CBF80214FF4807103FB01F3062A4FEA3F
:1006C00043233FF479AF23490868834230D891F837
:1006D0003D30002B7FF470AF002A7FF46DAF6B6963
:1006E00085F83820062185F82810EB622846FFF7A8
:1006F00005FD012888D05FE7FFF756F80198ACE7C1
:10070000154B1A78002A7FF457AF95F82820002A55
:100710007FF452AF082185F8342085F82810D3F8EB
:100720005F206B692846C5E90B32FFF7AFFEE0E7B3
:1007300041F2E573012250460BF8032003B0BDE8F7
:10074000F08F924638E700BFF8B00020A4C8002020
:1007500020C9002088C80020C5C800202DE9F0432A
:1007600090F8384083B00546032C00F2A180DFE802
:1007700004F0021A8B0BFFF789FE012811D0022822
:100780000BD1032385F838302B6C002085F8280026
:10079000002B00F0898098470224204603B0BDE872
:1007A000F08385F838002B78022B79D0414A6F68A6
:1007B00041F64803D3581F40C7F34F272846F7F7A1
:1007C00073FEDFF8F48006463F1A0AE0D8F80030DE
:1007D0005A1E91454AD2FFF7B5F908B9FEF7E4FF72
:1007E0000136022201A900233046FFF74DF8BC195B
:1007F00001281FFA84F94FF400724FF000010446FB
:10080000CBD101985CF0D7F9EB694FF40071284621
:10081000002BDBD06B68002BD8D1019B4FF020322E
:100820004FF02E0C1A605A6083F800C0C3F80720FE
:100830004FF0100E6C6A1A625A6283F820C083F877
:1008400021C0C3F8272083F80BE0EA6B5C83C2F376
:100850000F4CC4F30F4483F82BE05A879C82A3F813
:1008600034C0D8F800305A1E9145B4D3C3EBC353FB
:10087000590201F500712846FFF764F908B9FEF73F
:1008800093FF022385F838302B6C002285F828204E
:1008900063B1284698470124204603B0BDE8F083A1
:1008A0006F68C7F34F2789E7022476E7012474E7CE
:1008B000002472E7E0B0002020C900202DE9F04FAD
:1008C00090F8303089B00446042B00F2A880DFE8AD
:1008D00013F0A900B20005008A00E800B64D41F609
:1008E0001003EB5C002B40F09A80B44F04F11C091C
:1008F000B84607F1380BBA4601AE32464946404683
:10090000FFF70EFA012840F018810198002800F046
:10091000FA800378E52B01D0002BEED1A84A821A89
:1009200048BF02F2FF12B2F5B05F4FEA622380F0D7
:100930003C811B01A34A13449A7B042A0CD041F248
:10094000C86104266A5801326A5041F2CC615A608B
:100950009E736B5801336B5041F60202AB565E1C1E
:1009600009D003F5B17305EB0313FF26D979AE5413
:100970006FF30001D97141F603016B565A1C0ED07A
:1009800003F5B17305EB0313FF26DA796E54C2F356
:100990004501013921EAE17161F34602DA71202251
:1009A00000215CF008F92346019A53F8311F58687A
:1009B0005060116019899B7A93721181019B627E4C
:1009C000DA7205A849F02CFCBDF81430002B40F079
:1009D0002F8144F28172019903200A82CB810A831C
:1009E000CB8284F83000237E980600F1A98020464F
:1009F000FFF736F92369002B00F0AE80237E03F069
:100A0000F70213F00403227640F0B480122A00F0BB
:100A1000BA80002384F828302046E36A984709B05A
:100A2000BDE8F08F6548FFF71BF94FF6FF72012311
:100A3000228484F83030614F04F11C0801AE04F1C7
:100A40003109324641463846FFF76AF901282FD06E
:100A50000228E4D1584D41F60202AB56591C09D088
:100A600003F5B17305EB0313FF20D979A8546FF395
:100A70000001D97141F603016B565F1C0ED003F5DE
:100A8000B17305EB0313FF20DA796854C2F3450113
:100A9000013921EAE17161F34602DA71042384F835
:100AA00030300020E36A2070984709B0BDE8F08F2D
:100AB000019D0B2249462846002D00F087802B78A7
:100AC000002B00F0838095F80BA01AF0080FB8D126
:100AD0005CF09DF80028B4D1637E8AEA0303DB064C
:100AE00040F1C780344D41F602016B565F1CC1D006
:100AF00003F5B17305EB0313FF26DA796E5460F347
:100B00000002DA71B6E73B782F49022B4FF0090259
:100B10005046C3D00B78002BC0D1C1E905330A7011
:100B20008BF800304A6B0B7351F8143CC1E9013269
:100B3000FFF714FE01283FF4E0AE0228AED06EE7C6
:100B4000E0690023112205A9FEF79EFE01283FF46B
:100B50004EAF09B0BDE8F08F237E19077FF559AF7E
:100B6000154A41F2C873D15C00297FF458AF0721C0
:100B7000D1544EE70023E26AA16884F82830204669
:100B8000FFF754F84BE7626AE06AA0630421C4E906
:100B90000233C4E90B2284F83C30636384F82810E4
:100BA00063622046FFF75CF839E7FEF7FDFD019828
:100BB0006FF00F03BEE600BFE0B00020C8C8002001
:100BC000F8B00020F8C60020F0C80020474D41F6DC
:100BD0000202AB565E1C09D003F5B17305EB03139B
:100BE000FF20D979A8546FF30001D97141F60301B0
:100BF0006B56581C0ED003F5B17305EB0313FF20A1
:100C0000DA796854C2F34501013921EAE17161F3EF
:100C10004602DA71237EDA067FF540AF3448FFF7EB
:100C20001FF84FF6FF720223228484F8303056E614
:100C3000304B05A9B3F9382902A849F043FB9DF8C8
:100C40000C309DF80D609DF80A509DF80B20BDF802
:100C500008109DF80E00DB0243EA461342EA4512F3
:100C6000A1F2BC7143EA500342EA41229BB292B224
:100C7000B1E6A98A6B8B204A43EA0143126863629A
:100C8000EB69A3605202B3FBF2F102FB113109B12F
:100C900013445B1A154DE36041F6020184F819A074
:100CA0006B565E1C09D003F5B17305EB0313FF20EF
:100CB000DA7968546FF30002DA7141F603016B567A
:100CC000581C0ED003F5B17305EB0313FF20DA793E
:100CD0006854C2F34501013921EAE17161F346022A
:100CE000DA71032384F830307DE600BFE0B00020E5
:100CF000C8C80020F060002020C900202DE9F04382
:100D000090F82830013B83B00446082B41D8DFE837
:100D100003F048054D525865406A4300384B466819
:100D2000056B41F6480103F5C2525F58136837401E
:100D3000EA19B2EB432F4FEA432816D258E0216953
:100D4000207EFEF7E1FE012823D1256B666823692A
:100D50006361A5EB08053D444644F61B019B6660B4
:100D6000A84525634F46236142D82046F7F778FB14
:100D700001AA81460028E2D06668A368E26A9E4222
:100D800038BF1E460023A66084F828300AB12046EA
:100D9000904703B0BDE8F083FFF7E0FC03B0BDE887
:100DA000F083FFF78BFD03B0BDE8F083FFF762F837
:100DB00003B0BDE8F0830021FFF7C6FA03B0BDE839
:100DC000F0830121FFF7C0FA0128E2D10023216C52
:100DD00084F828302046FFF7BDF8DAE7FFF78EF9F0
:100DE00003B0BDE8F083FFF751FB03B0BDE8F0832B
:100DF0002046F7F735FB0028BFD12E446660BCE7DC
:100E0000E0B000202DE9F04782B0054602AF184659
:100E10001C460E46904657F0A3FF083020F007000E
:100E2000ADEB000D0DF1080A013CD14614F8013F6D
:100E30005BB989F800304246CDF800A0314628461B
:100E40003DF0BAFFBD46BDE8F087184648F0D0FF38
:100E5000C3B2A3F120023F2A88BF202309F8013B37
:100E6000E4E700BF2DE9F04704460D469046002117
:100E700044221E46089F5BF09EFE01234FF6FF7240
:100E80002676628384F828302B782E2B4CD02E4681
:100E900004F1310A307804F1390968B12E280BD0F9
:100EA00048F0A6FFC0B20AF8010BCA4506F10106D8
:100EB00007D030780028F1D120200AF8010BCA456C
:100EC000F7D130782E2808BF707804F1380908BFB0
:100ED000013604F13B0A58B148F08AFFC0B209F864
:100EE000010FD14506F1010607D030780028F3D173
:100EF000202009F8010FD145F7D118F0100F14BFC9
:100F00000323012384F819802370E7622B782E2BAA
:100F100026D16B7823BB0323204684F83030FFF7BB
:100F2000CDFC2046BDE8F0876B78002BAFD1114B8C
:100F300041F2F47241F60C0041F2F0719A581858DF
:100F40005958E26041F601026062A1609A5C6276E3
:100F500041F2E8729B5C2370E7622B782E2BD8D08D
:100F60000023204684F83030FFF7A8FC2046BDE877
:100F7000F08700BFE0B0002010B5114C94F85A3350
:100F800023B9104B4FF480225A6110BD0E4A1368EA
:100F900023F00603136057F0AFFE94F85A33002B8A
:100FA000EFD0D4F860339B68DB07EAD5D4F85C2433
:100FB000136823F0030161F307031360E1E700BF47
:100FC000F84F0020003C014010ED00E008B5012181
:100FD000032003F0ADFC72B64AF0A8F82DE9F04FFB
:100FE0008DB0CF4CDFF84C93CE4D00904FF0000801
:100FF00054F80B0C002800F0FE8039F0C9FB0646BF
:10100000002800F0DB81D9F8083944F8073CE026D5
:101010000023C54F04F8033CA4F10B0B06FB08F6B4
:1010200054F80B0C39F0B4FB002800F0E48054F8BD
:101030000B0C39F0A5FB14F8023C5A1E82460B2A11
:101040000DD8DFE812F01F003A004600530083007D
:101050009B00E30017013701420179019101242827
:101060000CD0009A3AB995F87E24824240F08281F1
:10107000012204F8032C0D2BD2D186E0012304F8C1
:10108000023CCDE700234D28C4F8C53084F8CD30AC
:1010900084F8CE3004D0582808D004F8023CBFE7CA
:1010A000022204F8022C84F8C430B9E7032304F8C0
:1010B000023C022384F8C430B2E704233C2804F83D
:1010C000023C0BD0BAF13E0F0CD0002304F8023CD6
:1010D000A6E70A233C2804F8023CF3D1002304F8D5
:1010E000013C9DE7012304F8013C99E7D4F8C500D1
:1010F000BB190344421CC4F8C52083F8AFA994F877
:10110000CD00022A8AEA000184F8CD1088D1237824
:10111000C02BDAD86278FF2A08D1052BD5D9012354
:1011200084F8C430072304F8023C79E7A4F8C1200E
:1011300000229342C4F8C93014BF0523062384F863
:10114000C320C4F8C52004F8023C69E7D4F8C50000
:10115000BB190344421CC4F8C52083F8AFA994F816
:10116000CD00D4F8C9308AEA00019A4284F8CD1043
:101170007FF456AF062304F8023C51E794F8CD30D3
:101180008342A2D10D2304F8023C14F8017C002F05
:1011900040F0F680654B08940FCB04AE86E80F0054
:1011A000D4F8C930D4F8D100ADF82C702344099399
:1011B000B4F8C130ADF8283094F8C3308DF82A3037
:1011C00001238DF82E30324603AB08A9039730F087
:1011D00017F948B1049B059394F8C420544B049329
:1011E000314658462DF000FD039E002304F8023CD2
:1011F000002E40F0DB8008F10108B8F1030F04F184
:10120000E0047FF4F5AE0DB0BDE8F08FD4F8C50072
:10121000BA190244431CC4F8C53082F8AFA994F847
:10122000CD2094F8CE0001938AEA020284F8CD2002
:101230005146D52249F0B6F8019B84F8CE00072B21
:101240007FF4EEAEB4F80530C02B3FF63EAFB4F8F5
:101250000320A4F8C120A27884F8C320002293427E
:10126000C4F8C93014BF08230923C4F8C52004F802
:10127000023CD5E6D522014694F8CE0049F092F81A
:1012800094F8CD3084F8CE008AEA0303D4F8C50080
:1012900084F8CD30BB190344421CC4F8C52083F840
:1012A000AFA9D4F8C9309A427FF4BAAE092304F842
:1012B000023CB5E694F8CD30434084F8CD3094F844
:1012C000CE3083427FF401AF54E7D4F8C500BA1999
:1012D0000244431CC4F8C53082F8AFA994F8CE008C
:1012E0000193D522514649F05DF8019B84F8CE0068
:1012F000052B7FF495AEB4F80120B4F80330A4F8C0
:10130000C120227884F8C32000229342C4F8C93057
:1013100014BF0B230C23C4F8C52004F8023C7FE65D
:10132000A7590020F0600020F84F002014CE0608D6
:101330001C8D0120101D0020D522014694F8CE00FE
:1013400049F030F884F8CE00D4F8C500BB19034446
:10135000421CC4F8C52083F8AFA9D4F8C9309A421A
:101360007FF45EAE0C2398E694F8CE3083427FF48F
:10137000ACAE07E7232804BF022204F8032C7AE668
:10138000012F4FF0000602D004F8026C33E7D4F8C6
:10139000C93008942344099308A8B4F8C130CDE9B2
:1013A0000A66ADF828302CF04BFEEDE754F80B0C34
:1013B0002DF058FE54F80B0CB0471CE714F8033C12
:1013C000002B3FF418AFD9F8082954F8071C521A1B
:1013D000632A7FF610AF012B31D0022B7FF40BAFC5
:1013E00054F80B3CC5F83C39C5F84039C5F84839C4
:1013F000402385F84C39134BC5F89833C5F890391C
:1014000095F89B3985F84D09003B4FF0010218BF54
:1014100001230D4885F83A290C4AC5F8442985F876
:1014200094393EF045FB4FF400502FF0A7FE0848DA
:101430003EF034FB85F8A96985F8AA69DBE6FFF779
:10144000C5FD00BF346A0020FA5D07089149040811
:10145000305E070800000000034B93F824000038BA
:1014600018BF0120704700BF481D002020230148FD
:101470000B8070472C0C0020642301480B807047C0
:101480004C0C0020432301480B807047B00C002017
:1014900010B5074CD4F8C800FF2807D0054951F80B
:1014A000042BF6F715FFFF23C4F8C830002010BD49
:1014B0002C0C002038C90020EAE700BF08B5D0F89E
:1014C000E4355B6A9847002008BD00BF08B5D0F836
:1014D000E4351B6A9847002008BD00BFD0F8E4350A
:1014E00010B504461B689847D4F8E8359B689847C0
:1014F000002010BD08B5D0F8E435DB6903B198478A
:10150000002008BD08B5042290F81211D0F8E83583
:1015100080F8131180F81221DB689847002008BD7D
:1015200010B5D0F8E83504461B699847032384F8C2
:101530001231002010BD00BF0B0630B41CD401EBEB
:10154000810200EBC202002300EB810582F87413D4
:1015500082F8753301241A4604FA01F16D6D61F3C6
:101560001F4201696FF3CF332B60CB6923EA02037B
:10157000002030BCCB61704701F07F0101EB81049A
:1015800000EBC404012200EB8105002384F81C1148
:1015900084F81D2102FA01F11A46AD6961F30F02C8
:1015A000DFE700BF10B581210446FFF7C5FF2046E5
:1015B0000121FFF7C1FF024B0020187010BD00BFD2
:1015C000086A002010B581210446FFF7B5FF2046C8
:1015D0000121FFF7B1FF82212046FFF7ADFFF6F7AB
:1015E000BDFE002010BD00BF38B50D460446832166
:1015F000FFF7A2FF29462046FFF7E4FF002038BD91
:10160000F0B416460A063AD401EB810500EBC50595
:101610002824002204FB0104022B85F87413C5F86A
:101620007C6385F8773385F8752304F55D7448D0BD
:10163000154600EB8107012202FA01F17F6D61F38B
:101640001F45D7F800C01CF4004F11D1E488204991
:1016500046F0805242F4004242EA834204F00F0412
:101660001C4B42EA845211400CEA030319433960CF
:101670000269D3692B430020F0BCD361704701F0AD
:101680007F0101EB810500EBC5052824012204FB45
:101690000104022B85F81C11C5F8246185F81F315F
:1016A000A5F8221185F81D2104F58E740CD00025B3
:1016B00000EB8107012202FA01F1BF6961F30F0516
:1016C000BFE722711546B4E700252571F0E700BF9A
:1016D000FF87CC13007833EC002310B5194604467D
:1016E0004022FFF78DFF8021204600234022FFF794
:1016F00087FFD4F8E835A078012284F812215B68CE
:101700009847002010BD00BF70B44B78012B26D045
:101710000B784A6900EB83035C6D25682369D2B1BD
:101720008A684A6102F07F0223F4002323F07F03DA
:1017300042F4002213432361C378012B04BF0B69D9
:101740006361C5F3076363F07B0363F31F65256083
:10175000002070BC70478A6802F07F02E4E782696B
:101760004C691568136944B38E68B4428CBF06F0A7
:101770007F0404F07F0423F4002323F07F0344F468
:10178000002443EA040388BF4E611361C378012B30
:101790001DD0C5F3076464F07B0464F31F65156016
:1017A000002BD5D14B69002BD2D002690878516B40
:1017B000012383400B435363CAE723F4002323F040
:1017C0007F0343F400231361C378012BE1D10B782D
:1017D0000C6900EB8300C5F30763816963F07B0349
:1017E00063F31F654C610020156070BC704700BF3B
:1017F0002DE9F0434B78012B30D00B784C6900EB8E
:1018000083035E6D356837691CB38B681C44013CEB
:10181000B4FBF3F4C4F3090203FB02F3C3F31203B2
:101820004B61144643EAC44363F31C073761C37832
:10183000012B04BF0B697361CB78012B44D0C5F336
:10184000076363F07B0363F31F6535600020BDE829
:10185000F0838A680124C2F31203E3E791F8008061
:101860004E6900EB880EDEF818C0DCF80050DCF89A
:10187000107076B3D1F80890384A06EB0904013CA1
:10188000B4FBF9F402EAC444C6F312022243CC7852
:1018900007F060473A43012C174649D0CCF8102096
:1018A000C278012A55D00269516B03FA08F30B4341
:1018B0005363C5F3076363F07B0363F31F65CCF8E1
:1018C00000500020BDE8F0834B7973B345F000551C
:1018D000B5E707F0604747F40027CC78CCF81070E4
:1018E000C378012B2FD0012CE3D102699268D20575
:1018F00054BF45F0005545F08055C5F3076262F0CE
:101900007B0262F31F65CCF80050002B9ED1B0B271
:1019100003308010DEF8D04098D0CA6852F8041B1B
:10192000216001339842F9D190E745F0805586E770
:1019300064F35E77CCF81070C378012BD5D10A69B7
:10194000CCF81420D1E70A69CCF81420012CB0D1CE
:10195000CBE70B69CCF81430ABE700BF0000F81FF1
:101960000E4BDA68D20310D4DA68D1060FD4DA68E5
:10197000D20510D4DA6812F0E00F0AD1DB6813F058
:10198000020F14BF0820092070470120704706206D
:101990007047072070470220704700BF003C02409C
:1019A00000207047104AD068A8B113699BB18842E3
:1019B0000FD88B4234BF00230123DBB243B19369BC
:1019C0005161994204D0094B9161142083F8CC00F5
:1019D00070470023F1E7A1F59C53083BB3F57A7FEC
:1019E0002CBF00230123E9E738C900202C0C00207C
:1019F000054B5A7F19778A4204D0044A597714203C
:101A000082F8CC00704700BF38C900202C0C0020A1
:101A1000704728B1034B987F012894BF0020012014
:101A2000704700BF38C9002008B5FFF7F2FF50B17A
:101A3000054AD37F127F5B0003F00203002A18BF20
:101A400043F001030B6008BD38C9002008B5FFF75B
:101A5000E0FF10B1014B1B6A0B8008BD38C90020A4
:101A600070B5FFF7D6FF50B10A4A958C35B1966A2A
:101A70000023B3421C4603DB002000E00D7070BD64
:101A800002EB44040133A48DAC42DBB2F1D10B7004
:101A9000F5E700BF38C9002008B5FFF7BAFF10B15D
:101AA00000230B70137008BD0420704728B1034B4E
:101AB00093F9CE00003818BF012070472C0C00208D
:101AC00008B5FFF7F3FF50B1054B93F9CE20012A7B
:101AD000C3BF93F8D130C3F340030B60002008BDAF
:101AE0002C0C002008B5FFF7E1FF18B1024B93F86A
:101AF000D0300B7008BD00BF2C0C002070B5FFF774
:101B0000D5FF38B10E4C94F8D130DB0703D5002354
:101B10000B70137070BD0B4D94F9CF3095F83C608D
:101B200093FBF6F301330B7094F9CF4095F83C101A
:101B300094FBF1F301FB134301331370EAE700BF99
:101B40002C0C002038C900200320704770B50A4AC9
:101B500092F8403006255E1CB6FBF5F405FB1464D4
:101B600092F84150AC4205D002EBC303C3E9110126
:101B700082F8404070BD00BF38C90020002230B557
:101B800004461046914200DC30BDA35C0825584055
:101B900010F0800F4FEA400318BF83F0D503013DDA
:101BA000D8B2F5D10132EDE710B5D9B10E4B586F6F
:101BB000814217DCB2B1DB6B9A4213DC0B4C013A69
:101BC000013903FB012184F8DC1004F1D800052160
:101BD000FFF7D4FF062184F8DD0004F1D800BDE84A
:101BE0001040B3E710BD00BF38C900202C0C002006
:101BF0000023038083708380C3800372704700BF1B
:101C0000074A084992F8783009780133DBB29942E3
:101C100082F8783004BF002382F87830704700BF24
:101C200038C9002054490020F8B5794CE36F83B1DE
:101C3000784B1B6893F82E305BB1774B94F880207B
:101C4000A3FB0013012A4FEA931330D0022A08D0D5
:101C500002B1F8BD714B9842FBD9012384F8803062
:101C6000F8BDD4F8842064329A423ED894F8783093
:101C700004EB031393F8F824FF2A06D068490132D5
:101C8000012083F8F82481F8DE00FFF7B9FF654BE7
:101C90001B780122092B84F88020DAD1B4F87A3538
:101CA000614A01339BB2A4F87A355380F8BD94F8A9
:101CB00078105C48C4F884308C2303FB014300781F
:101CC00083F89A20002384F8963004F18C050A22C8
:101CD00002230928C4F8885084F8972084F88030BB
:101CE000B7D1514B01311980F8BD94F8962094F882
:101CF00097309A42ADD104F18B0004F19405002392
:101D000010F8012F082153405A0013F0800F08BF2C
:101D10005B0082F0070214BFD3B2DBB20139F3D10A
:101D20008542EDD194F895209A4239D194F87860A3
:101D300094F8935094F89430B4F88F00B4F891204C
:101D400094F88DC004EB061743EA052394F88E50EF
:101D500087F8F81440BA52BA81B292B245EA0C2020
:101D60002F4DC7F8FC141BB294F98C10C7F800254E
:101D7000032E4FF00102A7F8FA04A7F8043587F8FC
:101D8000F91485F8DE2008D8264A12780C2A29D0C2
:101D90000D2A02D1244B23F81610FFF731FF5CE720
:101DA00094F8783004EB031393F8F824FF2A06D054
:101DB0001B490132012083F8F82481F8DE00FFF787
:101DC0001FFF184B1B780122092B84F880207FF419
:101DD00040AFB4F87835144A01339BB2A4F8783593
:101DE0009380F8BD1149124A91F822100E4803EB76
:101DF000830303EB830349089B0093FBF1F382FB0E
:101E00000312DB17C3EBA20320F81630C5E700BFAF
:101E100038C90020F45F0020D34D62103F4B4C00C6
:101E20002C0C0020F9420020FC420020D42E00207F
:101E3000676666660B4B93F8961093F8972091426D
:101E40000ED010B493F89620D3F88840511CD2B22B
:101E5000C0B2C9B283F89610A0545DF8044B704725
:101E6000704700BF38C90020FD2870B522D0F02887
:101E700004D0EF2822D00224204670BD114D03204B
:101E8000052641282E444FF0000405F1010580F09D
:101E900080030DD0042B0BD9FFF7E6FF2044B54299
:101EA000C4B2E9D015F8010B412880F08003F1D1CC
:101EB0000420F3E7044D0B200426E2E7034D0C2039
:101EC0000626DEE73CCE060838CE060844CE0608D5
:101ED0000E4BD3F88025B3F97C05530707D400EBEC
:101EE0008000400080B200F5C87080B27047084B97
:101EF000084A1B6C323382FB0312D817C0EBA200D6
:101F000080B200F5C87080B2704700BF38C90020A9
:101F1000B43C0020676666660C4AD2F8983530B447
:101F20001C68D2F890555D6019810025611C19600C
:101F30009D812070D2F89835D2F890151A685A60B1
:101F40004FF6F67230BC19609A81704738C900208C
:101F5000114B30B4D3F83C27C3F8402703F29C5010
:101F600003F22C6103F21C6503F22C740132C3F8F6
:101F70009455C3F89845C3F83C2730BCC3F88C058A
:101F8000C3F81C06C3F82006C3F89015C3F82C1735
:101F9000C3F83017704700BF38C9002000B583B0C0
:101FA0000268084B8188CDF801203222D3F84437EB
:101FB000ADF805108DF800206846984703B05DF82D
:101FC00004FB00BF38C900205E2810B511D05D2881
:101FD00005D00D4BBDE81040D3F8483718470A4CE0
:101FE000D4F848379847D4F848373D20BDE810402A
:101FF0001847054C5D20D4F848379847D4F848373F
:102000003E20BDE81040184738C9002070B5094E81
:102010000546D6F848375E200C469847D6F848372C
:1020200028469847E0B2FFF7CFFFC4F30720BDE88A
:102030007040C9E738C9002003682DE9F041002B42
:102040003D4D3E4F3E4EB8BF5B42A5FB0321890D7F
:1020500007FB0137C7EB0717BF0096F8523785FB20
:102060000725FA170446C2EBA555002B57D101EB03
:10207000810101EB810105EB810109B2DFF8BC8030
:102080001320FFF7C3FF2F4908FB057581FB0531BE
:10209000ED17C5EBA11109B21B20FFF7B7FF2368AD
:1020A000254D002BB4BF53214E212320FFF7AEFF57
:1020B000636896F8522783EAE376A6EBE376A5FBFE
:1020C0000631890D08FB0168C8EB08184FEA88083B
:1020D00085FB08354FEAE873C3EBA5552ABB01EB36
:1020E000810101EB810105EB810109B21220FFF7AB
:1020F0008DFF124B134903FB058581FB0531ED175D
:10210000C5EBA11109B21A20FFF780FF6368002B0D
:10211000BDE8F041B4BF57214521222076E7C1EB4D
:10212000011105EB810109B2A8E7C1EB011105EB33
:10213000810109B2DAE700BF6BCA5F6B806967FF94
:1021400038C90020D34D621030B400230225152475
:102150004FF4167140F2D93205808471018130BC90
:102160004281438083808381704707B50DF1060269
:102170000FF02CFE68B1084BBDF80620B3F87017BD
:102180009A84914205D00549A3F87027142081F85C
:10219000CC0003B05DF804FB38C900202C0C0020F3
:1021A00013B50446FFF782FC08B300230DF10602C5
:1021B0002046ADF806300FF009FEC0B10D4C9DF879
:1021C000062094F9CE1084F8E320032908BF62F0BA
:1021D0007F024FF00501084808BF84F8E320FFF7AD
:1021E000CDFC062184F8E4000348FFF7AFFC02B001
:1021F00010BD00BF2C0C00200B0D002008B5044BB7
:10220000D3F8740738F0C4FAB0FA80F0400908BD7A
:1022100038C900202DE9F84F1B4C05461E2094F8C4
:1022200078A794F879B794F87A67B4F87C97B4F8FB
:102230007E8794F8807723F0C1FE30B1B8F1000FAB
:1022400003D0C14601264FF0000A94F88237DA071E
:102250000AD494F887273AB9012F12D0022F03D15C
:1022600013F0020F08BF012685F800A085F801B021
:10227000AE70A5F80490A5F806802F722846BDE838
:10228000F88F3E46F0E700BF38C90020144B30B449
:10229000D3F8AC4714B300220F2583F8B217090A0C
:1022A00083F8B10783F8B317C3F8B427C3F8B82786
:1022B000C3F8BC2783F8B05703F5F660012110F886
:1022C000015F01312A440E29D2B2F8D183F8BE272A
:1022D0002046044930BC102238F02ABA30BC70477E
:1022E00038C90020E8D00020034B002183F8C01734
:1022F000C3F8C417CAE700BF38C9002013B50446A5
:102300002620019123F05AFE019920B9204602B0FF
:10231000BDE81040BAE702B010BD2DE9F743B74C55
:10232000D4F8AC370D464BB14FF0020800264FF001
:102330000109D4F8AC0738F02BFA58B90027A37F6D
:10234000042B00F25781DFE813F08F00E400F70060
:102350003D014601D4F8AC0738F012FAD4F8C4377E
:102360005A1C2344C4F8C42783F8C80794F8C0371C
:10237000012B0AD0022B11D0002B70D10F280CBFDB
:1023800084F8C097C4F8C437D3E7A0F17203012BD7
:1023900001D9762863D184F8C087CAE7102AC8D14A
:1023A00097490023012211F8010F013203440E2A3C
:1023B000DBB2F8D194F8D62784F8C0679A42C4F803
:1023C000C467B6D194F8D737002BB2D194F8C97747
:1023D000732F37D0762F0DD0722FAAD194F8CB2738
:1023E00094F8CA3753EA0223A3D0E360B4F8CC3799
:1023F0002361A4E794F8CB2794F8CA3753EA022361
:1024000097D094F8CD1794F8CC2794F8D10723628D
:1024100042EA012294F8CE17E17794F8CF1784F8B6
:10242000DA1794F8D017A4F8D82741EA0021A4F8C5
:10243000DC17616901B96361A38C002B7FF47FAF66
:10244000A2847CE794F8CF2794F8CE3743EA02239E
:102450001AB2002B3FF46DAFA4F8DE276FE784F8C3
:10246000C067C4F8C46764E7722F44D10123A3771F
:102470000022644B1B78402B2FD1634E94F8DAC7AF
:10248000A08CA37FB4F8D8E7338005024FEA0C3361
:10249000217F778005F4706503F440532B434FEAA6
:1024A0000E1543EA8133EDB22B43276A65691BB2EF
:1024B000BD4214BF0825002513432B43704514BFAC
:1024C000042000201843514B614514BF0221002114
:1024D00093F8CC30F3800143B180636F1BB1A36AE2
:1024E000002B40F09D804A494A481F2203B0BDE8B6
:1024F000F0435AF09EBBD4F8E037474AEB1A9342B8
:1025000001DC0022B5E77220FFF7EEFEC4F8E057C9
:10251000F7E7762F03D10223A3770022A9E7D4F8A7
:10252000E0373D4AEB1A9342EBDD7620FFF7DCFE05
:10253000C4F8E05700229CE7344ED4F8E03796F810
:10254000CC20EB1A82B3344A934230DDE27FD207CB
:102550001BD46169226A91420ED089B24620FFF7EE
:10256000CDFE96F8CC30C4F8E057013B86F8CC306D
:102570000423A37701227CE7A18CB4F8D8278A42F0
:1025800003D05020FFF7BAFEEBE7217F94F8DA275B
:102590008A4206D0B1FA81F149094920FFF7AEFE1F
:1025A000DFE7142286F8CC201C4A9342BDDC762F4C
:1025B000A7D17320FFF798FE0323A377C4F8E05751
:1025C000002256E7732F9CD0D4F8E017124B691AFB
:1025D0009942A0DC95E7D4F8E0370F4AEB1A934212
:1025E0008FDD7620FFF780FE0223A377C4F8E05743
:1025F00000223EE70023A3771A463AE738C90020B5
:1026000000D10020F9420020FC4200202C0C0020C8
:10261000355E0708110D00203F0D03003F420F00FB
:10262000334DD4F8E4672A2385F8E5300DF1020232
:1026300020230DF10101304685F8E6300FF05DFCF6
:1026400030B19DF801109DF8027051EA070339D1AD
:10265000552385F8E730462385F8E830202301A983
:10266000304685F8E9300FF042FC0346214813B1AB
:10267000BDF804209ABB204948F0F2FBB4F8DC779F
:102680001E4D87B30DF1030130460FF033FC50B3FC
:102690009DF803100DF1060230460FF097FB10B3C2
:1026A000BDF8062016493B46BA420CBF20222A221A
:1026B000284648F0D5FBB4F8DE37A4F8E83703B075
:1026C000BDE8F08330460FF0FDFB394685F8E700A2
:1026D00030460FF0E3FB037885F8E830BEE70949A0
:1026E00048F0BEFBCAE70849284648F0B9FBE2E7D4
:1026F0002C0C0020160D0020575E07081A0D002034
:102700004F5E0708DB970708565E070838B50B6869
:102710000E4D5A1C0A6005221A700B6895F8CE20DF
:102720000C46591C21601A70236895F8D120591C59
:1027300021601A70B5F8D410204647F055F9236887
:1027400095F8D620591C21601A7038BD2C0C002039
:102750002DE9F84F2DED028BFFF7A8F9002844D0A2
:10276000254B93F9CE0001283FDD93F80441DFF8B3
:1027700090809FED228A0FF2780BDBE900AB1546C3
:102780008E1E02EB44094D4504D1BDEC028B204660
:10279000BDE8F88F38F8027B26F8027F07EE907AC2
:1027A000F8EEE77A67EE887A17EE900A56F044FC66
:1027B00052465B4656F098FC41EC100B59F05CFF1A
:1027C00051EC100B56F052FF0E2F80B20AD919307F
:1027D0003223B0FBF3F080B200EB800000EB80000E
:1027E000400080B225F8020BCDE70024CDE700BF02
:1027F0001655B5BBB16B02402C0C0020CDCCCC3DA6
:1028000022D1002038B50D46FFF750F9044638B103
:102810000C4890F8D130DB0704D5B0F8D2002880FE
:10282000204638BD084A90F9CF3092F83C2093FBFF
:10283000F2F102FB11320132013100F584700FF028
:10284000D9FAECE72C0C002038C9002038B5134C1D
:1028500094F8413094F840209A4219D004EBC30315
:102860000F49D3E911200023984212DC93780D4AD6
:10287000C4F8FC075B081370FCF776F894F8413055
:1028800006210133B3FBF1F201FB123384F841302E
:1028900038BDD55C01F8015B0133E5E738C900209C
:1028A0007C690020AA6900202DE9F04FA84B1B7815
:1028B0008BB08146002B40F0B380A64DD5F8E4677D
:1028C000002E00F0AD80A44AD2F80C4104F0F021B3
:1028D000B1F1E02F6DD1C2F80C31D5F80028944247
:1028E00067D004930593ADF81830B5F87C3795F8A8
:1028F00078E7ADF8143095F879C795F8803795F8F2
:102900007AA78DF818300DF110088DF810E08DF8C9
:1029100011C08DF812A098E8070007AB03C38F4FD2
:102920001A80C4F342533B44C4F30342997CC5F874
:1029300000488E4502F1010201D1944508D030468D
:102940008DF81C108DF81D200FF054FAADF8200002
:1029500030460FF0A0FC032804F0070B34D0042805
:1029600035D000239A4501A9304618BF8DF81E3096
:102970000FF0BAFA48B1019BC4F3001103F0010350
:102980008B4202D030460FF05DFB0A2207A9404679
:102990005AF0E9F868B19DF81E30BDF81C2085F8A2
:1029A0007A37BDF82030A5F87827A5F87C3747F0AE
:1029B00053FE95F804A804AF95F80438032B79D892
:1029C000DFE803F0083174A15F44FB7DCAE75F4490
:1029D000FB7FC7E7394630460FF08CFA044658B102
:1029E00007A8FFF717FC9DF81E109DF810308B42CA
:1029F00060D030460FF0B2FB95F80438013303F095
:102A0000030385F804380CB99A45D5D195F8823777
:102A1000DB0700D524B1336849461B683046984728
:102A20000BB0BDE8F08F01A8FFF7F4FB95F88287A3
:102A30009DF8044008F00108ECB1B8F1000F39D15D
:102A40003A460DF1030130460FF057FA044688B3B9
:102A500007A8FFF7DFFB9DF81C109DF803309DF8D9
:102A60001D208B4203D19DF81030934222D0304676
:102A70000FF07EFBC0E7B8F1000FBDD139463046FC
:102A80000FF035FA0446A8B107A8FFF7C3FBBDF85D
:102A90002010BDF810308B420CD085F8058885F8E1
:102AA0000688336830469B699847A5E795F88237D2
:102AB000D80701D500249FE707A930460FF014FA84
:102AC00004460028F6D01E2023F078FA95F807383F
:102AD00083428046EED085F8070860B1B5F87E37AE
:102AE000002BE7D1079BD907E4D4012130460FF032
:102AF000A9FA444680E7079BDA07DBD50146304652
:102B00000FF0A0FA78E73846FFF784FB97E8070054
:102B100007AB03C31A809DF810309BB10DF11D0265
:102B200007A930460FF0E9F90DF11E0130460FF00C
:102B3000E1F90A2207A938465AF015F8041E18BF11
:102B4000012459E708A930460FF0D1F9ECE700BF9E
:102B50002A6A002038C900202C0C002038CE060834
:102B6000024B0146D3F8080837F016BE38C90020DA
:102B70002DE9F041FD2984B0044600F0DD80F02904
:102B800000F0BC80EF2900F02F814AB1034686187F
:102B900003AD002003F8010B9E4205F8010BF9D1AB
:102BA000994B0B2003F1090501E013F8010F814255
:102BB00000F0C780AB42F8D14B1E832B00F292800D
:102BC000DFE813F03001370184004101AE01B401A8
:102BD000480153015F0190009000650165016501A6
:102BE0007B017B017B015F019000900086018E01DB
:102BF0009000900090009000900090009000900055
:102C00009000900090009000900090009000900044
:102C10009000900090009000900090009000900034
:102C20009000900090009000900090009000900024
:102C30009000900090009000900090009000900014
:102C400090009000A40190009000900090009000EF
:102C500090009000900090009000900090009000F4
:102C600090009000900090009000900090009000E4
:102C700090009000900090009000900090009000D4
:102C800090009000900090009000900090009000C4
:102C900090009000900090009000900090009000B4
:102CA00090009000900090009000900090009000A4
:102CB0009000900090009000900090009000900094
:102CC00090009000900090001D011D014F4B93F863
:102CD0005717002900F0618101922BF051FC019AF5
:102CE000ADF80C003AB1224403AB13F8011B04F811
:102CF000011BA242F9D104B0BDE8F081444F032189
:102D00004FF00508B844002501370CE0FFF7ACF898
:102D1000064660193246FFF72BFF70194745C5B2CA
:102D2000E9D017F8011B412981F08003084601D042
:102D3000042BEBD80426ECE7364F0B214FF00408A8
:102D4000E0E7324BD3F8800580060CD4002AD2D0BD
:102D5000224403AB13F8011B04F8011B9442F9D180
:102D600004B0BDE8F08193F80C08870741D52A4DDF
:102D7000287D052834BF02260326142916D97C395C
:102D8000C8B20628E2D80629E0D801A050F821F000
:102D9000732F0108732F01085D2F01084D2D0108C5
:102DA000832F01087D2F0108892F01080929CDD91A
:102DB0000A390A29CAD801A757F821F0432F010878
:102DC0008F2F01084D2D01084D2D01084D2D0108B3
:102DD0004D2D01084D2D01084D2D01084D2D0108E7
:102DE000552F0108732F01080C4F0C214FF00608D6
:102DF00088E7094B0B29187DA8D10126C8E0084BAC
:102E0000DB6B03936EE700BF60CE060838C9002075
:102E10003CCE060838CE06080C65002044CE0608D5
:102E2000B43C00200192FFF753F8019AADF80C0072
:102E300058E76A4BD3ED037AFDEEE77A17EE903A46
:102E4000ADF80C304EE701922BF09AFB019AADF8E9
:102E50000C0047E7624D95F88237DE0700F1A68047
:102E6000B5F83438ADF80C303CE75D4B5D49B3F94B
:102E7000C03881FB0301DB17C3EBA103ADF80C30B5
:102E800030E7574BB3F8C238ADF80C302AE7564B51
:102E9000DFED566AD3ED007A0C39C9B203EB81033A
:102EA00093ED167A67EEA67A67EE877AFDEEE77AFB
:102EB00017EE903AADF80C3014E7494B03EB4101A3
:102EC000B1F89E3803EB83035B00ADF80C3009E7E3
:102ED000434B93F8823703F00103ADF80C3001E760
:102EE0003F4BB3F85018CD055ABFCB4303F0010355
:102EF000032311F0440F18BF042311F0020F18BF71
:102F0000072311F4806F18BF0923ABE70192FEF786
:102F1000DFFF374B019A5B6C43EAC0400390E1E668
:102F20002F4BD3F84438ADF80C30DBE62C4BB3F81C
:102F30003418002934D001922BF03AFB019A80B268
:102F4000CEE62B8A03EB830303EB83039B00ADF8F0
:102F50000C30FBE6EB89ADF80C30F7E6EB89254940
:102F600003EBC3039B00A1FB03135B09ADF80C301B
:102F7000ECE6B3F80E38ADF80C30E7E66B68039377
:102F8000E4E62B680393E1E6AB680393DEE6F6B272
:102F90008DF80C608DF80D00D8E6B3F810089FE6A8
:102FA000D3F84C0880F3100080B299E605F61805B6
:102FB000019223F067F8D5ED037A019AFCEEE77AE7
:102FC00017EE903A9BB200287FF44CAF0A4909688B
:102FD00011F0100F18BF002344E700BF50D10020AC
:102FE00038C90020676666668CD1002000007A44EC
:102FF000B43C00201F85EB516864002070B5214D62
:1030000095F8C438EA181C4692F8C8288AB11E4EB2
:1030100009225C1CA6FB04135B0803EBC303E31A41
:10302000E918DCB291F8C81809B1013AF1D185F874
:10303000C44802681549561C06600C2616700268C2
:10304000561C0660002616700268561C066003EBCC
:10305000430603EB8603147019440D2246F07CFCF2
:1030600095F8C418084B4A1CA3FB02035B082944CB
:1030700003EBC3030120D31A81F8C80885F8C438CC
:1030800070BD00BF38C90020398EE3380CD2002053
:103090002DE9F041684ED6F8E47784B0044638460E
:1030A0000D460FF0F8F886F8490957B10DF10902FD
:1030B00002A938460EF021FF002840F08E8096F8D5
:1030C00049090023ADF808308DF80A301A46431E2E
:1030D000DBB20021FF20FD2B8DF80C20ADF80E1087
:1030E0008DF80B0003D9002004B0BDE8F0819DF8F5
:1030F0000830042B00F09680052B00F09980032BFC
:1031000000F09880022B00F08C80012B08BF042176
:1031100000F088809DF809309DF80A10D6F8E40781
:10312000013B0DF10E028DF809300EF04FFE96F8BE
:103130004939032B73D0042B0CD1404A9DF80A0067
:103140000121002301E012F8011F81426DD20133F9
:10315000082BF8D1D6F84C29029B394F9A420DF131
:1031600008084FD023680D22591C21601A7023686B
:103170000022591C21601A7023689DF80820591CF0
:1031800021601A7023689DF80920591C21601A706B
:1031900023689DF80C20591C21601A7023689DF843
:1031A0000A20591C21601A70BDF80E10204646F006
:1031B0001BFC23689DF80B20591C216020461A70C7
:1031C0000721FAF7BFFE98E8030087E80300012013
:1031D000C6F8545904B0BDE8F08101A938460EF094
:1031E00083FE00283FF46BAF38460DF10A010EF064
:1031F00081FE00283FF463AF019B96F8490903F074
:10320000010264E77A68D8F804309A42AAD1D6F865
:1032100054390C4AEB1A93427FF665AFA2E70A4A8B
:103220008CE703218DF8081074E78DF80A3091E7D8
:103230000121F7E70221F5E738C9002057CE06083B
:1032400084D2002080841E004FCE06082DE9F04174
:103250002A4C2B4AD4F84438B4F85879B4F84C685E
:1032600082FB0352DB17C3EBA2031FFA83F8474527
:1032700082B00D4603D1B4F85A39B34233D0026854
:103280000190511C34230160137002680023511C0B
:1032900001601370414646F0A7FB0198314646F0A5
:1032A000A3FB019847F6FF7146F09EFB019847F695
:1032B000FF7146F099FB019847F6FF7146F094FBC9
:1032C000019847F6FF7146F08FFB01980221FAF74B
:1032D00039FE0120A4F85889A4F85A69C4F85C5949
:1032E00002B0BDE8F081D4F85C39064ACB1A9342AB
:1032F000C5D8002002B0BDE8F08100BF38C9002069
:103300006766666680841E00026810B57F21541CC3
:103310000460117002680024511C01600E211470B9
:10332000FAF710FE012010BD2DE9F04FC24B1B68CB
:10333000804613F0800083B000F07181BF4B93F89A
:103340000C0810F0020000F06A81DFF810B39BF85F
:103350001430052B40F26881DBF80030B84D009343
:10336000002BB8BF5B42A5FB0342B648B649920D9D
:1033700000FB0233C3EB03139B0085FB034502EB09
:103380008202DC1702EB8202C4EBA55400FB04337B
:1033900004EB8204A4B281FB0321DB17C3EBA11170
:1033A000BCB10025A94F2E46A7FB0432D20802EB80
:1033B0008203A4EB4303E8B2A4469BB2800083409F
:1033C000BCF1090F94B246EA030605F10105EBD8FA
:1033D000340489B2B9B100259C4F2E46A7FB0132B7
:1033E000D20802EB8203A1EB4303E8B28C469BB206
:1033F00080008340BCF1090F91B246EA030605F153
:103400000105EBD83443DBF804E08D4D8D4E8E4939
:103410008EEAEE70A0EBEE70A5FB0032920D06FB7B
:103420000200C0EB0010830085FB035002EB820218
:10343000DD1702EB8202C5EBA05506FB053305EB59
:103440008205ADB281FB0321DB17C3EBA111C5B12E
:103450000020DFF8F8C10646ACFB0532D20802EBCB
:103460008203A5EB4303C7B2A9469BB2BF00BB4092
:10347000B9F1090F95B246EA030600F10100EBD855
:10348000350489B2C1B10020DFF8C0C10646ACFBEB
:103490000132D20802EB8203A1EB4303C7B2894693
:1034A0009BB2BF00BB40B9F1090F91B246EA0306D7
:1034B00000F10100EBD83543DBF80830634A019393
:1034C000002B1846B8BF5842A2FB0030604E61493D
:1034D000030AA6FB0363DB0901FB03F1C1EBD00187
:1034E00089B2B9B1002691463746A9FB0132D2080C
:1034F00002EB8203A1EB4303F0B28C469BB2800047
:103500008340BCF1090F91B247EA030706F10106B7
:10351000EBD8B9B2BBF81070DFB10026DFF82CA1F0
:10352000B446AAFB0732D20802EB8203A7EB43039F
:103530005FFA86F938469BB24FEA890903FA09F324
:10354000092897B24CEA030C06F10106E9D81FFAE4
:103550008CF7BBF812303D4AA2FB0306F608632E37
:1035600028BF6326092B63D9002093468146ABFB15
:103570000632D20802EB8203A6EB43035FFA80FA1D
:10358000B4469BB24FEA8A0A03FA0AF3BCF1090F68
:1035900096B249EA030900F10100E8D85FFA89F917
:1035A000009B019A002BCCBF392338231616BEF19D
:1035B000000F26F07F0635DD274A3343964543F05A
:1035C0000206C8BF43F00606D8F800301622581C81
:1035D000C8F800001A70D8F800300022581CC8F84B
:1035E00000001A70404646F0FFF92146404646F07A
:1035F000E3F92946404646F0DFF94046394646F0B1
:10360000F3F9D8F800305A1CC8F8002083F800906D
:10361000D8F800305A1CC8F8002001201E7003B0F2
:10362000BDE8F08F1E43CFE7002003B0BDE8F08F68
:103630004FF00009B4E700BF6864002038C90020DB
:103640006BCA5F6B806967FFD34D6210CDCCCCCC69
:10365000C55A7C0AA0860100FFC99A3B0C65002070
:103660002DE9F047AB4B1B68064613F0800084B091
:1036700000F09E80A84B93F80C0810F0020000F0B8
:103680009780A64F397D052940F29780632900F283
:1036900092800024DFF898C289B22546ACFB013243
:1036A000D20802EB8203A1EB4303E0B28E469BB249
:1036B00080008340BEF1090F91B245EA030504F191
:1036C0000104EBD8EDB2BB68954A82FB0312D9170F
:1036D000C1EB623189B2002900F018814FF0000C73
:1036E000DFF84CE26446AEFB0132D20802EB820303
:1036F000A1EB43035FFA8CF088469BB280008340C5
:10370000B8F1090F91B244EA03040CF1010CEAD8B4
:10371000E4B2FB8983494FF4F36707FB03F7A1FB8E
:103720000737C7F38F1742F20F739F4249D8CFB1C3
:103730000020DFF8FCE18446AEFB0732D20802EB42
:103740008203A7EB4303C1B2B8469BB289008B400A
:10375000B8F1090F97B24CEA030C00F10100EBD865
:103760001FFA8CF7704BD3E9002313433ED14FF07F
:10377000FF3833681722591C31601A7033680022F1
:10378000581C306039461A70304646F02DF94146D3
:10379000304646F011F933685A1C32601D703368A8
:1037A0005A1C326030461C700621FAF7CBFB012010
:1037B00004B0BDE8F087992585E7002004B0BDE896
:1037C000F0870021DFF868C10F46ACFB0302D20886
:1037D00002EB8200A3EB40039BB28B400431102923
:1037E00047EA030793B2F0D1BFB2BBE701A846F0A6
:1037F00017FD9DF80810002900F08A804FF0000C9A
:10380000DFF82CE1E046AEFB0132D20802EB820386
:10381000A1EB43035FFA8CF089469BB280008340A2
:10382000B9F1090F91B248EA03080CF1010CEAD88A
:103830004FEA08289DF80910E1B10020DFF8F0E018
:103840008446AEFB0132D20802EB8203A1EB4303B4
:103850005FFA80F98A469BB24FEA890903FA09F3B5
:10386000BAF1090F91B24CEA030C00F10100E8D85B
:1038700048EA0C089DF80A104FEA0828E1B1002038
:10388000DFF8ACE08446AEFB0132D20802EB8203E3
:10389000A1EB43035FFA80F98A469BB24FEA89099C
:1038A00003FA09F3BAF1090F91B24CEA030C00F1E3
:1038B0000100E8D848EA0C08BDF80C301B49632B1E
:1038C000A1FB03214FEA08184FEA51117FF651AFCF
:1038D0000020DFF85CE08446AEFB0132D20802EB48
:1038E0008203A1EB43035FFA80F98A469BB24FEA59
:1038F000890903FA09F3BAF1090F91B24CEA030CF2
:1039000000F10100E8D848EA0C0832E70C4600E76D
:1039100088468FE76864002038C900200C650020C5
:1039200089B5F814D34D621098D200201F85EB5151
:10393000CDCCCCCC08B5A0F10103B3FA83F30228B7
:103940004FEA531301D0184608BD0F2022F0A8FA01
:1039500030B9064B93F8823703F00103184608BDCF
:10396000BDE808400F2022F029BB00BF38C9002065
:10397000014B1B681B6A184744590020024B18680A
:1039800008B183691847704744590020024B1868F2
:1039900008B14369184770474459002010B5074CD7
:1039A000606D40B13AF0A8FF94F8513013B180F047
:1039B0000100C0B210BD012010BD00BF481D002095
:1039C00030B40A490A480A78531CDBB20525042B97
:1039D00000EBC20400F8325008BF00234FF4045239
:1039E0000B7062604FF0FF3030BC7047D46900202C
:1039F000D8690020037870B4FBB10446C0F1010619
:103A0000A31914F8015FDBB2002DF9D101335B007B
:103A1000DCB2032513800C704D7004785CB1022376
:103A200000255A1CD2B2CC548D5410F8014F0233E9
:103A3000DBB2002CF5D170BC704702242346E8E7C6
:103A40000B0617D401EB810300EBC30310B400EBAA
:103A500081000124002283F8764383F8741383F8ED
:103A60007523426D5DF8044B136843F40013002086
:103A70001360704701F07F0101EB810300EBC3038A
:103A8000012200EB810083F81C1183F81E2183F8CA
:103A90001D2182691368002B01DA43F0804343F44F
:103AA000001313600020704770B501F07F0505EB2F
:103AB000850400EBC404282101FB05010126C4F89C
:103AC00030310023C4E94A2284F81C5184F81D6176
:103AD000C4F8343101F58E711DB9FDF715FE0020D3
:103AE00070BDFDF785FE002070BD00BF2249F8B50E
:103AF000D1F868390F2B04D05A1CC1F8682900206E
:103B0000F8BD1E4C25780023C1F86839002DF6D188
:103B10001B4E1C4B3268B2F5006F17D01B689A42DF
:103B200027D017D9C2F50063402B15D9403B02F1CD
:103B30004005C1F86C3901232370356092B24023EF
:103B400011490A448121FFF7AFFFD8E71B683560B0
:103B50007BB12A469B1AE7E74FF0000502EB03070B
:103B6000C1F86C590CBF02210121376092B221705B
:103B7000E6E700232370C2E738C900201C26002096
:103B8000F0250020F425002020260020AEE700BF0D
:103B9000F8B51D4C2378012B03D0022B09D000204F
:103BA000F8BD01461948D0F86C3953B9237000208C
:103BB000F8BD00231A468121FFF776FF002323700A
:103BC000F5E7402B11D9124C2268403B02F1400529
:103BD000C0F86C39256092B240230E4C084622444E
:103BE0008121FFF761FF0020F8BD094D2A684FF0E1
:103BF000000603EB0207C0F86C6908BF02202F60C3
:103C000092B208BF2070E8E71C26002038C90020C7
:103C1000F02500202026002038B5134602250A464C
:103C2000C0E94E3380F811510021FFF73DFF00201D
:103C300038BD00BF10B50C7814F0600413D0202CF0
:103C40000AD14B78023B092B18D8DFE803F01B217F
:103C5000171717171717272E22490122FFF7DCFF26
:103C60000024204610BD4B78062B24D00A2BF3D01D
:103C70001D4B8A78C3F87829204610BDFAF7A6FEB6
:103C80000224EEE719490122FFF7C6FF0024E8E706
:103C900017490122FFF7C0FF0024E2E74B88124AD0
:103CA0001B0AC2F874390024DBE70F4B8A78C3F88B
:103CB00070290024D5E74B881B0A222B0CD0212B1E
:103CC00004D021462246FFF7A7FFCAE7CA88094960
:103CD000092A28BF0922F6E7CA880749362A28BFD9
:103CE0003622F0E7B0D2002038C90020ACD2002044
:103CF000A8D20020860D00203C0D002038B501EB35
:103D0000810400EBC4040D46002184F87453C4F808
:103D10008C1384F87513C4F88833C4F88023C378EF
:103D20002821012B01FB050108BFEDB201F55D71F2
:103D300008BFC4F884231DB9FDF7E6FC002038BD98
:103D4000FDF756FD002038BD144B9A6870B5044647
:103D500062B1134A1B7B92F87C592B4316D0812108
:103D60002046FFF76DFE022D09D070BD0C4B93F875
:103D70007C5981212046FFF763FE022DF5D12046B4
:103D8000064ABDE870401F230121B7E70121FFF774
:103D900057FE20468121BDE8704051E6B4690020FD
:103DA00038C9002070B5094A094D1173094B1360D9
:103DB0000021044629700D238121FFF775FE20465E
:103DC000054ABDE870401F23012197E7146A0020CF
:103DD000086A002055534253B469002010B5064BC1
:103DE000597B0446FAF700FE002800DB10BD204690
:103DF0000121BDE81040D5E7B46900202DE9F0416C
:103E0000314D2C7834B1012C01D1FFF7E7FF0020B0
:103E1000BDE8F0812D4FDFF8D080B0F8B4337A6878
:103E2000C8F804201F2BBA68C8F80820064606D137
:103E3000274B3A689A4202D1797B01291AD9254A3F
:103E400025491378052401F8334001EBC300013301
:103E5000DBB2042B08BF00234FF4005113701F4B3B
:103E600041600222304683F87C29FFF76DFF002075
:103E7000BDE8F081BB7B013B0F2BE0D8FAF7B4FD26
:103E8000002819DB2B78013B022BC0D9144B198871
:103E9000B1B1BB68D8F8082088F80C408B4228BF25
:103EA0000B46D11A0424C8F808100E4A2C7030466C
:103EB0008121FFF7F9FDAAE73046FFF745FFA6E7A6
:103EC0003046FFF76FFFA2E7086A0020B4690020C0
:103ED00055534243D4690020D869002038C90020D6
:103EE000FC690020788C0020146A002008B5084B7B
:103EF0001B78022B07D0033B012B02D80021FFF7D0
:103F000051FF002008BDFFF769FF002008BD00BF7A
:103F1000086A002010B501EB8101084A00EBC101DD
:103F20000446B1F88C131046F4F7A8F9034A20466A
:103F300040230121FFF7E2FE002010BDB8D200208F
:103F4000E8E700BF70B50A7812F060050C46064637
:103F500011D0202D16D1CD88D5B113062AD52A46E9
:103F60001F496078F4F7B4F9E2881D493046FFF73D
:103F700053FE00250AE04B780A2B16D00B2B0ED0EF
:103F8000062B03D13046FAF721FD0225284670BDE5
:103F9000022260781144F4F79BF9284670BD8B78B3
:103FA000D3B9104BC3F8C059F0E70F490122FFF70E
:103FB00033FEEBE70D4964780A4AC1F8C840032193
:103FC000C0E9E45542F8045B2B4680F8111100214A
:103FD000FFF794FE0025D9E7FAF7F8FCD6E700BF13
:103FE0003CC9002038C90020F8D200202C0C002049
:103FF0000B7803F00303012B03D0022B04D0002025
:1040000070478B881BB915E68B88832BFBD099E70B
:1040100010B50223044640228121FDF7F1FA204623
:10402000022340220121FDF7EBFA822120460323DF
:104030000822FDF7E5FA064B02229A80F4F796F97A
:10404000044A204640230121FFF758FE002010BDFE
:10405000B0010020B8D2002038B509220D46044630
:1040600003238321FDF7CCFA29462046FFF7D0FF32
:10407000002038BD82B00023016801930B690193D1
:104080000E4B03E00A690192013B13D0019A002A0A
:10409000F8DA019A094B42F001020192019A0A6191
:1040A0000A69019203E00A690192013B02D0019A78
:1040B000D207F8D4002002B0704700BF400D0300C3
:1040C000436D064A1A61C278012A06D100F2CC502B
:1040D00058614FF0802219681A6070471800086014
:1040E00010B5002304220446194680F811211A460F
:1040F000FFF7DAFC2046FFF7E3FF002010BD00BF0A
:1041000010B5044629B990F81131032B0DD00020C9
:1041100010BDD0F8E4359B69002BF8D090F812213F
:10412000032AF4D19847002010BDD0F89013D0F89E
:104130007C33994214D9C078D4F880230128A1EBAC
:10414000030104BFD218C4F880238B4228BF0B465A
:10415000C4F890139BB220460021FFF7CFFDD6E7AD
:10416000D0F8E4351B691BB190F81221032A03D063
:104170002046FFF7B5FFCAE79847F9E7F0B50121F8
:1041800090F8D17590F8D36590F8CFC590F8CE55DA
:1041900090F8D03590F8D22580F8111190F8CC1510
:1041A00085B005EB0C2503EB072302EB062201F09B
:1041B0001F06AFB292B290F8CD558DF808109BB2A1
:1041C000012E0446ADF80A70ADF80C30ADF80E20A3
:1041D000C0F840218DF8095017D0022E1FD036B1FB
:1041E00001F08001FFF72CFC002005B0F0BD092D87
:1041F0000FD8DFE815F0BF00AC000E00D5000E00B0
:10420000EA0085000E007700540090F81221032A7E
:104210002FD02046FAF7DAFB002005B0F0BD01F000
:1042200060012029DAB234D0012D00F02081032D65
:1042300000F00681002DD7D190F81211022900F06C
:10424000DF800329E5D11B0600F14B8102EB8202DE
:1042500000EBC20393F87633002B00F04D81BF4B87
:104260000122C3F8D429BE4920460222FFF7D4FC1C
:10427000BAE7DAB2012ACCD8D0F8E43502A99B68B3
:104280009847BDF80E30002BAED12046FFF728FF2F
:10429000AAE7D0F8E43502A99B689847A4E7F9B2E9
:1042A000AE4D012985F8C419B3D890F81231022B0C
:1042B00000F02781032BACD1002900F0868190F813
:1042C00010110129E1D0D0F8E4355B68984795F8E2
:1042D000C41984F810112046FDF700F92046FFF7B5
:1042E000FFFE81E7012A94D190F81231022B00F0F1
:1042F0001781032B8DD100F58871FFF78DFC73E7D3
:104300003D0A022DADF8062000F05081032D00F08B
:104310000B81012D7FF47DAFD0F8EC3580781B68E0
:104320000DF106019847BDF80620002A3FF45CAF66
:10433000BDF80E30002B3FF457AF9A4228BF1A4603
:1043400001462046ADF80620FFF766FC4CE790F8E2
:104350001231023B012B3FF65CAF012F7FF444AFDB
:10436000D0F8E43500229B68C0F8182102A9204645
:1043700098478AE790F81231023B012B3FF649AF8C
:10438000764BD0F818210021C3F8CC1912B10222C3
:10439000C3F8CC29734920460222FFF73DFC23E7EE
:1043A000012F00F09880022F7FF41EAF13F0FF0F53
:1043B0007FF41AAF02691B0A023B5268032B00F21A
:1043C0001D81DFE803F0393531241A437FF421AF32
:1043D00090F81231032B3FF41CAF036907F07F05FF
:1043E00080F81451196867F30A120A431A60FFF73C
:1043F00077FE002D00F0E580022384F81231F3E609
:1044000051063FF4F1AE1146FFF71AFBECE6052327
:1044100063F30612514B012184F816112046C3F8AC
:10442000D029FFF75DFEDFE6042363F30612F1E710
:10443000032363F30612EDE7022363F30612E9E7B1
:1044400090F81231022BDBD0032B7FF4E2AE27B9B8
:10445000550602D01146FFF7F3FAD4F8E43502A965
:104460009B68204698472046FFF73AFEBCE690F846
:1044700012110229C4D003297FF4CBAE002F7FF4A0
:10448000B3AE12F07F013FF400AF180600F1A78031
:1044900002EB820304EBC30304EB810083F8767321
:1044A00083F8741383F87573282303FB0243416D6B
:1044B00003F55D73DA780B68023A6FF35553012AFE
:1044C000D4F8E42598BF43F080530B6020469368EE
:1044D00002A99847D9E6D0F8E435C0F818719B686E
:1044E00044E702F07F0202EB820200EBC20393F882
:1044F0001E31002B7FF4B3AE184B0022C3F8D42931
:10450000B1E600293FF4C1AE0121032380F8101168
:1045100080F81231FCF7E2FF2046FFF7E1FD63E689
:104520001149FFF779FB5FE6FDB2052D3FF671AE4D
:10453000DFE805F0342C241C0B03D0F8EC35807830
:104540009B690DF106019847EDE6D0F8EC358078CF
:104550005B690DF106019847E5E600BF38C9002008
:104560000CD3002004D3002000D30020D0F8EC3579
:1045700080781B690DF106019847D4E6D0F8EC3538
:104580008078DB680DF106019847CCE6D0F8EC3571
:1045900080789B680DF106019847C4E6D0F8EC35A9
:1045A00080785B680DF106019847BCE6D0F8E435E9
:1045B00080789B6A0DF1060198474570C4F8F005B4
:1045C000B1E6012384F812310EE60222D0F8E43578
:1045D00080F8101180F812215B68984755E6282270
:1045E00002FB014304EB810083F81E7183F81C1168
:1045F00083F81D51816903F58E735BE7012363F333
:10460000061207E770B5044649B990F81131022B3C
:104610001BD094F81631012B0DD0002070BDD0F8BE
:10462000E4355B69002BF8D090F81221032AF4D10D
:104630009847002070BD2A4A2369D2F8D0295A60D1
:10464000002384F81631002070BDD0F83831D0F83E
:104650002451AB4217D9C278012AD0F82821A3EB04
:10466000050308BF5219C0F8383108BFC0F8282127
:104670009BB20021FFF718FA00231A46194620467C
:10468000FFF73CFBC5E7D0F83C31B3FBF5F605FB83
:10469000163666B99D420AD8D0F84021934206D218
:1046A00033463246FFF700FAC4F84061E4E7D4F835
:1046B000E435DB681BB194F81221032A0CD00023E7
:1046C000052284F8112119461A462046FFF716FBE9
:1046D0002046FFF7F5FC9CE720469847EFE700BF30
:1046E00038C9002082B000230193019A094B42F09F
:1046F00010020192C168019A0A610A69019203E0FD
:104700000A690192013B02D0019AD206F8D4002036
:1047100002B07047400D030082B000230193019A5C
:104720000B4B42F020020192019A61F38A1201922E
:10473000C168019A0A610A69019203E00A6901925B
:10474000013B02D0019A9206F8D4002002B07047D3
:10475000400D0300F8B50B7813F060050C460646D3
:104760001CD0202D17D14A78FE2A44D0FF2A3DD1F3
:104770004A88002A56D1CD88002D53D11B0651D42A
:104780003749384B0D70012183F87C19364A1F23B5
:10479000FFF7B4FA00E000252846F8BD4B780A2B55
:1047A0004BD00B2B44D0012BF6D191F904308988E2
:1047B000002B47DBFFF796FF21792A4F3046FCF7A5
:1047C000BBFE0223217940223046FCF719FF97F8FF
:1047D0007C39022B3BD094F90420002ADCDA012B2F
:1047E000DAD030460121FFF7DDFAD5E70225FAF7E6
:1047F000EDF82846F8BD4D88A5B9CC88012C11D11B
:104800001A060FD5194B1B689B6998471549C0B20A
:1048100081F8D80930B1224601F6D8113046FFF7A9
:10482000FBF9B9E730460225FAF7D0F82846F8BD7B
:104830000C4B4A8883F8D929AEE70D490122FFF7CE
:10484000EBF9A9E701F07F01FFF766FFB4E7304617
:104850008121FFF7F5F8002387F87C399CE700BF3A
:10486000086A002038C90020B4690020F8690020D7
:1048700011D3002038B50446FCF794FE20460223ED
:1048800040228121FCF7BCFE204602234022012168
:10489000FCF7B6FE0C4B0D491B680D4A00250D7048
:1048A0001B6882F87C59284698472046FFF71AFF74
:1048B00020460121FFF730FF064A20461F23012131
:1048C000FFF71CFA284638BDF8690020086A002066
:1048D00038C90020B4690020012905D008B503219A
:1048E000FFF71AFF002008BDFFF752B900B583B0EB
:1048F00009238DF80730FDF733F88DF807009DF890
:104900000730012BF7D09DF8070003B05DF804FBDA
:1049100082B0064B002201920193019B03EB8000C1
:104920000190019B186802B0704700BF50280040FA
:1049300082B0064B002201920193019B03EB8000A1
:104940000190019B196002B0704700BF50280040E1
:104950000023C0E90033C0E90233C0E90433C0E9F1
:104960000633C0E90833C0E90A33C0E90C33836376
:10497000704700BF0B6870B4D1E90524CD682B43A4
:104980001343D1E9072523431343D1E909422B43BC
:10499000D1E90D652343134304680B4A3343224096
:1049A0002B4313430360D1E90B3442690D6922F0B4
:1049B000070223431343D1E9014243614560846008
:1049C00070BCC260704700BF3F801CF0026836496F
:1049D000002310B422F00102212488420260036007
:1049E00043608360C3600361446138D02F4B9842B9
:1049F0002ED02F4B98423CD02E4B984240D02E4B7D
:104A0000984232D02D4B984241D02D4B984246D0FF
:104A10002C4B984217D02C4B98423CD02B4B9842B1
:104A200016D02B4B984224D02A4B984228D02A4BA0
:104A300098421AD0294B984229D0294B98422ED01F
:104A4000284B984208D14FF03D5243F8AC2C03E07C
:104A50004FF4746243F8202C5DF8044B7047224BEE
:104A60005DF8044B3D229A607047204A43F8642C5D
:104A7000F2E74FF474125DF8044B43F8382C70479A
:104A80004FF074625DF8044B43F8502C7047184A9D
:104A900043F87C2CE0E73D2243F8082CDCE7154A7C
:104AA00043F8942CD8E700BF106002402860024011
:104AB00040600240586002407060024088600240DE
:104AC000A0600240B86002401064024028640240C6
:104AD00040640240586402407064024088640240AE
:104AE000A0640240B8640240006002403D00002023
:104AF000400F002000003D200B88F0B433BB028C37
:104B00004C880E898B88C98822F001021204120C8D
:104B10000284058B028CADB225F0F30592B22B43D3
:104B200022F00A0243EA061322439BB242F001023A
:104B300003830284038B23F00C031B041B0C0383ED
:104B4000038B9BB21943F0BC01837047042B048C88
:104B50002CD0082B4E888A880D89C98851D024F41E
:104B600080542404240C0484838B078C2C0344EA93
:104B7000022440F6FF421A4045F6FF733B4043EAE9
:104B8000063322439BB292B243F480538283038460
:104B9000828B22F440621204120C8283838B9BB2BC
:104BA00043EA01239BB2F0BC8383704724F01004D6
:104BB0002404240C4D880F898A88C9880484068BB4
:104BC000038C12029BB242EA073423F0A00340F6A2
:104BD000FF42324043EA051322439BB292B243F0B4
:104BE000100302830384028B22F440621204120C2D
:104BF0000283038B9BB243EA01239BB2F0BC038385
:104C0000704724F480742404240C0484848B038C63
:104C1000A4B29BB224F0F30423F42063224343EABA
:104C2000062342EA05129BB243F4807392B2828358
:104C30000384838B23F00C031B041B0C8383838B63
:104C40009BB21943F0BC8183704700BF214A03889F
:104C500090429BB212D002F5806290420ED0B0F129
:104C6000804F0BD0A2F58032904207D002F58062CF
:104C7000904203D002F58062904203D14A8823F02B
:104C800070031343144A904218D002F58062904298
:104C900014D030B423F440730C894D6802F56C4293
:104CA0009BB2234390420C880380C56204850DD1DA
:104CB0008B7A0386012330BC8382704703800B8884
:104CC0004A68C2620385012383827047034B98427E
:104CD000EED0EFE70000014000100040000401406A
:104CE000024A536A23EA00005062704700380240CB
:104CF000024A136A23EA000010627047003802403B
:104D0000484B98422ED0B0F1804F32D0464B98425B
:104D100036D0464B98421ED0454B984237D0454B33
:104D200098423BD0444B98423FD0444B98424BD0A2
:104D3000434B984240D0434B98424CD0424B984210
:104D400051D0424B984256D0414B98425AD0414B99
:104D500098425ED07047404A136A43F004031362DE
:104D60000420C5E73C4A536A43F001035362012023
:104D7000B6E7394A136A43F0010313620120B7E72B
:104D8000354A136A43F0020313620220B0E7324A45
:104D9000136A43F0080313620820A9E72E4A136A36
:104DA00043F0100313621020A2E72B4A136A43F06A
:104DB0002003136220209BE7274A536A43F4803381
:104DC00053624FF480308BE7234A536A43F0020367
:104DD0005362022084E7204A536A43F4003353624B
:104DE0004FF400307CE71C4A536A43F4802353623B
:104DF0004FF4802074E7184A136A43F040031362AB
:104E0000402075E7144A136A43F080031362802040
:104E10006EE7114A136A43F4807313624FF4807093
:104E200066E700BF000001400004004000080040A9
:104E3000000C00400010004000140040000401403D
:104E4000004001400044014000480140001800407B
:104E5000001C00400020004000380240224A9368B5
:104E600003F00C03042B10B421D0082B22D01F4BCD
:104E700003601D4C1E4AA168C1F30311114491F84F
:104E80006C11CB404360A168C1F38221114491F8B9
:104E90006C1123FA01F18160A1685DF8044BC1F344
:104EA00042310A4492F86C21D340C3607047114BE1
:104EB0000360DEE75468516852686302C2F38812E7
:104EC0004CBF0C4B094B01F03F01B3FBF1F303FB6B
:104ED00002F3054A5268C2F3014201325200B3FBA9
:104EE000F2F30360C5E700BF003802400024F4007D
:104EF0002C0C002000127A002DE9F04700230F68E7
:104F000001264FF0030C02E00133102B41D006FACA
:104F100003F232EA0704F7D1D0F800E05C000CFAA3
:104F200004F52EEA050EC0F800E091F80490D0F8E0
:104F300000A009FA04FE09F1FF394EEA0A0EB9F1A0
:104F4000010FA846C0F800E06FEA050515D8D0F8B3
:104F500008E005EA0E0585604D79D0F808E0A54027
:104F600045EA0E058560456825EA020242608A79B5
:104F700045689A4092B22A434260C26822EA080217
:104F8000C260CA79C568A24001332A43102BC260AF
:104F9000BDD1BDE8F0870D4B93F88227D20703D52A
:104FA000012283F8DA29704793F8DA2962B9D3F835
:104FB000E4274AB193F87827104493F8792783F8C7
:104FC0007807114483F87917704700BF38C900206B
:104FD00010B50E4C40F0080284F8802194F9CE20E0
:104FE000022A06DD420704D583071CBF012384F88B
:104FF000D63005210648FCF7C1FD062184F8810161
:10500000BDE810400248FCF7A1BD00BF2C0C0020F9
:10501000A80D002010B5FCF749FDA8B31B4C94F96E
:10502000CE30012B30DD59B3022B2DD094F8D63081
:105030009BB971B180230521154884F88631FCF7AE
:105040009DFD062184F88701BDE810401048FCF75B
:105050007DBDBDE810400420BAE7002914BF002040
:10506000042094F8D1301A0748BF40F002005B07D3
:1050700001D411B108B940F00100BDE81040A7E724
:10508000022BD3D10420ECE710BD00BF2C0C002074
:10509000AE0D0020F8B5224C04F5C477030A84F85D
:1050A0008D0105460621384684F88C31FCF766FDF3
:1050B00094F8D13084F88E01DB072AD4B4F8D220DA
:1050C000AA4226D1174DD4F88831C5F8DB39C3B2CE
:1050D00085F8E13941F26F714FF6FF738A4218BFCC
:1050E0000123134405F6DB16C3F3072206213046DD
:1050F00085F8DF2985F8E039FCF740FD072185F8C0
:10510000E1093046FCF722FD052104F28F10FCF77F
:105110001DFDBDE8F84004480721FCF717BD00BF9E
:105120002C0C002038C90020B40D002008B5FCF775
:10513000BDFC48B1A1F59C53083BB3F57A7F03D27F
:10514000BDE808400846A5E708BD2DE9F0476B4ECD
:105150003368002B3AD06A4D6A4C05F1CE073068AF
:1051600035F016FB002833D1674B198809291D46F5
:1051700009D95F8864227A43B2FBF1F2452A40F3F1
:10518000A4811880588094F8193A012B00F0C88146
:10519000022B00F0E38133B95C480521FCF7D6FC13
:1051A000012384F8193A5A4B1D685A4B1B78002B7F
:1051B00000F0DE81584B1B68EB1A782B40F2D88147
:1051C000D4F8FC07F9F7D0FBC4F81C5ABDE8F08707
:1051D000306835F0D5FA94F8E2398046052BBED810
:1051E000DFE803F00309171D3745AA28B7D10123CB
:1051F00084F8E239B3E7552803D1022384F8E23971
:10520000ADE7414A938801339380002384F8E23963
:10521000A5E7032384F8E30984F8E2399FE713281C
:1052200084F8E409C4F8FC0907DD374AD388013360
:10523000D380002384F8E23991E718B9052384F874
:10524000E2398CE70023C4F8003A042384F8E239F9
:1052500085E7D4F8003AE218013382F8E509D4F87A
:10526000FC29C4F8003A93427FF479AFE6E7D4F81A
:10527000FC392A4803F1020A4FFA8AF1FCF77EFC56
:10528000804594F8E39940F01781262020F096FE9F
:10529000204B48B100221A701B4A538801335380B7
:1052A000002384F8E2395AE71A784A4519D10022D6
:1052B0001A7009F1FF33102B00F2F980DFE813F0C8
:1052C00030008E008E00E1008E00F700F700F7003E
:1052D0003000F700F700F700F700F700F700F700DD
:1052E0003000B9F1090F02D0B9F1110F01D1012A33
:1052F000DDD0054A538901335381DAE7786900200C
:105300002C0C002038C900209C690020BB0D002017
:1053100018260020AA690020AC6900201BD30020B9
:10532000BAF1060F5ADDB9F1010F06D0B9F1090F34
:105330000CBF4FF002094FF0030994F8E80994F804
:10534000E91994F8E72994F9E5E994F9E7C994F89B
:10535000E63985F8CE9041EA002109B2900785F838
:10536000CFE085F8D1C0A5F8D21006D512F00C0F09
:1053700014BF0122002285F8D620B9F1030F13D102
:10538000BAF1090F2ADD94F9EB29082AA8BF0822EF
:1053900022EAE27285F80421002043B29A4200F129
:1053A00001005CDC94F8EA39D4F828A00020024619
:1053B0009BB2524590465ADB7D4B85F8D0001B7856
:1053C000232B0BD109EB89037A4A03EB83030CEB04
:1053D00083031380A2F802E09180D0807649774859
:1053E0000A2257F0C0FB10B1002384F80E3A724B2A
:1053F0003A681A607A685A603A891A8194F80E3AC3
:1054000043BB95F8D63094F8782784F8102A002BFF
:1054100014BF0223012384F80E3A95F8D13094F892
:105420007A0784F8140A13F001031CBFB2FA82F35E
:105430005B0994F8792784F8112AD9B2B4F87C274B
:1054400084F80F1AA4F8122A13B10AB1A4F8162A84
:1054500084F8181A0DF052FB0DF050FB1CE704EB1A
:105460004308234493F8ED39A8F8EA3795E704EBAD
:1054700048080132B8F82C8052B2984508BF10464F
:1054800097E7BAF1040FA9DD94F8E52994F8E63915
:1054900043EA022359041AB204D5C3F30D03A5F855
:1054A000D4309BE7002AF8DBA5F8D23096E7444ACF
:1054B000938901339381EFE619F0010F7FF4F0AE89
:1054C0003F4A138901331381EAE63E4BD3F8942116
:1054D000B3F89811012A1AD141F25632914203D100
:1054E0004FF0FF32C3F89421D3F89421306802EBD7
:1054F000820202EB820201EB420189B2A3F8981109
:1055000003681B69984700232B806B803BE60132C0
:10551000EAD1B1F5965F04BF0122C3F89421E3E715
:10552000284D95F9CE60002E3FF43DAE022E11D1EC
:105530004FF48040FFF7AEFD84F8196A95F9CE303C
:10554000012B7FF730AE95F8D130C3F3400385F8D7
:10555000D63028E6032384F8193AEFE7194BB3F85D
:10556000D430002B3FF41FAE032384F8193A1AE617
:1055700094F8402094F841309A4204D0FDF766F93F
:10558000C4F81C5A22E6D4F81C3AEB1AB3F57A7F19
:10559000BFF41CAE0C4B1B68ED1A952D7FF616AEB2
:1055A0000A480521FCF7D2FABDE8F047FDF74EB9ED
:1055B000F9420020FC4200203CD30020FA0C0020DD
:1055C0009C6900202C0C0020AC690020BB0D002041
:1055D00010B5134CD4F8E40700B394F8781759B118
:1055E00094F879270CF006FCB4F87C3783421ABF94
:1055F000A4F87C0701210021B4F87E2762B141F2B2
:1056000088339342B8BF13469A4205D0A4F87E3738
:10561000BDE8104045F020B80029F9D110BD00BF09
:1056200038C9002010B401440446002014F8013B9E
:1056300008225840430010F0800F08BF400083F05C
:10564000070314BFD8B2C0B2013AF3D18C42EDD1F6
:105650005DF8044B704700BF30B54FF4806085B0F3
:105660002BF046FA40B3154C90F9040094F8203A18
:10567000134A002B18BF08234FF4E1310125CDE96F
:105680000153009100234FF480612BF092FAFF2325
:10569000E067003818BF012084F8F83484F8083532
:1056A00084F8183584F8283584F8383584F8483576
:1056B00084F8583584F8683505B030BD38C9002005
:1056C000351E0108374B1B6813F000635CD02DE9D1
:1056D000F04F354B1F78B84251D3FF2856D1334B8A
:1056E00093F8DE30002B47D0DFF8D4A00022CAF8B0
:1056F000242ACAF8282ACAF82C2AAAF8302A002F05
:105700004CD00AF59F6310461446114615461646BE
:1057100003EB071BB946B3F802C09F8993F80080DA
:1057200093F901E061443A444645D3E901C738BFE3
:10573000464610337545B8BF75469B4509B212B24F
:1057400064443844E7D191FBF9F192FBF9F28AF80D
:10575000246A8AF8255ACAF8284ACAF82C0A144B2F
:10576000AAF8261A1B781149AAF8302A092B4FF0FB
:10577000000281F8DE200CD00E48BDE8F08F0E4A02
:1057800002EB0010BDE8F08F184670470020BDE81E
:10579000F08F0A4B9AF8242ADA80EDE73A46394628
:1057A000DDE700BF68640020544900202C0C002075
:1057B000F94200205CD3002030CE0020FC420020C3
:1057C00038C900200268F8B53A4E3B4CB6F9343A75
:1057D000511C01607E2111700168054603EBC30373
:1057E00084FB0302481CDC17002328600B70FF2099
:1057F000C4EB6204FFF766FF2034304BA4B20028EC
:105800004DD01B78B0F90C1023BB2D4BA1F57A724B
:105810009A4246D82B48B0FBF1F189B2284644F0B1
:10582000BDF896F857377BB128F0AAFE0146284606
:1058300044F0B4F82146284644F0B0F82846082140
:10584000F8F780FB0120F8BDB6F81018284644F0A0
:10585000A5F8EFE71C4B1F78002FD6D01B4800237C
:1058600000EB830201339289BB421144F8DB184BF1
:105870009FED186A93F8223007EE103A07EE901A5F
:10588000B8EEC77AF8EE676AC6EE077A67EEA67AD0
:10589000FCEEE77A17EE901AB1FBF7F1B5E71B784B
:1058A00013B94EF69C21B9E7074B1F78002FF8D0AB
:1058B0000146D3E738C9002067666666F95F0020B5
:1058C00017839303008793035449002070D300206B
:1058D000D42E0020000048432DE9F8434A4C42787A
:1058E00094F8BC3A02F00F05C3B9EDB92B4600217C
:1058F00084F8C01AEB1AD9B20E290BD8234493F8B6
:10590000581739B102F0F002802A4AD0902A5FD0AD
:10591000A02A0DD000273846BDE8F8830021AB420D
:1059200084F8C01AF6D8E5E784F8BC5A2B46DEE7BF
:10593000412966D081F08003042B62D90846FCF728
:1059400093FA031D0246DBB2304884F8C03A65F092
:105950005F0584F8C15AFDF70BF994F8C07A002F5F
:10596000D8D0BE1E16F0FF0024D1FF25A94602277D
:1059700056B1DFF89C80464418F8011BD4F8E40ABD
:1059800034F00AFF4645F7D1D4F8E40A494634F02A
:1059900003FFD4F8E40A294634F0FEFE3846BDE899
:1059A000F88365F07F050427022684F8C15A84F83D
:1059B000C07A3046164A4FF6FF71104412F8015B68
:1059C000491B904289B2F9D15FFA81F90D0ACFE7FC
:1059D000412914D081F08003042B10D90846FCF72C
:1059E00043FA65F06F050627042684F8C30A84F895
:1059F000C15A84F8C21A84F8C07A3046DAE7042023
:105A0000EFE7082304229FE738C90020FAD30020DB
:105A1000F8D300202DE9F047C31DDFF8348182B0B0
:105A200003F4FC7300AFD8F89865ADEB030DC7F82D
:105A300000D03268D8F8903568449A420C4698F8FD
:105A4000E83A78606D4658D0591C0DF1010203F018
:105A50000F0388F8E81A8DF800303A60A0EB0209CD
:105A6000D6E900125FFA89F9521A09F107035FFAC1
:105A700082FA03F4FC73CA45ADEB030D55D25246CE
:105A8000684657F037F833685344336052466946E6
:105A9000384643F061FFD8F89825D8F8903530683B
:105AA000117A7060C21A4A40D2B28342336088F8D9
:105AB000E92A09D00133336013F8011C984282EAC5
:105AC0000102F7D188F8E92A3B68591C39601A703D
:105AD000D7E90032D21A012A08DD00215A1C3A60A7
:105AE0001970D7E90032D21A012AF7DC2846A047FC
:105AF00000200837BD46BDE8F087B6F90C20591CD8
:105B000003F00F0343F01003002A2A46B8BF43F006
:105B1000200302F8023B88F8E81A691C3960D6E9CC
:105B200000135B1A3A606B7098E74A46684656F075
:105B3000E1FF33684B4433604A466946384643F0D8
:105B40000BFF2846A04701200837BD46BDE8F08777
:105B500038C900202DE9F04F7C4C83B0D4F898551B
:105B6000D5E900535B1B002B00AF83460D4616465C
:105B70002ADD002384F8EA3AFCF7EAF900200BEB6F
:105B800005030BF1010AC4F88835C4F884A59BF815
:105B90000050D4F894856909012940F09F8005F0F0
:105BA0000F0915F0100514D150B194F8EC2A013208
:105BB00002F00F024A4500F09A8084F8EA5A28461B
:105BC0000C37BD46BDE8F08F94F8EA0A0028D6D11C
:105BD000D2E70BF10203C4F884350BF103029BF802
:105BE0000130D4F88C05C4F884259BF80250C8F81D
:105BF0000000C218C8F804206B404FF0000C84F875
:105C0000EB3AD4F884A5D4F8883584F8EA1AA8F8D1
:105C10000850A8F80CC0A3EB0A03DDB2121AEB1D62
:105C20005FFA82FB03F4FC73AB45ADEB030D6BD263
:105C30005A465146684656F05DFF0AEB0B035A463A
:105C400040466946C4F8843543F086FED4F88C3566
:105C5000D8F8000094F8EB2A8342C8E900300AD053
:105C60000133C8F8003013F8011C984282EA01029F
:105C7000F6D184F8EB2AD4F884351B78934239D1D5
:105C8000B8F90830FA2B54D0D8F80020D4F88C3565
:105C9000D4F89415D4F84007C8E90032D4F8982510
:105CA000D4F8903553600025158195813B1D84F80B
:105CB000EA5A7D602BF0A4FB01303FD07B680BB12A
:105CC00000209847D4F89835D4F890251968012019
:105CD0000C37C3E90021BD46BDE8F08F002108461E
:105CE000FCF71AF901200C37BD46BDE8F08FD8E962
:105CF000000290E700230120B8F9081084F8EA3A7E
:105D0000FCF70AF901205BE72A465146684656F03F
:105D1000F1FE0AEB050340462A466946C4F884357D
:105D200043F01AFE00200C3784F8EC9ABD46BDE81B
:105D3000F08F002EA8D005233370A5E7D4F898255E
:105D400013680221581C10601970B7E738C9002089
:105D50000B4B93F8322812B1B3F868274AB9B3F95C
:105D6000C038084AD81782FB0323C0EBA30000B257
:105D70007047D3F84C0890FBF2F000B2704700BFB8
:105D800038C9002067666666F8B5184CC6B2054685
:105D90003146D4F8F00A34F0FFFC94F8F41AD4F841
:105DA000F00AC5F307274E40394684F8F46A34F008
:105DB000F3FC94F8F41AD4F8F00AC5F307464F4000
:105DC000314684F8F47A34F0E7FC94F8F41AD4F805
:105DD000F00A2D0E4E40294684F8F46A34F0DCFCBB
:105DE00094F8F41A4D4084F8F45AF8BD38C90020EC
:105DF00070B50C4DC6B231460446D5F8F00A34F001
:105E0000CBFC95F8F41AD5F8F00A240A4E40214646
:105E100085F8F46A34F0C0FC95F8F41A4C4085F823
:105E2000F44A70BD38C9002038B50B4C0023054634
:105E30002421D4F8F00A84F8F43A34F0ADFCD4F814
:105E4000F00A542134F0A8FCD4F8F00A2946BDE841
:105E5000384034F0A1BC00BF38C900202DE9F04320
:105E6000DFF894932DED028B99F8F54A83B00E4636
:105E70001546002C00F03982013C89F8F54A9FED67
:105E8000D88AD84FDFF874833378002B62D099F822
:105E9000F54A002C5ED135B131F092F92B68C01A69
:105EA000002880F2028499F8F64A002C40F0A6837C
:105EB00099F8F70A062840F2D781CB4A92F8A13127
:105EC00092F8A011994200F00082D2F89C1199F842
:105ED000F8CA31F8134064440130013302F5CE7240
:105EE000A4B2C0B2DBB2B4F5E06F89F8F70A53711F
:105EF00000F0D18100F2AA80B4F5806F00F0F88242
:105F000064D9B4F5A06F00F0CC823CD9B4F5A16F90
:105F100025D8601EC0B2FFF7D5FBC8B1B0F90C3070
:105F2000B24AADF8014092F82210D9F8442703EBA9
:105F3000830303EB830349089B0093FBF1F31021D8
:105F4000CDF803308DF80010684690470023337079
:105F5000002D99D103B0BDEC028BBDE8F083B4F500
:105F6000C06FF5D1B9F83438002B00F0548328F015
:105F70001FFB10220024CDF8030006238DF800201B
:105F80008DF801401FE2B4F5826F00F05082B4F545
:105F9000846F40F0358199F80C389A07D8D5B9F854
:105FA0000E38CDF803301021202204238DF8001084
:105FB0008DF801208DF80230D9F844376846002466
:105FC00098473470002D7FF45FAFC3E7B4F5067FC8
:105FD000BED8B4F5007FC0F02C81A4F50073182B57
:105FE000B6D801A252F823F0656301085363010893
:105FF00053630108536301085363010853630108A5
:10600000536301085363010853630108515F01089A
:10601000515F0108515F0108515F0108515F01089C
:10602000515F0108515F01082F63010819630108DE
:10603000196301081963010819630108196301084C
:10604000196301081963010819630108B4F5116F98
:1060500000F0E0815BD8B4F5026F00F0BF8121D978
:10606000B4F5036F00F07282B4F5046F7FF470AF83
:10607000B9F9C038D9F8442703EB83035B0010203B
:10608000CDF80330402108238DF800008DF8011071
:106090008DF802306846002490473470002D7FF45C
:1060A000F3AE57E7B4F5E46F00F07881B4F5006F14
:1060B00076D199F80C2891077FF54AAF13F0010FBC
:1060C0004B4B00F005835A6882EAE273A3EBE2735C
:1060D00003EB5303A7FB0313DB08002AACBF43F019
:1060E000004343F04043102100240822CDF8033040
:1060F0008DF800108DF80140D9F844378DF8022052
:10610000684698473470002D7FF4BEAE22E745F212
:1061100030239C4200F0B1811DD945F240239C42BE
:1061200000F0298245F250239C427FF411AFD9F848
:106130004C38CDF803301021502252238DF8023014
:106140008DF80010D9F844378DF8012068460024F6
:106150009847347036E7B4F5376F00F031826FF44A
:1061600037616318072B3FF6F3AEA4F17100C0B29C
:10617000FFF7A8FA00283FF4EBAE90F90130CDF814
:10618000033010238DF80030ADF80140D9F84437C2
:106190006846984700233370002D7FF475AED9E62A
:1061A000B4F5E26F7FF4D4AE124B93ED170AD3ED42
:1061B000007A20EE270A002420EE080A54F0C4FBDF
:1061C00010230722CDF803008DF800308DF8013040
:1061D0008DF80220D9F8443768469847347092E722
:1061E0000000C8421F85EB512C0C0020D42E00204B
:1061F0000C6500208CD1002038C90020C5B3A291C5
:1062000040F201439C427FF4A3AEB9F9343ACDF891
:1062100003301021012204238DF802308DF8001084
:10622000D9F844378DF80120684600249847347027
:10623000C8E6B4F5807F00F01481B4F5887F7FF460
:1062400087AEB9F9C238CDF80330012210238DF89A
:1062500000308DF801308DF80220D9F844376846B7
:10626000002498473470ADE60130CD4AC0B292F8B0
:10627000A91192F8A8318B4222D04B1CDBB2490005
:10628000D2F8A441C74A645A89F8F70AB4F5E06F16
:1062900053717FF42FAEC44B93ED160AD3ED007A01
:1062A00020EE270A002420EE080A54F04DFB1022AD
:1062B0000723CDF803008DF800208DF8014082E01F
:1062C000002182F8A9110123DAE7B84999F8F83AD0
:1062D000097882F8A1410133DBB201318B4289F8A0
:1062E000F83A00F087810120C1E700283FF4C7ADEC
:1062F0000378303B012B3FF6C2AD013009F6F522A1
:106300000621FFF727FC99F8F53A89F8F60A002BE1
:106310003FF4B5AD3470B2E5A4F11100C0B2FFF79F
:10632000D1F900283FF414AEB0F9023027E799F80C
:106330005737002B40F0B081B9F81008CDF80300B2
:10634000102302228DF800308DF801308DF80220E4
:1063500083E7601EC0B2FFF7B5F900283FF4F8AD3F
:1063600043680CE7D9F844389149D9F8442781FBB0
:106370000301DB17C3EBA10300241021CDF8033088
:1063800002238DF800108DF801408DF80230684628
:1063900090473470002D7FF477ADDBE5824B93EDB1
:1063A000180AD3ED007A20EE270A002420EE080A0E
:1063B00054F0CAFA102320228DF80030CDF80300E3
:1063C00007238DF801208DF802306846D9F844374C
:1063D00098473470002D7FF457ADBBE599F80C3821
:1063E0009B077FF5B5AD734AD9F844379268CDF86D
:1063F0000320102220218DF8002008228DF80110A2
:106400008DF802206846002498473470002D7FF4F0
:106410003BAD9FE528F0B4F810230922CDF8030026
:106420008DF800308DF801308DF8022015E7D9F88D
:10643000803513F0200440F0F1805F4B1B681B0691
:1064400040F13981102304228DF803408DF8044077
:106450008DF805408DF806408DF800308DF801303C
:106460004AE6D9F8FC3ACDF8033010220024012383
:106470008DF800208DF80140A5E7B9F9BE38CDF8B8
:1064800003301021302252238DF802308DF8001095
:10649000D9F844378DF801206846002498473470B5
:1064A00090E5FF20FFF70EF900283FF451ADB0F959
:1064B0000C304249D9F8442791F8221003EB8303AA
:1064C00003EB83031020490800249B0093FBF1F3A6
:1064D00005218DF80000CDF803308DF801408DF8CE
:1064E0000210684690473470002D7FF4CDAC31E542
:1064F00099F8003B0133DAB2042A00F0D08042F26E
:10650000107389F8002B03FB02F3D9F8042B002A3F
:1065100000F0C080023399F88227D207B9F85028DA
:1065200048BF0433D40748BF0A33900748BF143329
:10653000D10548BF2833540748BF6433500648BFCD
:1065400003F57A63102100240422CFE599F80C3872
:1065500098077FF5FDAC174BD9F84427D9894FF43C
:10656000F36303FB01F3A7FB03135B091020CDF8D2
:106570000330302187E5B9F9BC38CDF8033010215C
:10658000402252238DF802308DF80010D9F844379C
:106590008DF80120684600249847347012E500BF4A
:1065A0002C0C0020D00D00208CD10020544900205C
:1065B000676666660C65002068640020D42E0020A3
:1065C000FF20FFF77FF800283FF4C2AC90F90130BC
:1065D000CDF80330102170220B238DF802308DF896
:1065E0000010D9F844378DF80120684600249847F8
:1065F0003470E7E489F8F84A012038E65C4906205F
:10660000FFF708FA002389F8F60A337003B0BDECEF
:10661000028BBDE8F083D9F84C08AAE4554A99F8F2
:106620000C18538A643BC3EB4370C3EBC00388FB75
:1066300003401844DB17C3EB20230933092BA8BF01
:10664000092323EAE37303EB830311F0020F03EB47
:10665000830314BF4FF47A7000209B00C90748BF22
:1066600000F5FA60117DD9F844279BB203440B442E
:10667000042010218DF80200CDF803308DF80010B1
:106680008DF801106846002490473470002D7FF487
:10669000FBAB5FE401333EE727F072FF4EE60123D8
:1066A00089F8003B42F210732FE7347003B0BDEC61
:1066B000028BBDE8F08399F85637002B3FF448ACC5
:1066C00099F8083B032B4ED8DFE803F043392A1131
:1066D0001A6882EAE273A3EBE27303EB5303A7FBAE
:1066E0000313DB08002AB8BF43F08043FBE4D9F86A
:1066F000102B537A907AD17A03F1407303EB002385
:10670000002203EB014389F8082B10220421CDF865
:1067100003308DF800208DF801208DF802104BE435
:10672000D9F80C1B8A7D087C897A120402EB0022BE
:106730000A44591C89F8081B02EB0363E5E7D9F802
:106740000C1B4A7DC87B497A120402EB00220A44E2
:10675000EFE7D9F80C1B0A7D887B097A120402EB5B
:1067600000220A44E5E75A1C89F8082B1B06CCE7EF
:106770009D1F01080C65002030B5A0F17D03012BA1
:10678000044683B00D46104608D9214634F004F87B
:1067900015B1288804442C8003B030BD7D210192BE
:1067A00033F0FAFF019884F0200133F0F5FFEFE7B2
:1067B00030B50F4B85B0D3F8742700230446C51DB0
:1067C000ADF80E3014F8010B01920DF10E01FFF738
:1067D000D3FFA542019AF5D10DF10E0016F0EEF9A6
:1067E000019A9DF80E000021FFF7C6FF05B030BDED
:1067F00038C900207E28F8B50F4652D0324E96F8A0
:10680000AC4164B9314D95F81C1B51B11B2885F87A
:106810001C4B3DD00D2837D0012386F8AC31002029
:10682000F8BD7D284AD095F8202B1AB180F02000C1
:1068300085F8201B95F81B2B062A14D8B5F81E4B9B
:10684000511C2A440444C9B2A5F81E4B85F81B1BF1
:1068500082F8140B002BE2D10729E0D101231C4858
:1068600086F8AC31F8BDB5F81E3B1844C0F30723D9
:1068700053FA80F0FF284FF00103A5F81E0B86F8AD
:10688000AC31CCD11248F8BDA5F81E4B2046F8BD5E
:1068900090470028C0D0012320463B7086F8AC31D9
:1068A000F8BD0A4B084A0024012183F81B4B83F8EA
:1068B0001C1B3C7082F8AC412046F8BD0123084601
:1068C00085F8203BF8BD00BF2C0C002038C9002003
:1068D0004CD40020044AD2F8243B43F4DF2343F491
:1068E0008063C2F8243B704738C90020013070B57E
:1068F000094EC4B203E044F075FB013448B9E5B277
:10690000152D21463046F6D9162D04BF034B93F8BA
:10691000285B284670BD00BF5CD4002038C9002029
:1069200000B1D7E7044AD2F8243B23F4DF2323F451
:106930008063C2F8243B704738C9002070B5114C01
:1069400084B00546D4F82C0B0E462AF08FF894F844
:10695000502794F85137003A18BF01220BB142F08A
:106960000802CDE9016200234FF4964195F9000039
:1069700000911A4608212AF01CF9C4F82C0B04B027
:1069800070BD00BF38C9002010B5064C03E0D4F834
:106990002C0B33F0F5FED4F82C0B33F0F9FE002865
:1069A000F5D110BD38C9002010B50D4CD4F8303BDE
:1069B0001B791E3B012B0DD9D4F82C0B012138304B
:1069C000FFF7BCFF0023C4F8343B84F8383BBDE834
:1069D0001040D9E7D4F82C0B012133F0C9FEF1E7C0
:1069E00038C900200B2814D810B401EB4103094C1E
:1069F00001EB83032344184490F8D438934205D024
:106A00002144002380F8D42881F8C8385DF8044B6D
:106A10007047704738C90020F0B5454C94F8393BB1
:106A2000012B83B005464FD994F83A0B4149424EA9
:106A300094F83B7B421CA1FB02C1184406EB80008A
:106A400001F4FE7606EB9101521A466B84F83A2B5C
:106A50002FB1D4F83C1B04F5346291420DD06EB9CD
:106A6000364A0133A2FB031222F0010101EB52026C
:106A70009B1A84F8393B03B0F0BD314E94F8543B77
:106A800093B9304B019348F2A501123B15226F4692
:106A9000A4F8581B009384F85A2B29463846B0476F
:106AA00058B994F8393BDBE76F46384614F026FFB7
:106AB00029463846B0470028F3D094F8541B51B10A
:106AC000384614F095FEECE71B4A02EB8302566B46
:106AD000002EC5D0D2E7009E1B4A964214D9013A37
:106AE000013E41F2210512F8013F81EA032108230A
:106AF00011F4004F85EA41000ABF490081B289B212
:106B0000013BF5D19642EED1384642F06DFF0F4978
:106B1000009D6D1A152DA8BF15252A4601F11800F4
:106B200055F0E8FF94F8393B84F8855B98E700BF9F
:106B300038C90020CDCCCCCC38CE0608ABAAAAAA46
:106B4000FD2F0108A5D4002093D4002090D400206C
:106B500070B50C4E054606F68A31D52243F000FC8E
:106B60002C686C6006F68831641A182CA8BF1824AB
:106B70002960224606F53A6055F0BCFF86F8B84B0E
:106B800070BD00BF38C90020F0B58BB004461F4B64
:106B90001F4A2049009302A81F4B44F061F9266860
:106BA0000025731C2360357023682922591C21603D
:106BB0001A702368EA22591C21601A702368C822BF
:106BC000591C216002A81A7052F0CAF8471C02A989
:106BD0003A46206855F08EFF236829461F440C234F
:106BE00000E027687A1C013B22603970F9D12268E5
:106BF000511C2160137023680122991821601A70BA
:106C000023689B1B33700BB0F0BD00BF8F6A002060
:106C1000985C0708645E07085C5E070870B50C4E58
:106C2000054606F6BE31D52243F09AFB2C686C600F
:106C300006F6BC31641A402CA8BF402429602246C5
:106C400006F6FC3055F056FF86F83C4C70BD00BF90
:106C500038C9002030B50C4B0C4AC3F8BC2B83B0AC
:106C6000C822014603F6FC3503F6C13483F8C02B75
:106C700068463A22CDE9004542F06EFE6846FFF7CD
:106C8000CDFF03B030BD00BF38C90020C83E7BEA4D
:106C9000F0B53F4B3F4C1B68590583B005460AD4FD
:106CA00094F8413C0F2B14D83B4A3C4902EB830338
:106CB0001B6D8B420DD094F8403CDA072FD49B0714
:106CC00005D5D4F8440C281AB0F57A6F12D203B067
:106CD000F0BD334B0193C8223F3B6846009384F8D4
:106CE000BC2BFFF751FF6846FFF798FF14F028FE12
:106CF00003B0F0BD94F8413CD4F8480C0F2B97BF7B
:106D0000254A264902EB8303196D03681B699847DE
:106D100094F8403C6FF3410384F8403CD7E794F883
:106D2000412C1F4E1F4F01960F2A8CBF00220122BB
:106D300084F8C42BC3F3820340F6C822A6F1370CB3
:106D4000A6F13E0184F8C33B68467123A4F8C02B2A
:106D5000BA22CDF800C084F8C23BC4F8BC7B43F033
:106D6000FFFA009B3F3E9E1B684684F8BD6BFFF711
:106D700055FF14F0E5FD94F8403CC4F8445C23F062
:106D8000030343F0020384F8403C03B0F0BD00BFAE
:106D90006864002038C9002038CE0608A0680600C4
:106DA00034D50020C80032EC044BD3F86C3730EAFD
:106DB000030314BF01200020704700BF38C9002022
:106DC000AB4A38B50820002382F8A931FFF7ECFF61
:106DD000002800F08C80D2F8A4314FF480610220AA
:106DE0004FF48264198082F8A90101465C804FF457
:106DF0000020FFF7D9FF50B14B1CD2F8A401DBB241
:106E000040F2014482F8A93120F811401946994C0A
:106E100094F83138002B6CD194F83238002B40F0C4
:106E200088804FF40070FFF7BFFF50B14B1CD2F8C1
:106E3000A401DBB24FF4046582F8A93120F81150A7
:106E40001946D4F88045A50700F11881600700F1C4
:106E5000EB80894B1B681B0600F1A38000234FF4D5
:106E6000803082F8A81182F8A93182F8A131FFF7A9
:106E70009BFFD0B3D2F89C3101214FF4047082F80B
:106E8000A11118804FF40040FFF78EFF50B14B1C4A
:106E9000D2F89C01DBB24FF4007482F8A13120F8E3
:106EA000114019464FF40030FFF77EFF50B14B1CE4
:106EB000D2F89C01DBB24FF4A06482F8A13120F833
:106EC000114019464FF48020FFF76EFF38B1D2F819
:106ED0009C014FF437644B1C20F81140D9B20023B9
:106EE00082F8A01182F8A13138BD0146CAE70146F7
:106EF0007DE70120FFF758FF00288DD04FF4803048
:106F0000FFF752FFD2F8A45128B94FF4047325F8C3
:106F100011300131C9B20BB2481CC1B24FF411603B
:106F200082F8A91125F8130094F83238002B3FF4A9
:106F300078AF0220FFF738FF00283FF472AF4FF41C
:106F40000040FFF731FF50B94B1CD2F8A401DBB26F
:106F50004FF4007582F8A93120F811501946042029
:106F6000FFF722FF50B14B1CD2F8A401DBB24FF463
:106F7000C06582F8A93120F8115019464FF48010ED
:106F8000FFF712FF00283FF44CAF4B1CD2F8A401CE
:106F9000DBB245F2502582F8A93120F8115019468C
:106FA0003FE74FF40050FFF7FFFE50B14B1CD2F803
:106FB000A401DBB24FF4036482F8A93120F8114038
:106FC00019464FF48050FFF7EFFE68B1D2F8A401E4
:106FD0004B1C4FF40064DBB28D1C20F81140E9B269
:106FE00082F8A91120F813404FF48040FFF7DCFE2F
:106FF00050B14B1CD2F8A401DBB24FF4846482F888
:10700000A93120F8114019464FF48060FFF7CCFEFB
:1070100000283FF423AFD2F8A4014FF402644B1CC4
:1070200020F81140D9B219E74FF48060FFF7BCFE99
:1070300050B14B1CD2F8A401DBB24FF4807482F83B
:10704000A93120F8114019464FF40060FFF7ACFE5B
:1070500000283FF4FEAE4B1CD2F8A401DBB24FF483
:10706000887482F8A93120F811401946F1E600BF72
:107070002C0C002038C90020686400208020FFF715
:1070800093FE50B14B1CD2F8A401DBB245F230257F
:1070900082F8A93120F8115019464FF48070FFF79B
:1070A00083FE50B14B1CD2F8A401DBB245F240255F
:1070B00082F8A93120F8115019461020FFF774FE0C
:1070C00050B14B1CD2F8A401DBB24FF4E06582F85A
:1070D000A93120F8115019462020FFF765FE50B164
:1070E0004B1CD2F8A401DBB24FF4E26582F8A9315F
:1070F00020F8115019464020FFF756FE00283FF4B3
:10710000A5AE4B1CD2F8A401DBB24FF4E46582F8C3
:10711000A93120F81150194698E600BFF0B5CA4CC5
:1071200094F8503CD4F88015C4F84C0C013388070F
:1071300085B084F8503C12D411F0340F35D10907D2
:1071400094F8502C42D412F007055BD0282A00F0A6
:10715000DB80D4F848375E20984705B0F0BD70203A
:10716000FFF722FE0028E7D004F6AC06242504F63B
:107170005407F6EC017A97ED007A67EE877A284695
:10718000FDEEE77A013517EE901AC1EB411301EBE2
:107190008301C90009B2EDB2FAF738FF272DE8D113
:1071A000D4F8801511F0340FC9D04FF40060FFF708
:1071B000FBFD002840F0278194F8502C12F00301C9
:1071C00000F0FD80D4F880150907BCD54FF400709D
:1071D000FFF7EAFD0028B6D012F00305B3D19B4AB1
:1071E000B4F9C038D91782FB0323C1EBA30109B25C
:1071F0001420FAF70BFF29461C20FAF707FF94F832
:10720000502CA0E7FF20FEF75DFA002800F0018176
:107210000378FF2B00F09A8090F901100220FAF712
:10722000F5FEFF20FEF74EFA002800F0918003786B
:10723000FF2B00F08D80B0F90C20854B834893F82C
:10724000221002EB820202EB82029300490893FBB8
:10725000F1F3D91780FB0320C1EBA00001B203209A
:10726000FAF7D4FE94F83138002B79D1D4F8803570
:107270009A0640F198804FF40050FFF795FD0028E2
:1072800040F0CB80734D4FF48060FFF78DFD0028F8
:1072900040F04C816B8A94F8502C297DB3F5967F91
:1072A00002D9100740F1118194F85337002B40F0B8
:1072B000B280A1F1200307EE903A9FED677AF8EED5
:1072C000E77AF6EE006A67EE877ABEEE007AF5EEB0
:1072D000C07AF1EE10FA58BFB0EE667A77EE877A90
:1072E000FDEEE77A17EE903A19B20520FAF78EFE16
:1072F0004FF48050FFF758FD002840F0BD8094F80F
:10730000502C282A7FF425AF544A554B156855490F
:10731000A3FB0535AD09A1FB05367609A1FB0631B6
:107320004909C1EB0111A6EB81010902C6EB061662
:10733000002309B21720A5EB860684F8503CFAF723
:1073400065FE31B21820FAF761FE02E7294665E7CB
:1073500000210320FAF75AFE94F83138002B85D02B
:107360000120FFF721FD002840F0F28094F8323828
:10737000002B3FF47BAF0220FFF716FD002840F002
:1073800040810420FFF710FD00283FF46FAFB4F8F0
:107390003438002B00F0428127F00AF901B20420B2
:1073A000FAF734FE62E71B07A9D52F4B93E80300D9
:1073B00002AB83E803001846FAF73EFE9FE74FF45E
:1073C0008060FFF7F1FC00283FF4FCAE274BD4F8B7
:1073D0004C2CD4F8FC5A9A4240F2F080244BE91726
:1073E00083FB0523C1EB6313642101FB13510DB231
:1073F00019B21020FAF70AFE29462120FAF706FEF4
:1074000094F8502CDEE6B4F9C2183020FAF7FEFDED
:10741000D2E6014602E709B267E794F80C389F0705
:1074200059D44FF48060FFF7BFFC0A4D00283FF4A9
:1074300031AF002631460120FAF7E8FD3146092038
:10744000FAF7E4FD26E700BF38C9002067666666E4
:10745000D42E00200C650020E4380E3F18260020B2
:10746000D34D621089888888C8CE06083F4B4C00EF
:107470001F85EB510050C34794F80C280023920756
:10748000CDE9003347D494F8543C012B43D0B4F9F0
:107490004C375FED086A07EE103AB4F94E3707EE45
:1074A000903AB8EEC77AF8EEE77A27EE267A67EEDA
:1074B000A67ABDEEC77AFDEEE77A02A88DED027AD4
:1074C000CDED037AFAF7B8FD19E742F20F71994250
:1074D000A8BF1946E8E6544D544BE9894FF4F366CA
:1074E00006FB01F14909A3FB0131C9091120FAF793
:1074F0008DFDE9894E4B06FB01F1A3FB01214909F2
:10750000A3FB01235B09642202FB131109B21920BA
:10751000FAF77CFDB7E6D5E9002301216846CDE9FD
:10752000002384F8541CFAF787FDE8E694F80C3839
:107530009E077FF57EAFAB683D4AD91782FB0302F9
:10754000C1EB6211642606FB113636B209B272E74E
:1075500094F8511C00293DD10B460620A4F8523C5A
:10756000FAF754FDB4F8523C0133A4F8523C27F02A
:1075700013F894F8543794F8512C012B94F857379A
:107580001ED000EB800086B213B10AB1B6FBF2F652
:10759000274BA3FB062343F34F113A205D09FAF76B
:1075A00035FD642101FB1561224B89B20531A3FB36
:1075B0000131C9083B20FAF729FDD7E60D4618E747
:1075C0001BB112B1B0FBF2F080B201B23920FAF770
:1075D0001DFDCBE6B4F8520CB4F81028B0FBF1F363
:1075E00001FB1303642000FB02129BB24900B2FBB3
:1075F000F1F2110241EA0311C2F30322114309B26D
:10760000ABE7D4F844380C49DA1781FB0313C2EB1B
:10761000A30319B22820FAF7F9FCB2E6D4F84C38E3
:1076200083F3100319B2BAE60C650020C55A7C0A30
:107630001F85EB51CDCCCCCC6766666603685A06D5
:1076400007D513F4057F04D007298CBF0020012043
:10765000704703F48253B3F5825F03BFC81FB0FACB
:1076600080F040090020704770B5BC4C94F8553C40
:10767000012B84B000F04C8194F8610CFCF75AF9AE
:1076800094F8623C834205461FD0002800F0D58064
:10769000D4F8303BCBB194F8512793F90400002A79
:1076A00018BF08224FF4964100230325CDE901526B
:1076B00000911A46082129F07CFAC4F82C0B20B15D
:1076C000FFF772F9012384F8623C94F8633C012BC4
:1076D00000F0C080D4F86C6C3EB1A14B30465978B4
:1076E000FFF7ACFF002840F0F18094F8710CFCF734
:1076F00021F994F8703C8342054621D0002800F01F
